:020000040000FA
:10000000000E040000000000020C0000060C0000BE
:100010000A0C00000E0C0000120C0000160C000070
:100020001A0C00001E0C0000220C0000260C000020
:100030002A0C00002E0C0000320C0000360C0000D0
:100040003A0C00003E0C0000420C0000460C000080
:100050004A0C00004E0C0000520C0000560C000030
:100060005A0C00005E0C0000620C0000660C0000E0
:100070006A0C00006E0C0000720C0000760C000090
:100080007A0C00007E0C0000820C0000860C000040
:100090008A0C00008E0C0000920C0000960C0000F0
:1000A0009A0C00009E0C0000A20C0000A60C0000A0
:1000B000AA0C0000AE0C0000B20C0000B60C000050
:1000C000BA0C0000BE0C0000C20C0000C60C000000
:1000D000CA0C0000CE0C0000D20C0000D60C0000B0
:1000E000DA0C0000DE0C0000E20C0000E60C000060
:1000F000EA0C0000EE0C0000F20C0000F60C000010
:10010000FA0C0000FE0C0000020D0000060D0000BD
:100110000A0D00000E0D0000120D0000160D00006B
:100120001A0D00001E0D0000220D0000260D00001B
:100130002A0D00002E0D0000320D0000360D0000CB
:100140003A0D00003E0D0000420D0000460D00007B
:100150004A0D00004E0D0000520D0000560D00002B
:100160005A0D00005E0D0000620D0000660D0000DB
:100170006A0D00006E0D0000720D0000760D00008B
:100180007A0D00007E0D0000820D0000860D00003B
:100190008A0D00008E0D0000920D0000960D0000EB
:1001A0009A0D00009E0D0000A20D0000A60D00009B
:1001B000AA0D0000AE0D0000B20D0000B60D00004B
:1001C000BA0D0000BE0D0000C20D0000C60D0000FB
:1001D000CA0D0000CE0D0000D20D0000D60D0000AB
:1001E000DA0D0000DE0D0000E20D0000E60D00005B
:1001F000EA0D0000EE0D0000F20D0000F60D00000B
:10020000FFFFFF00FFFFFF00FFFFFF00FFFFFF00FA
:10021000FFFFFF00FFFFFF00FFFFFF00FFFFFF00EA
:10022000FFFFFF00FFFFFF00FFFFFF00FFFFFF00DA
:10023000FFFFFF00FFFFFF00FFFFFF00FFFFFF00CA
:10180000FFFFFF0020AA04000000000020AA04003F
:101810000000000020AA04000000000020AA04002C
:101820000000000020AA04000000000020AA04001C
:101830000000000020AA04000000000020AA04000C
:101840000000000020AA04000000000020AA0400FC
:101850000000000092670400000000006A2D0400F0
:101860000000000020AA04000000000020AA0400DC
:1018700000000000AE6704000000000020AA040081
:1018800000000000E66704000000000020AA040039
:101890000000000032460400000000007A4104000D
:1018A00000000000264204000000000020AA0400FE
:1018B0000000000020AA04000000000020AA04008C
:1018C0000000000020AA04000000000020AA04007C
:1018D0000000000020AA040000000000FE920400A6
:1018E0000000000020AA04000000000020AA04005C
:1018F0000000000020AA04000000000020AA04004C
:101900000000000020AA040000000000CA670400D4
:101910000000000020AA040000000000269304003C
:1019200000000000106904000000000020AA04006C
:1019300000000000B2410400000000006642040004
:101940000000000020AA04000000000020AA0400FB
:101950000000000020AA04000000000020AA0400EB
:101960000000000020AA04000000000020AA0400DB
:101970000000000020AA04000000000020AA0400CB
:101980000000000020AA04000000000020AA0400BB
:101990000000000020AA04000000000020AA0400AB
:1019A0000000000020AA04000000000020AA04009B
:1019B0000000000020AA04000000000020AA04008B
:1019C0000000000020AA04000000000020AA04007B
:1019D0000000000020AA04000000000020AA04006B
:1019E0000000000020AA04000000000020AA04005B
:1019F0000000000020AA04000000000020AA04004B
:101A00000000000020AA04000000000020AA04003A
:101A10000000000020AA04000000000020AA04002A
:101A20000000000020AA04000000000020AA04001A
:101A30000000000020AA04000000000020AA04000A
:101A40000000000020AA04000000000020AA0400FA
:101A50000000000020AA04000000000020AA0400EA
:101A60000000000020AA04000000000020AA0400DA
:101A70000000000020AA04000000000020AA0400CA
:101A80000000000020AA04000000000020AA0400BA
:101A90000000000020AA04000000000020AA0400AA
:101AA0000000000020AA04000000000020AA04009A
:101AB0000000000020AA04000000000020AA04008A
:101AC0000000000020AA04000000000020AA04007A
:101AD00000000000EC41040000000000A8420400E7
:101AE0000000000020AA04000000000020AA04005A
:101AF0000000000020AA04000000000020AA04004A
:101B00000000000020AA04000000000020AA040039
:101B10000000000020AA04000000000020AA040029
:101B20000000000020AA04000000000020AA040019
:101B30000000000020AA04000000000020AA040009
:101B40000000000020AA04000000000020AA0400F9
:101B50000000000020AA04000000000020AA0400E9
:101B60000000000020AA04000000000020AA0400D9
:101B70000000000020AA04000000000020AA0400C9
:101B80000000000020AA04000000000020AA0400B9
:101B90000000000020AA04000000000020AA0400A9
:101BA0000000000020AA04000000000020AA040099
:101BB0000000000020AA04000000000020AA040089
:101BC0000000000020AA04000000000020AA040079
:101BD0000000000020AA04000000000020AA040069
:101BE0000000000020AA04000000000020AA040059
:101BF00000000000FFFFFF00FFFFFF00FFFFFF00EE
:101C00002F7E22000E7F24000E01880000000000BD
:101C10000C00070060862A00010020001100070068
:101C2000000020000000E00002003200000002007E
:101C300000000000B8270200000000000040DA00A9
:101C40000000FE004440A900E08D20000000E000FC
:101C50000300320010002000A00188004440A800CA
:101C60000000060091018800800078000000EB0071
:101C700015003700E280400032A0B4009101BA00A4
:101C8000E280400032A0B4009102BA00E28040003D
:101C900032A0B4000002EB00472BDE00F507B200D3
:101CA000602CE10004003A000059EB008301E900D8
:101CB000FDFF3E00040037006128E1000100320012
:101CC0000082EB00040007001101BA000200E000EE
:101CD000E8FF3A00000006003159BA008301E9002C
:101CE0000C0032002159BA008301E90008003200DB
:101CF0000400E00003003A00E280400032A0B4009B
:101D0000F5FF370011D9BA008301E900FAFF3A0064
:101D10008100E800E180400032A0B400000006002D
:101D20002800FA00889FBE008A9FBE008C9FBE00DC
:101D300007067800878669000C003B0003047800E2
:101D40008704780008F0A10009F0A100840F50007A
:101D5000858F5800860F5900890F5C0003003300FF
:101D60000CF0A20001003A000CF0A10008020700EC
:101D70006400E1005F003200780147006408E10080
:101D8000610032006C014700748557003200BE00CC
:101D90001201BE003A04BE001A05BE001E039000E8
:101DA000BE0A90008503530006003D000004FD00BC
:101DB0008104FD000205FD008305FD008703EA00A4
:101DC000050378000DF8A30004003200600414003D
:101DD000E0841C0060051D00E0851D006022B80045
:101DE0007D0320000D38E1008006EB000B00390078
:101DF0004433DD00F300B200830173003900370083
:101E0000848272000D027800E10664008B85D100A7
:101E10000A85D3008984D3000884D3008703E900AE
:101E2000F7FF3B0008004000898048000A01490094
:101E30008B81490004003B0060001000E080180026
:101E400060011900E08119000358A3000900320065
:101E50008D82720084827200610260008301D10071
:101E60000281D3008180D3000080D3000603E80004
:101E70001B0037000348A30017003A000600E000EB
:101E8000170034000603E9000D00A300000048001D
:101E90008180480002014900838149000348A30072
:101EA0000F003A000600E000090034000603E900D4
:101EB0000000400081804800020149008381490000
:101EC00001003A000003EB000348A300F5FF3200D5
:101ED0006022B800020037008482720061826600CE
:101EE0007F01070003F0A1000CF0A70003F0A000A1
:101EF000BB013700640147006408E10002003A00BA
:101F00000DF8A300B3013A003200BE001201BE007A
:101F1000B301370003F0A200889FBE008A9FBE0075
:101F20008C1F7800A9020700B00233006450E10062
:101F30004F0032006420E1005200320003826C0046
:101F400007003B000905D0000306D000820F5400B3
:101F50000C065D00020039000200320089017800A1
:101F6000030678008582550004003D000003FD0053
:101F70008103FD008502EA008B854200840F720018
:101F800002003B0060001000E08018006011B80003
:101F90000005EB007A28E1000A003900060078000D
:101FA000C75DDD00F707B200878075002D003700A0
:101FB000828171000A017800610560008180D10092
:101FC0000080D3008502E900F9FF3B0006044000D1
:101FD0008784480002003B0060041400E0841C0079
:101FE0000988A300070032008A8171008281710094
:101FF000610164008904D1000884D3008B05E800E6
:10200000170037000978A30013003A000B00E00026
:10201000130034008B05E9000804440089844C0057
:102020000A4474000978A3000D003A000B00E00098
:10203000070034008B05E9000804440089844C0043
:1020400001003A000B0020000978A300F7FF3200DE
:102050000001EB0002003700828171000A01780064
:102060001F0207000CF0A70001F0A0006802370073
:102070006420E10002003A00838F6C0068023300A4
:102080000801BE000200BE0061023700889FBE004A
:102090008A9FBE008C9FBE000004BE00360207006F
:1020A0000800BE00890678006420E10008003900BD
:1020B000040032000160A0001202200002F7880034
:1020C0005300370091FC2300B0FD20004E00370084
:1020D0000006EB0009F0A10003F823000200200035
:1020E0000800BE006A0107000600340001F8230062
:1020F000000020000801BE00B20007000004BE007E
:102100002C0020000800BE0093E82300320A2300C0
:102110005F010700120034000801BE00D1FD23005A
:10212000703D2B007CFF07000005BE00B3F32300C9
:10213000F27A26000800BE00B102070003F823006F
:102140000200200073FF07000801BE0072FF0700B5
:102150000A01BE009B0007000004BE000C06E80058
:102160000800BE0001F0A100020020000398230037
:10217000470107000800BE00160035000801BE0038
:102180009F0207000005BE0032CD2C0043FB230058
:1021900061FF0700809FBE001269280003D52B0055
:1021A0000A00BE0096020700620F210013EF2B0009
:1021B00059FF07000A01BE00910207004F01BE004F
:1021C000800007000801BE008D0207000801BE0064
:1021D00051FF07000C00E0000B0032000C10A700BC
:1021E00001F0A200B2FD200093FC23006260E10038
:1021F0000400320022A9200063F023000C10A70085
:1022000063F8230044FF07000DF0A70001F0A200CF
:102210004F06BE004F05BE004F04BE000000060082
:102220000001EB00F3000700040032000200200070
:1022300003F8230001F0A60037FF070000000600A6
:102240000081EB00850337008F1FD1005804070081
:102250008F87E9000000E000000006002800FA0077
:10226000889FBE008A9FBE008C9FBE0003866B00C5
:10227000C70007006400E100440032006408E10088
:102280004A0032006100E100460032006108E100CE
:1022900049003200EC0647006000B8003D02BE0075
:1022A0003D03BE00F48657006011B8003D04BE0037
:1022B0003D05BE007D0320000B0037000000A0009C
:1022C0008D06E900130032000402420085824A00B4
:1022D00006034B0087834B000000400081804800CC
:1022E00002014900838149000802520089825A0094
:1022F0000A035B008B835B00F0FF3B000802420097
:1023000089824A000A034B008B834B008D06E9004B
:10231000EDFF3A008482720086827200F707B200F5
:102320008782720001003200150020001E04900018
:102330003E0B900006035400E63FB0000368A30084
:10234000070032000000A7000500A0008301D100B3
:102350000281D3008180D3000080D3000603E8000F
:102360008301D1000281D3008180D3000080D3009B
:102370000002EB000482D2005900070003F0A10024
:102380000CF0A70003F0A00095003700640247009E
:102390006408E1008F0032003400BE003401BE004A
:1023A000F6FF37006108E1008A0032006011B800D2
:1023B0006000B800F1FF370003FF27000200200093
:1023C000FBFF3700889FBE008A9FBE008C1F7800ED
:1023D0007E0107008501330003866C006450E10034
:1023E0002E0032006420E100330032006150E10031
:1023F0002F0032006120E100310032008585550058
:10240000EB07B00009002000080420000500370099
:102410000804440089844C000A003100060343008C
:1024200087834B000001530081815B00F8FF33007C
:102430000203BE000800A0000804440089844C0088
:10244000F6FF3900C639DD00830173000100320058
:10245000130020008904D1000884D3000998A30048
:10246000050032000800A7000300A0008904D10085
:102470000884D3008B05E8008904D1000884D300C8
:102480000001EB000281D2001501070001F0A1005C
:102490000CF0A70001F0A0005D0137006420E1000E
:1024A0005F0132000801BE000200BE00F7FF3700E6
:1024B0006120E1005A0132006000B800F3FF3700EC
:1024C0000000200001F82700F0FF3700801FEB001C
:1024D000B70307008F87E9000000E0000000060056
:1024E0001800200057002000080453000D003D0094
:1024F0000600200097FC2F000740E1001E0034007A
:1025000084827200610260008301D1000281D300E5
:102510008180D3000080D3000804E800F8FF3A006F
:102520004700200061046000050474000404640096
:102530000D00320061004000E08048006001490069
:10254000E081490003B8A500070032000603E80057
:102550006538E10004003A008301D1000281D30014
:102560008180D3000080D300F87F20000830E10094
:1025700003003500080378006000B8006011B8005F
:102580004433DD00F300B200830173000000060055
:10259000680447000294BE000094BE00FC0447009B
:1025A0008694BE008494BE0009007800C903070029
:1025B00008007800C703070099007800814F700079
:1025C0000B003B000800BE00A20307004F00B10053
:1025D00003003700F3FF2700F2FF2F006110B9005E
:1025E0004F06BE004F05BE004F04BE000080FA003B
:1025F00000000600889FBE008A9FBE000003BE0048
:10260000DD0007008505780082815200020020006D
:102610006220E10004003A00F307B1000400350035
:102620007718E100040035000600BE0014003700F2
:102630006000B8000F003700F50F2000FAFF2F00F0
:102640008502D1000A85D3008301E900FCFF3B002D
:102650008184620000046500890F7400F2FF32007B
:102660008582EA000A85EA00818462000004650030
:102670009B00070007F0A70001F0A0000081EB001D
:102680000200E0004F05BE004F04BE00000006003F
:102690001400200018043700F4FF2F001604370040
:1026A0000001BE00B40007000470A70003F0A10001
:1026B0006509B100160032000D0035006828E10000
:1026C00006003500F0FF2F00F1FF27000300E000B7
:1026D00013003B000100280000000500000040003E
:1026E000818048008502E900FCFF3A0008003700BD
:1026F000F88F420002003C008000EB000000050063
:102700008100D1000080D3008502E800FCFF3A0080
:102710000300E00002003B0060001000E0801800B1
:10272000000006001400FA00889FBE008A9FBE00C9
:102730008C9FBE000004BE000205BE00680047007A
:102740000A90BE000890BE00620307000070A70058
:102750000BF0A1000BF8A30016003A009E029000B7
:102760003043200080825200B0FE2F000028E1009C
:102770000D003C00B0FC2F000028E1000D003400EB
:102780001E0990008E0890007E0090000501B000A8
:102790000201D1008180D3000080D3008502E800CF
:1027A000FBFF3A008EFF37000100280000002000E8
:1027B0008BFF37006000B80089FF37000001BE00C2
:1027C0006D0007000470A70003F0A10003F8A30048
:1027D00013003A006509B10010003200090035000D
:1027E0006928E10002003500010028000000050012
:1027F00000004000818048008502E900FCFF3A00AB
:1028000000000600F88F4200050035008100D1006D
:102810000080D3008502E800FCFF3A0000000600BB
:102820008000EB00000005004F89DE008201780087
:10283000CC033700889FBE008A9FBE000105780048
:102840000100E0000400350008003C000000E0004A
:10285000200032000500370060001000E080180002
:1028600002003B0001F02C001A0037000004BE00FB
:102870006011B8006B0920000982CF000200390006
:102880000882CF000441B000694252000E003200BD
:1028900008003B0082817100610164008904D1005D
:1028A0000884D3008B05E8000442E800F9FF3A00F1
:1028B000050037000804440089844C008B05E900BA
:1028C0000442E900FBFF3A00050007000AF0A700F8
:1028D00001F0A0004F05BE004F04BE00000006003E
:1028E00081002000618055000B003D000B0020009E
:1028F00061FE2F000100E1001D00340082817100A3
:10290000610164008904D1000884D3000000E8005C
:10291000FAFF3A00710020006100640003007000BB
:10292000020060000900320061044400E0844C00B1
:102930000988A500050032008B05E8006808E10061
:1029400002003A008904D1000884D300F20F20006D
:102950000258E10005003D00C75DDD00F907B20047
:102960008980750008007800000006000BF8270039
:102970008B00780000000500C70ADE00F107B200F6
:10298000F50FB20008003200E1CF42000200320031
:102990000170A00024000500810F700001003200CA
:1029A0000408050044000500810F700002003A0091
:1029B000140005008502E9000000400081C04800C5
:1029C000FCFF3B000170A000240005000004BE00D5
:1029D000E9FF07000003BE000405BE000200BE00C0
:1029E000E5FF0700844F7500000006000200BE00EE
:1029F0006450E100050036006420E100020036006A
:102A00000968A30001003A000800BE000160A000B0
:102A10004F0678004F05BE004F04BE0000000600C0
:102A2000F0FF2F00F1FF2700F9FF37002800FA0020
:102A3000889FBE008A9FBE008C9FBE0003866B00ED
:102A4000D3FE07000028A30064003A000128A30079
:102A500067003A000008A30062003A000108A300E2
:102A600065003A001E009000BE08900081064000FC
:102A7000ED3FB100F4805700EE019000111AB8004C
:102A80008E099000311BB8009E099000311CB800DF
:102A9000511DB800F485570046000700FE01900064
:102AA0003A0007008B85E8003E0007008E09900081
:102AB00040000700EE019000340007008B85E8001D
:102AC000380007008E099000400007009E09900022
:102AD0001B18B800890440000A854800FE019000D8
:102AE000340007008B85E80038000700EE019000F5
:102AF000300007008E0990001B18B80089044000C0
:102B00000A8548000A98A30008003A00040242001F
:102B100085824A0006034B0087834B0008044C0063
:102B200089844C000A054D008D06E90084827200FC
:102B3000850273004C3ADD0085027200010032000C
:102B400015002000443ADE001400B2004538DE00D3
:102B5000CB45DD000B007000C540DE00CB4DDD0035
:102B60008B8070004549DE00CB55DD000B01710004
:102B7000C551DE000D03780059FE070003F0A100E7
:102B80000CF0A70003F0A00095FE37001B18B8005A
:102B90008502400006834800E0834B0060044C003F
:102BA000070037001B18B800060340008783480061
:102BB000FAFF37001B18B80087034000088448005C
:102BC000E0844C0060054D00000006001B18B800B2
:102BD0000804400089844800FAFF37000108A30078
:102BE0007CFE3A005800BE005801BE00E3FF3700EB
:102BF0000008A30077FE3A0009047800F9FF3700C7
:102C0000889FBE008A9FBE008C1F78006FFF070060
:102C100076FF330003866C006450E100240032002C
:102C20006420E100270032006150E1002200320000
:102C30006120E100210032008B854200EB07B100EA
:102C40000134B800003AB8000804420089844A0000
:102C5000013AB8000030B8008880400009014A00FD
:102C60000400330000004000818048000201490058
:102C70008B05E900C909DD00830170000100320005
:102C800013002000C814DE004814DD004709DE00F0
:102C90001200B200C808DE000884700010FF0700B0
:102CA00001F0A1000CF0A70001F0A00058FF3700D0
:102CB0006120E1005AFF32000801BE000200BE00A0
:102CC000F7FF37006150E100FCFF3A0054FF370086
:102CD0000C00FA00889FBE008A9FBE008C9FBE0039
:102CE0003AFF07000206BE00840578000200BE001D
:102CF000020020003FFE070005003A008B02B300EF
:102D0000120020003BFE070001003A00F8856D002C
:102D10000C01BE00C60007000800BE009B00320088
:102D20000B08A3009E003A000DF0A7000BE0A000E6
:102D300009F0A7000BF0A00009F0A1000801BE00F7
:102D4000BB0007000BF0A6009500320001003C001C
:102D50000BD0A0008ACF7500B20033006000B8002D
:102D60006250E10099003900A1003E000B28A30049
:102D7000A2003A000BF8A300060032000B58A30093
:102D8000A70032000801BE00A90007000800BE002D
:102D9000940032000800BE00780107000004BE0065
:102DA000050578000BF0A7000B30A6000BF0A10082
:102DB0005B079800324F200053F3230034FE0700D6
:102DC00005003D000800BE0012002000ED020700D3
:102DD0000004BE000A05E9004A0798006150B900E6
:102DE00094FE0700008FBE000C01BE0084FF0700A8
:102DF0002BFE0700300798000100E00002003D00B4
:102E000060001000E0801800F2FF2700820F5000E1
:102E1000E08F580064003E000C00BE0020FE07005A
:102E200020079800F2072000820F5000E08F580022
:102E300005003C0012F82F00F3FF2F00820F500016
:102E4000838F580009003D000A00E00003003200B3
:102E500001003C000201EA00020578006000B800B1
:102E6000200798003A079800190037003E009000AC
:102E70006100B9006FFE0700809FBE000C00BE001D
:102E80004109DD004811DE007208B100D9FD0700DC
:102E90000005BE001E01BE0059FF07004F01BE0025
:102EA0001CFC0700809FBE000C00BE000A01BE0093
:102EB00018FC07001E01BE0051FF07004F01BE00B5
:102EC00015FC07008221270013F323004CFF0700A5
:102ED0000005BE002E0090006100B90055FE0700FD
:102EE00001F0A2000C01BE000BFC07000006BE00B2
:102EF0000800BE00C50207000C01BE0040FF07002D
:102F00000A01BE0004FC0700809FBE004A000700C3
:102F10002E0590000AF0A7000A05EA000500370018
:102F20000800BE000801BE0035FF07000004BE0017
:102F30000C00BE000801BE000A00A70030FF070019
:102F40000006BE000A05D100F5FF3A005E019000C0
:102F500002E0A600030037000001BE0036000700B3
:102F600018FD07000004BE004F00BE0080010700EE
:102F70000801BE0022FF07003E0190008102070009
:102F8000DE0590000BF0A70001F0A2004F06BE0086
:102F90004F05BE004F04BE000080FA00000006008E
:102FA00025000700F9FF3700270007006000B80080
:102FB0000BD0A7000BC0A0000BE0A7000BC0A20025
:102FC0000BC0A70001F82700F0FF37000DF8A300A1
:102FD000020032001E000700190007000BF8A300D2
:102FE000EAFF32000B30A70001F0A200E7FF370034
:102FF0000DF8A300F9FF3A00F7FF37000801BE0003
:103000000B000700E6FF320001003C000DF0A200BB
:103010006000B8000DF0A70009000700DBFF3700D3
:103020000B000700F1FF2700F0FF2F00D7FF37004C
:103030000100070096FD370001F82300000005009D
:1030400001F82700000005002002200001003700E1
:103050001002200000F7880000000600889FBE00D4
:103060008A9FBE008C9FBE00820578000004BE00CF
:1030700041FE07000800BE006420E100070039009F
:1030800002003A00F1FF2700F0FF2F000160A000CE
:103090001202200002F78800550037006120E1008D
:1030A00003003A000B00A70001F82300500037008E
:1030B00001F0A100020021009364240074FD0700C8
:1030C0000800BE0004003500B2FD2000930C24006F
:1030D000DB0107000004BE000005EB000B00A600AA
:1030E0004F0DDE0001F0A1000004BE0032982F0059
:1030F00023EA2300C2FE07000001EB0003F02300D7
:103100000B00A70003F8230083FB070064FD070002
:103110000000A7000A00A200C6FD07000B00E000A7
:10312000030032000200200003F0230079FB0700B7
:1031300001F0A2000006BE0002002000930424005B
:10314000AFFE07000801BE0073FB0700809FBE00B2
:103150000C00BE0022A22A00D3A72300A8FE07006D
:103160004F01BE006CFB07000004BE0001F0A1008F
:10317000020020000398230045FD07000800BE0060
:10318000190035000001BE009DFE07000006BE00CC
:10319000B2C52900E362230099FE070022222B001A
:1031A000F3942B005CFB07000C01BE0094FE0700AB
:1031B000E273280083C0230057FB07000C01BE0008
:1031C0008FFE070042AA2A00A3E22B0052FB070051
:1031D0000C01BE008AFE07000801BE0088FE070041
:1031E0000801BE004CFB07000A00A70001F0A20086
:1031F0004F06BE004F05BE004F04BE000000060093
:1032000007F0A200C6FA3700889FBE008A9FBE0062
:103210000004BE00D8FD07000800BE006420E100E5
:103220000700390002003A00F1FF2700F0FF2F00ED
:103230000160A0001202200002F788004C00370055
:1032400001F0A10002802000935C240010FD070023
:103250000800BE0004003500B2FD200093042400E5
:10326000770107000004BE0032982F0023F22300EC
:1032700063FE07000200200003F0230001F0A70016
:1032800003F0A00024FB070005FD0700801F780065
:1032900068FD070001F0A2000005BE00020020004A
:1032A00093FC230056FE07000801BE001AFB07002E
:1032B000809FBE000A00BE0022A22A00D39F2300E6
:1032C0004FFE07004F01BE0013FB07000004BE00C5
:1032D00001F0A1000200200003982300EEFC07008B
:1032E00003003D000000200001F823001800370013
:1032F0000800BE000001BE0041FE07000005BE0040
:10330000823B230043DC2B003DFE07000801BE008A
:103310003BFE07000801BE00FFFA07000004BE00E4
:103320000A00BE0052372300F3C1230034FE070019
:10333000F27A2B00B3ED2B00F7FA07000A01BE006A
:103340002FFE07000200200003F82300F2FA070016
:103350004F00A600030037000801BE0003F0A200E2
:10336000020037000001BE000800BE0015FC070087
:103370004F05BE004F04BE00000006000003BE0063
:103380007DFD07006220E100020032000600BE0061
:1033900005000500E507B100F107B20004F02300C5
:1033A0008480700007F0A70001F0A0002400050051
:1033B000889FBE008A9FBE008C9FBE000404BE0092
:1033C0000605BE00809FBE00829FBE002F00070042
:1033D000040678000800BE000A01BE002B000700AA
:1033E000840678004F03BE004F02BE008D4F76006A
:1033F0007FB0970013003300F0FF2F008B8F6B001E
:1034000006003B000D0666000C00A7000A0037000E
:1034100007F0A600100020000A003700880F5200B5
:10342000898F5A008A0F5B008B8F5B000300390085
:103430001000200001003E000000200007F0A7005F
:103440000000EA004F06BE004F05BE004F04BE005C
:1034500000000600E48240001078A300070032005C
:10346000640240001178A3003400BE001401BE00C5
:10347000040032000330A700000006003500BE0043
:103480001501BE000330A0000000060005FF270064
:1034900005826100070032000428E10001003200CB
:1034A000240005000600070001003A004400050062
:1034B0000408050002000700F9FF3A0014000500A7
:1034C0006F826100810270008502710085027200C6
:1034D00000000600800078005002BE005003BE00CD
:1034E0004439DE00F700B200F37F200003016100E1
:1034F000090032000218E10016003A00850172004E
:1035000083017300838173000008200015003A00D6
:103510004000200013003700850172008301730012
:103520008381730005003A0004A8BE0006A8BE000F
:10353000100020000B0037000201E90004024200E5
:1035400085824A0006034B0087834B000748A3008F
:10355000F9FF32000740A00004A8BE0006A8BE0084
:1035600020002000800098009200980000000600D3
:10357000889FBE008A9FBE008C9FBE000004BE00D4
:10358000FDFC07000800BE006420E10048003E008A
:103590005500320072212700132B24003EFC070047
:1035A00047003C000800BE00C2EC2800E32C2C00C1
:1035B00037FC0700470035000800BE0001F0A100FD
:1035C000020020000338230031FC070043003500CF
:1035D0000800BE00B2A32A0083FB230088FD070079
:1035E0000200200003F0230001F0A70003F0A00078
:1035F00049FA07002AFC07000005BE008DFC070001
:1036000001F0A2000006BE000200280013F3230010
:103610007BFD07000801BE003FFA0700809FBE0047
:103620000C00BE0032082800E3952B0074FD070053
:103630004F01BE0038FA07000006BE000001BE00C0
:103640006FFD0700809FBE004241250083B8230024
:103650006BFD07000200200003E823002EFA07009C
:103660000C01BE0066FD07000006BE004F00BE0054
:10367000F2F92B00C3D4230061FD070002002000F3
:1036800003F0230024FA07000C01BE0021FA070012
:103690000001BE000C00BE004AFB07000200200033
:1036A00003F023001CFA070061014500B500070084
:1036B0004F06BE004F05BE004F04BE0000000600CE
:1036C00001F82700000020002202200002F78800F5
:1036D000F7FF37006000B800FBFF370001F8230058
:1036E00000002000F2FF370009F8A300F0FF3200CD
:1036F0006000B800EEFF3700889FBE008A9FBE00C2
:10370000841F7800B1FC07004F00780011003300DF
:10371000F0FF2F00838F6C0006003B00040565005E
:103720000A00A7000800370009F0A60010002000DA
:1037300008003700820F5400838F5C0003003900BB
:103740001000200001003E000000200009F0A7004A
:103750000000EA004F05BE004F04BE000000E0007C
:1037600000000600889FBE00830478000300E0008C
:103770002C00350003003C00008270000402710040
:103780002600320036432000C50020008383CF008E
:103790000A0039000541B1008283CF0007003900DB
:1037A0000541B1008183CF00040039000541B1001B
:1037B0008083CF00010039000541B10085C353006B
:1037C0006022B800120032000A003B0084827200BE
:1037D000610260008301D1000281D3008180D300A7
:1037E0000080D3000603E8008743E800F7FF3A00B3
:1037F00007003700000040008180480002014900B6
:10380000838149000603E9008743E900F9FF3A0094
:1038100033FB070009F0A70003F0A0004F04BE002F
:103820000000060060001000E08018006001190030
:10383000E0811900D3FF3B00033E2C00F7FF370067
:103840000400200000003700889FBE008A9FBE0051
:103850008C1F78004F26DD005CFC070063FC330002
:103860006120E100430032006250E10041003E006F
:103870003E0039006420E1003C0032000582550022
:103880000F003B000402E80038003A00800F5300AC
:10389000818F5B00350034000800BE0003F0A100FA
:1038A00001F0A60003F0A0000CF0A7009AF90700B1
:1038B00057FC37000603430087834B000C46460045
:1038C0000005530081855B00020033000A03BE003F
:1038D0000C00A0000402E900F6FF3B00850578001B
:1038E0000602430087824B0004003A006000B800E3
:1038F00009F0A70001F0A00045FC370000025200CB
:1039000081825A000704E0000400330006034300EC
:1039100087834B008B05E900FAFF37000905780023
:103920000604BE000203BE006011B800ECFB0700F5
:10393000E00F5200E08F5A000700350002003C0003
:103940000C08A300040032000601BE0003F0A00032
:103950000CF0A70070F907000A85680001F0A100CB
:103960000AF0A70001F0A00029FC37000800BE0003
:1039700027FC3700100220000CF0A60000F788009A
:1039800027FC37000003BE00FBFB07006220E100BC
:10399000020032000600BE00000006008502410061
:1039A000E30F20000328E10005003C00A3FE2F00E8
:1039B0000328E10007003D0005002000010037005A
:1039C000F50F20002002200000F788006000B800FA
:1039D00008003700130020008381520005003D00DD
:1039E0008100D1000080D3008301E800FCFF3A0091
:1039F00005002000C72ADD00F107B20085807000B5
:103A000007F0A70001F0A00000000600889FBE009C
:103A10008A9FBE008C9FBE0058FE07008504780078
:103A20000005BE006420E10049003E006220E10084
:103A300003003200090035000BF8A30044003200F7
:103A40000BF8A300080032001002200000F78800E5
:103A5000F0FF2F00F1FF27003D00370001F82F0095
:103A6000000020003A0037003D00070029F9070058
:103A70000006BE000A00BE00324F200053F32300B0
:103A800005FB0700060034000C00BE0034000700F0
:103A900020F907000006BE000A00BE000200370041
:103AA0008904E9000C00BE002D00070054FC07004B
:103AB0002B00070018F907000001BE000C00BE0033
:103AC00040FA07000005BE000001BE004CFC0700E4
:103AD0000006BE00A2F32300430D2C000EF90700E0
:103AE000809FBE000C00BE00D2E32700D3F02B0065
:103AF00043FC07004F01BE0032FA07000006BE007B
:103B00000A01BE003EFC07000A01BE0002F90700E0
:103B10000006BE006148B90046FB07000005BE0074
:103B200032082800E3952B0035FC07000C01BE008D
:103B3000F9F807000006BE000A00BE0002002800D7
:103B400013F323002EFC07000C01BE00F2F807005F
:103B50004F06BE004F05BE004F04BE000000060029
:103B600003F02300020005000001780000C2B3004A
:103B7000010037000201E8009240780080CF500039
:103B8000FCFF3200E9CF5000FAFF3200D0C2B30090
:103B900080CF500003003A000201E80014C0B300D7
:103BA000050037000042EB00B0C2B30080CF5000E8
:103BB00001003A000201E8008000EB0005FD2F0043
:103BC000040037006A08B900008041008500400009
:103BD0000201E8009201FB0005804100E90F50005E
:103BE000F8FF36000404E000010032008100EA0022
:103BF000010078000000060001002000A01E8900DE
:103C0000B11E890011C0B300203D22000148780098
:103C100000000600223D22001204E00006003A00E7
:103C20001000200001002000A01E8900B11E8900A4
:103C300010C0B30000497800D2E62400631C2400C1
:103C4000A01E8100B11E8100A70307000001BE0075
:103C50009003230001002000020040008380480000
:103C6000A01E8900B11E89004088DE00CF80DE00E2
:103C700000F0A1000000060080017800000178003B
:103C8000010037000201E8001204E000FDFF3A00E5
:103C900031407800005978000004E000FCFF3A0051
:103CA00003007800000006000C00FA00889FBE00A8
:103CB00000047800CFB09700F0FF2700D0BF9F002E
:103CC0008004EB0099BF9F0088BF9F00A8BF9F00A2
:103CD000200C2000B0BF9F007881570070805700F3
:103CE000080007000FB89700094878000FB8970040
:103CF00008045000080078004F04BE000080FA005D
:103D000000000600FE874700889FBE008A9FBE0015
:103D10008C9FBE008E1F7800F0B79F0001077800CF
:103D200082BF9F000000EB00A0B79F009F023700FA
:103D30008006EB0050C2B30080CF50000900320073
:103D40000100FB00FFB09700A3020700E10F400055
:103D500096023200AFB097008100E800A1B79F0043
:103D6000920237009E407800D0C2B30080CF50004E
:103D70000C00320007003C006D40500080CF500026
:103D80000A0032006B40400080CF50000E003A0025
:103D90000800370000C3B30080CF50000A003A008B
:103DA000060037000D30A000050037000D00A00010
:103DB000030037000D10A000010037000D20A00007
:103DC0000E07E800E7FF37000D18A30001003200DE
:103DD0000D00A1000D38A300010032000D20A1004C
:103DE0000100FB0002FD2F0002004000E90F50001F
:103DF0000E003E000002EB00C4B79F008201780075
:103E0000CFB297006A28B9001E01FB0000014100F3
:103E100003014100C2B79F005E00FB0003004000A9
:103E2000E90F50000B003E00F5FF37000006EB00E5
:103E3000CCB79F00A0C2B30080CF500005003A006D
:103E40000FB89700C000780080BF9F00C1B79F00E7
:103E50000E07E8000001EB00B2B79F00E0C2B3001C
:103E60009E4F100018003A000DE0A0008E00E80000
:103E700064405000914F10000200320001077800AA
:103E80000C0037000FBA9700C402780084BF9F006F
:103E9000B5B79F000E87E8000B0037003FB69700CC
:103EA0006A60B9000000410003004000B0B79F0005
:103EB0000E07E8001E01FB0003FD2F000300410078
:103EC000E90F5000F5FF3600BE407800E1D79F00B3
:103ED000C0C6B30080CF5000220032000F003C006B
:103EE0006940500080CF50007700320004003C0051
:103EF0000104E000310232006B4050000F00370037
:103F000040C6B30080CF50009300320065404000AF
:103F100080CF50008B003A008F00370030C7B300CD
:103F200080CF50001A00320007003C00644050006F
:103F300080CF5000110032000040E80080CF5000D8
:103F400080003A000F00370050C7B30080CF500008
:103F5000800032006340400080CF500079003A007A
:103F600009003700000028000D48A30001003A00B6
:103F70000001200080867600D3FF37000D60A0008E
:103F8000750037000D50A0000D70A00072003700C2
:103F90008FB897004100780081BF9F00000478002F
:103FA0000000E00001003A00283822008004EB0005
:103FB000010037008104E80089007800088044008F
:103FC0001004E000FBFF3A003FB197000200E00060
:103FD00003003200890F5100010031008204780093
:103FE0000002EB00E4AF9F00CFB29700898F520030
:103FF0000200360009805200E0AF9F004368DE00F7
:10400000E10660001B003A000D0678000900370049
:10401000FFB0970000022000EF010700E10F400011
:10402000030032002FB097000000E800A0B79F0007
:104030000C06E800EFA89700810F5600F4FF3A0045
:104040000081EB00E2AF9F000A0037008800780093
:104050003100FB0001047800FFB09700DE0107008B
:10406000E10F4000030032002FB297000402E80085
:10407000A4B79F000900E90080047800E10F400028
:10408000F2FF3A000006EB000D00E0000A003A00E3
:10409000C6013700FFB0970000022000CE010700E4
:1040A000E10F400003003200AFB297008502E80044
:1040B000A5B79F000C06E8006FA89700800F560078
:1040C000F4FF3A00B90137008FB89700410078003B
:1040D00081BF9F00CF80DE0001017800820178005F
:1040E0000205BE000004BE000203BE000002BE00C6
:1040F0004822DE00482EDD0004027600E4D79F004F
:104100000D48A3000A0032000404E0000800320059
:10411000E14F42000600320071FD2F000180470090
:104120000448780018409800290020000200370059
:10413000F0D79F001900200072FD2F000284470075
:10414000A1FF370064FD2F00048447001900200000
:104150009DFF37000D0CB3000D007800000CB2007D
:1041600028003A000D00E00005003D008FBA9700DE
:104170004505BE004504BE0085BF9F001400370002
:104180000D48A3000B0032000FBE97004C00BE008C
:104190008CBF9F004F89DE00CF91DE000002BE0081
:1041A00002037800820378000605BE000404BE0006
:1041B000070037008FB897004100780081BF9F004B
:1041C00000047800CFC4DE00090578008A05780075
:1041D000E00F5400E08F5C00E00F5D00E08F5D00B9
:1041E0001F003D003D00B3006000B8006011B80042
:1041F00008045000898458000A0559008B8559002D
:10420000170037000D00E00005003D000FB99700D2
:104210004205BE004204BE0082BF9F00100037006E
:104220000D48A300070032000FBA97004400BE00FB
:1042300084BF9F006011B8000205BE000004BE00EC
:10424000070037008FBA97004500780085BF9F00B0
:1042500000047800090020000A0020000B00200064
:104260003FB697000C00E00007003A00E00F540052
:10427000E08F5C00E00F5D00E08F5D0002003A001F
:1042800010002000B0B79F008D007800010CB20034
:10429000E1B79F0000042000808F50003000320002
:1042A00003003C000100E00008003200400037003D
:1042B000000820006FB19700800F510014003200F9
:1042C000000C2000800F510039003A0014C0B300E8
:1042D000252E22000B0037000400FB004300DD0008
:1042E000050040005001BE004000BE000040E1005B
:1042F00001C8E10002D0E10003D8E1002B00390041
:104300000442E800F44F5200F3FF3A002700370060
:1043100000012000010020006011B80014C0B300AB
:104320000040E10001C8E10002D0E10003D8E10053
:104330001E003900450020000000D0008180D2001E
:104340000281D2008381D2008502E900FAFF3A009F
:104350000442E800F04F5200F1FF3A00130037002A
:1043600080002000010020006011B80014C0B300DC
:104370000040E10001C8E10002D0E10003D8E10003
:104380000A0039003C0020000000D0008180D200EB
:104390000281D2008381D2000C06E900FAFF3A00C4
:1043A0000442E800F54F5200F1FF3A00E4D79F00C5
:1043B000EFD097000100FB003FB19700820F500043
:1043C00002003D00E2D79F00040037003FB2970093
:1043D000800F520001003D00B0B79F00CFB29700A0
:1043E0000500E00004003200638066000200320035
:1043F0008502E900C5B79F000DE8A3000B0032005D
:104400004FB697003FB09700800F560003003C0066
:104410008000EB00C1B79F00040037004FB1970048
:104420003FB2970004015100C2B79F00EFD297003E
:104430000500FB000006EB00DCAF9F00CFB097004B
:10444000808F50000200340000805000D0AF9F00E9
:104450000D28A30037003200E18066000D18A3008C
:104460000C003200D00220000100E00001003A0000
:104470000080E900FFB09700D7000700E10F40007F
:104480000E0032002FB197000201E800A2B79F0092
:104490000A0037000100E00008003200FFB097007A
:1044A00000022000CC000700E10F400003003200B2
:1044B0002FB297000402E800A4B79F00DFAA97007C
:1044C0000500E0000F0032000006EB00FFB097008F
:1044D00000032000C0000700E10F4000030032008D
:1044E0002FB097000000E800A0B79F000C06E8007E
:1044F000DFA89700810F5600F4FF3A000001EB009F
:10450000D2AF9F003FB29700C320DD00A02D220054
:104510008080400091B79F004220DD006400500081
:1045200080B79F006320B900F0AF9F006306500082
:1045300084003700DFAA97000500E0001100320078
:10454000688066000F003A0000067800FFB0970010
:1045500000022000A0000700E10F4000030032002D
:104560002FB097000000E800A0B79F000C06E800FD
:10457000DFA89700810F5600F4FF3A000001EB001E
:10458000D2AF9F00E18066000D18A3000C0032003E
:10459000D00220000100E00001003A000080E900A4
:1045A000FFB097008C000700E10F4000D5FF3200FC
:1045B0002FB297000402E800A4B79F00D1FF370094
:1045C0000100E000CFFF3200FFB0970000022000A2
:1045D00081000700E10F4000CAFF3200AFB2970030
:1045E0008502E800A5B79F00C6FF37000004200041
:1045F000EFB09700808F50003100320003003C0084
:104600000100E000080032003E00370000082000F2
:104610006FB19700800F510011003200000C200094
:10462000800F510037003A001FB097003002BE00E3
:104630002003BE000800BE000A01BE00D70107002B
:10464000A4002000050020006033B800DA01070054
:1046500004C3B30004424000E4D79F0029003700A0
:1046600095382200D5B79F000D58A30002003A00EC
:10467000A0392200D0B79F001400200005002000C0
:104680006033B8008FB097008100E9000500330067
:104690000402D0008582D2000683D2008783D20034
:1046A000F9FF37000800BE000A01BE00BB01070089
:1046B0006F0060005FB19700624078001000370023
:1046C00014002000050020006033B8000C007800C2
:1046D0000000E900050033000402D0008582D2000A
:1046E0000683D2008783D200F9FF37000800BE009E
:1046F0000A01BE00A9010700674060000043B00046
:10470000E0D79F00EFD097000100FB00FFB09700BB
:1047100031000700E10F4000030032002FB1970085
:104720000201E800A2B79F001FB297006802520082
:1047300094B79F008FB29700E482520085B79F0024
:1047400063065600D0FF2F003FB197000090B900DC
:104750007FAA97000000420063005000800F5600BF
:10476000A2FF3A000D38A30010003200DFAA970024
:104770000500E0000D0034000006EB00FFB09700DC
:104780000002200014000700E10F40000300320087
:104790002FB097000000E800A0B79F000C06E800CB
:1047A000DFA89700810F5600F4FF3A00BE40780062
:1047B000E1D79F000104E0005DFD3A002FB09700B3
:1047C0004F0778004F06BE004F05BE004F04BE00E5
:1047D000EF01B10000000600889FBE0000017800D4
:1047E00001047800B10090000118A30040003200DD
:1047F0000198A30003003A00180090000000E000B8
:104800003B003A000190A000310498008204780037
:10481000F90FB200180090000000E00002003A001A
:1048200028009000000C7800EA8F540006003A003F
:10483000380090000078A30003003A008800780058
:10484000D0002000E4FF0700180290006121B900A9
:1048500058009000E8009000800F5100818F5900AF
:104860000B0032000400E8001004980018007800E3
:1048700009587800000C780011C0B300C03D220038
:1048800001487800EA8F5400060032001900370012
:10489000880078000940780019000700800478003B
:1048A00014003700380090000088A3001100320087
:1048B00018019000A80090004800900053000700E5
:1048C00098009000810F50000400320038009000E2
:1048D0000003B300300498008084EB000000EB007C
:1048E0001004980028009000000C780001003700A8
:1048F0008084EB00090078004F04BE000000060031
:104900000200FA00889FBE00A0FF9F00010478000B
:10491000B1009000810478000904B2000200320066
:104920000000FB00360037000118A30005003A0024
:104930000103B30031049800190498000080EB00D3
:104940002F003700580090000000E00006003A00F9
:104950004800900012002000E68057002B0007005E
:104960001904980024003700280090000000E0009F
:1049700008003A00803D220020049800000C7800D6
:104980002000200050049800100498000130A0007E
:104990003104980018019000A80090004800900091
:1049A0001A00070028009000000C78000080EB003F
:1049B0001004980018007800AFF8970001587800AC
:1049C000000C78002FF89700EA4F50000A003A00D8
:1049D000380090000088A300070032001801900002
:1049E000A8009000480090000800070019049800F3
:1049F000A8009000010C7800AFF897000100FB00C0
:104A00004F04BE000080FA00000006000A00FA0011
:104A100080017800E20F500028003E00001F810056
:104A2000E10F500008003200802320000000E00069
:104A30000500320004232000252320004623200007
:104A40008001780004003700042220002522200085
:104A50004622200083222000144090000004E00041
:104A6000040035008009EB00144090000074A000A1
:104A700010429800154090000028A30003003A005F
:104A8000154090000024A000904298008001EB00A7
:104A900007003700154090000008A300FDFF32001A
:104AA00063C078000000FB00000B78008301E80081
:104AB000828F5100F7FF3A000800370030002000D5
:104AC000B0BF9F00C3BF9F00D1BF9F00E2BF9F0048
:104AD0006A80570000C0DA006FB9970002007800C2
:104AE0000080FA0000000600020AB900001BB900AD
:104AF0000200B8008100420081004300000006006F
:104B0000881F7800000478005001BE004000BE00FD
:104B10000400400085804800060149008781490063
:104B2000009CBE000294BE000400E1000588E10084
:104B30000690E1000798E10002003100680044009F
:104B40001008E8004F04780000000600F4874700D2
:104B5000889FBE008A9FBE008C9FBE008E1F78007B
:104B60000205BE000004BE00D4B79F00E5B79F0059
:104B7000F6B79F0087BF9F000000EB00C0B79F0003
:104B8000B0B79F00A0B79F0090B79F0080B79F006D
:104B90000D042000BFB097004FB097000001400007
:104BA0000000E0000F003D004F08DE000000710033
:104BB000C0B79F004D00070001003D00120020001B
:104BC0005000070001003D001200200055000700C2
:104BD00061000700660007000F004000C8FF0700E3
:104BE000220037004F08DE0000067100CCB79F009E
:104BF0003E00070001003D001200200041000700B8
:104C000001003D001200200046000700520007008E
:104C10000FB297009FB297002FB39700BFB39700D2
:104C2000590007000000520081805A0002015B0019
:104C300083815B0080B79F0091B79F00A2B79F0060
:104C4000B3B79F000007EB004F0007000020E10012
:104C500001A8E10002B0E10003B8E1000100310069
:104C60001E0020000E005600C0B79F004FB29700F4
:104C70000400E000070035001000200001002000C3
:104C80006011B80008047000898470000A05710082
:104C90008B8571008D06E900BEFF3A000400E0003C
:104CA00003003D00320007000F00400094FF0700A2
:104CB0004FA897000000E00004003A000FB49700EE
:104CC0009FB497002FB59700BFB597000800BE00AE
:104CD0000A01BE004F0778004F06BE004F05BE0018
:104CE0004F04BE004F01B1000000060001804000EB
:104CF00090B79F000001EB008FB097000100E0002B
:104D0000000006000200700090B79F000180400084
:104D100080B79F000001EB00FFA897000100E000B2
:104D2000000006000200700080B79F000180400074
:104D30006FAA9700CF20DE0001007000F0AF9F0047
:104D4000040242000800BE000A01BE004F18DE0047
:104D50000002720000000600E4AF9F000804440057
:104D600089844C000A054D008B854D00000006002B
:104D70003FB29700CFB297005FB39700EFB39700B1
:104D800000FE2F00000006003FB09700CFB0970054
:104D90005FB19700EFB1970000000600881F780010
:104DA00018002000881F780068FF07008F87E9003F
:104DB0004F04780000000600801FEB0063FF07002F
:104DC0008F87E90000000600889FBE008A9FBE0012
:104DD0008C1F78000205BE000004BE00E00F5000EA
:104DE000E08F5800E00F5900E08F59000C003D00A3
:104DF0006000B8006011B8000804500089845800B1
:104E00000A0559008B8559001C0020001F0007006F
:104E100008003D00180007000006EB000500370001
:104E20000006EB001900070002003D000F0007001C
:104E30001C0020000800BE000A01BE00D7FF0700CA
:104E40000203BE000002BE000C00E00001003200C0
:104E5000060007000400BE000601BE004F067800F1
:104E60004F05BE004F04BE00000006006000B80001
:104E70006011B8000000370004025000858258001D
:104E8000060359008783590000000600E00F520016
:104E9000E08F5A00E00F5B00E08F5B00000006002F
:104EA000889FBE008A9FBE008C1F78000205BE004E
:104EB0000004BE00E00F5000E08F5800E00F5900E2
:104EC000E08F59000A003D006000B8006011B80092
:104ED00008045000898458000A0559008B85590040
:104EE0001C0020001800070007003D0005003700E7
:104EF0000006EB001400070003003D006000B8004E
:104F00006011B800150007000800BE000A01BE00CD
:104F1000A9FF07000203BE000002BE000C00E00073
:104F2000030032006000B8006011B8000B000700F9
:104F30000400BE000601BE004F0678004F05BE000B
:104F40004F04BE0000000600E00F5200E08F5A0040
:104F5000E00F5B00E08F5B000000060004025000E1
:104F60008582580006035900878359000000060017
:104F70001804FA000000EB00203A88000080EB00E3
:104F8000601988000080EB0050198800D0F82500D7
:104F9000200888000000EB00000888008460A90059
:104FA0009460A800109EA90001C3B3000000EB00AC
:104FB000D50207005C360700DF31070068090700EB
:104FC0001812070036300700DC0E070049370700CB
:104FD000793507008739070010C0B300DCFEB70041
:104FE0000000EB003007980008003700BE0090007A
:104FF0006C004700808040000040EB008048780053
:105000003E0090000000E80030079800BE009000CD
:10501000F01F2000808F5000F4FF34000000EB00F0
:1050200030079800DC62A90010002000A0A08800D2
:105030000001EB00F10F20000000EB00E831070059
:105040000000EB003007980008003700BE00900019
:105050006C004700808040000040EB0080487800F2
:105060003E0090000000E80030079800BE0090006D
:10507000F01F2000808F5000F4FF3400BE0090002D
:105080006C00470000804000104078000004E00001
:10509000EEFF32000000EB00300798000000EB004C
:1050A0002007980009003700AE009000C0202000C3
:1050B0000E004000808040000040EB0080487800F7
:1050C0002E0090000000E80020079800AE0090003D
:1050D000F01F2000808F5000F3FF3400AE009000DE
:1050E000C02020000E0040000080400010407800EA
:1050F0000004E000ECFF32000000EB002007980005
:1051000000003700C50B07000004E000DC0032009F
:1051100010002000AF360700E40A0700304798006F
:1051200081F0800000022000008060000000E000AC
:1051300002003A003E409000B30907003E40900054
:105140000001FB00614120008E8040008208780051
:10515000604120000E00400010007800ED0F50006C
:10516000C5003200A0022000614120008E80400076
:1051700091007800808F5000910032006241200041
:105180000E01410012017800EA0F510001003200C7
:10519000AD0037006C00470011002000C72F07004A
:1051A00020479800AE40900020C3B30080CF50004D
:1051B00067003A006C004700104078000001FB00D7
:1051C000414120008E80400082087800C004200009
:1051D000414120008E80400091007800808F500077
:1051E00043003200C0042000424120000E01410073
:1051F00012017800800F510007003C00900420004D
:10520000414120008E80400091007800808F500046
:10521000330032004B003700D00420004241200010
:105220000E01410012017800800F5100070032008A
:1052300020052000414120008E8040009100780030
:10524000808F50003B0032003E00370050F6800057
:10525000224120000E014100000978004005200095
:10526000214120008E80400091007800808F500006
:105270001100320090062000224120000E01410062
:1052800012017800800F51000900320090042000C4
:10529000214120008E80400091007800808F5000D6
:1052A000010032000B003700B3340700280037003C
:1052B000B134070026003700807F2A00040A070067
:1052C000D0C0B30050090700A0C0B3004E090700CA
:1052D0001F00370000C0EB000C0907001C0037005E
:1052E0006C00470081080700080907001800370014
:1052F000333107000000EB0050079800060037002C
:10530000803E200001002000C40107005E009000E4
:105310000000E80050079800DE009000F018200020
:10532000808F5000F6FF34000000040000000000F1
:105330000700370001C3B30020002000F20107007E
:10534000030037006C00470091220700EF080700B8
:10535000D0C0B3002C090700A0C0B3002A09070081
:105360000000EB003007980008003700BE009000F6
:105370006C004700808040000040EB0080487800CF
:105380003E0090000000E80030079800BE0090004A
:10539000F01F2000808F5000F4FF3400BE0090000A
:1053A0006C00470000804000104078000004E000DE
:1053B000EEFF32000000EB00300798002E003700AF
:1053C0001E4090000004E0001C003200E0802A0033
:1053D000FA0907000040EB00104798000000EB00BE
:1053E0003007980008003700BE0090006C004700AE
:1053F000808040000040EB00804878003E00900034
:105400000000E80030079800BE009000F01F200068
:10541000808F5000F4FF3400BE0090006C00470005
:1054200000804000104078000004E000EEFF3200F1
:105430000000EB00300798000F00370010C0B300E9
:10544000104798000C003700BE009000F01F2000AD
:10545000808F500008003C00BE0090006C004700A8
:10546000008040003E419000024878003E009000DD
:105470000000E8003007980010C0B300DCFEB70061
:10548000F30A07000004E000F700320003350700CC
:105490001C0A0700304798003E409000DA080700D9
:1054A00060F680000000E0008F0032003E40900077
:1054B0000000FB00ED0F50000100320052003700E9
:1054C00061F68000004120000E00400001087800D5
:1054D000024120000E01410012017800E20F51004C
:1054E0001A003200004120000E0040001000780039
:1054F000E20F500006003C00014120008E80400079
:1055000091007800E18F50000C0032001F0037003E
:10551000024120000E01410012017800E30F51000A
:1055200010003200004120000E0040001000780002
:10553000E40F50001100320014003700C02020009A
:105540000E004000E001070010003700E0802A0054
:105550009A090700C02020000E004000D60A07006C
:105560000A003700C02020000E0040004B38070022
:1055700000C2B3006508070004003700C020200007
:105580000E004000022207009F0807000000EB0009
:105590002007980009003700AE009000C0202000CE
:1055A0000E004000808040000040EB008048780002
:1055B0002E0090000000E80020079800AE00900048
:1055C000F01F2000808F5000F3FF3400AE009000E9
:1055D000C02020000E0040000080400010407800F5
:1055E0000004E000ECFF32000000EB002007980010
:1055F00060F68000E30F50009B0032000000EB00DB
:1056000060F688009800370062F68000E1402000D4
:105610008E80400082087800E04020000E004000AC
:1056200010007800E40F500025003200E140200017
:105630008E80400091007800E58F50001E003200FF
:10564000E24020000E01410012017800E30F5100FA
:105650000100320084003700BE40900050C3B30008
:1056600080CF500003003A0010812A005309070040
:105670007D003700BE40900060C2B30080CF500074
:1056800003003A0000822A004C0907007600370028
:10569000AE009000C02020000E00400000804000BE
:1056A000BE409000014878002E0090000000E80005
:1056B000200798006C003700113107006A0037009E
:1056C000AE009000C02020000E004000008040008E
:1056D0003E419000024878002E0090000000E80053
:1056E00020079800600037003E4090000001FB005A
:1056F000C14020008E80400082087800D004200045
:10570000C14020008E80400091007800808F5000C2
:105710004C003200D0042000C24020000E014100A5
:1057200012017800800F510013003C00A0042000FB
:10573000C14020008E80400091007800808F500092
:105740002D003200B0042000C24020000E014100B4
:1057500012017800800F51002900320090042000CF
:10576000C14020008E80400091007800808F500062
:10577000250032003600370050052000C2402000CE
:105780000E01410012017800800F51002500320007
:1057900050052000C14020008E804000910078001C
:1057A000808F500007003C0040052000C2402000D0
:1057B0000E01410012017800800F510017003200E5
:1057C0002300370070052000C14020008E8040007B
:1057D00091007800808F50000E00320050072000AA
:1057E000C24020000E01410012017800800F5100DC
:1057F0000F003200160037007B3107001A00370017
:1058000089310700180037001000200060F688007A
:10581000150037004D3507001300370081370700AA
:10582000110037002000200060F688000E003700CD
:10583000C12020008E804000C00520008D0C070094
:10584000090037004000200060F68800060037009D
:10585000C02020000E0040008040EB00014878008E
:105860000000EB002007980060F68000E50F500074
:1058700001003A00A2300700020A07000004E0001D
:105880000600320035090700304798003E4090007E
:10589000DD0707000040EB0030479800901E07002E
:1058A00080F08000610060000000E0000500320030
:1058B00090F0800001202000010060000000E00066
:1058C0000A003A0070F0800001002400010060002E
:1058D0000000E00005003A0070F0800001082000A0
:1058E000010060000000E00006003200C0F280000D
:1058F0000000E0000300320040002000B534070043
:105900000B00370080F08000610060000000E000C4
:105910000700320090F080000120200001006000AC
:105920000000E00002003A000000EB0097100700C2
:1059300080F0800001022000010060000000E00013
:1059400005003200E0F280000000E00002003200BA
:10595000500020009F340700A0F280000000E0000B
:10596000230032002E0090000000E00020003200F2
:105970000000EB002007980009003700AE009000FF
:10598000C02020000E004000808040000040EB005E
:10599000804878002E0090000000E8002007980062
:1059A000AE009000F01F2000808F5000F3FF340005
:1059B000AE009000C02020000E004000008040009B
:1059C000104078000004E000ECFF32000000EB0023
:1059D0002007980060F68000E30F500002003200BC
:1059E0000000EB0060F688000000EB00A0F28800E9
:1059F00080F0800001082000010060000000E0004D
:105A0000C0FD3200F0F280000000E000BDFD320079
:105A1000600020006F340700BAFD37000600FA006E
:105A2000100798002107980010002000000F780050
:105A3000090037001E009000AE0090001200200008
:105A4000F3FF2F00000041008180490010079800FB
:105A5000210798001E0FE8001E019000AE01900083
:105A6000F0FF2F0001002000800F5100818F5900AE
:105A7000F0FF3E00110037000040EB0012F4B700C9
:105A80001E009000100888000000EB00000888004D
:105A900005E1A800010037000140FE0012D4BF005C
:105AA0000004E000FCFF3200F0FF2F0001002000A6
:105AB00010079800210798001E0FE9001E00E00063
:105AC000EDFF3A000040EB0012F4B7000080FA004E
:105AD00000000600801F78003400F800100020004D
:105AE000A00188000000FA008460A90005E1A90077
:105AF00010C0B30012F4B7000080FA003400F900BF
:105B00004F007800004006000600FA00000F780001
:105B1000214798001E007800200798002E00900072
:105B2000E10F50001A0032002E009000E20F5000EA
:105B3000200032002E0090000000E0000100320042
:105B4000230037000000EB0070F6880008003700E3
:105B500071F68000E04D2100808040000040EB00A5
:105B60008048780070F680000000E80070F6880039
:105B700071F68000F07F2000808F5000F4FF340029
:105B80000000EB0070F68800DC22A900100037004E
:105B900071F680002E419000E04D21000080400011
:105BA0000248780070F680000000E80070F6880077
:105BB00007003700DED4BF000004E000040032001C
:105BC000E04D2100C2070700E04D2100FB07070060
:105BD0000080FA00000006000400FA00D0F3800004
:105BE000E1F38000008FBE0010F4800021F48000FB
:105BF000D0F38800E1F3880012F4800023F48000E1
:105C00000000220001002000800F5100818F590008
:105C100006003600D0F38000E1F38000630040000E
:105C2000E08048001E01BE00AB0C07000000EB0046
:105C300040F488000080FA00000006000000FA002E
:105C400040F480000000E00015003200A0F6800063
:105C5000640040006101B90010F4800021F480006C
:105C6000020040008380480010F4880021F488007E
:105C70000000EB00A0F6880012F4800023F48000FE
:105C8000F0F3800001F48000930C070010F4800012
:105C900021F48000F0F3880001F488000800370048
:105CA000D0F38000E1F3800076004000E0804800FF
:105CB000F0F3880001F488001000200040F4880010
:105CC0000080FA00000006000E00FA00889FBE0067
:105CD000200798000000EB00C0F388002E00900021
:105CE000104078000000FB006101B9000080EB006B
:105CF0008080EB0002014000838148005207980039
:105D00006307980000022000010020005E0190005F
:105D1000EE019000800F5100818F5900C1033E00B9
:105D20005E009000EE00900000600100200037004F
:105D3000230037004B003700540037005D00370068
:105D4000BA033700B9033700B8033700B703370089
:105D500062003700630037006C00370075003700C1
:105D60007E003700B1033700860037008F00370010
:105D70009E003700AD003700BC003700000137003F
:105D80004A01370094013700E60137003802370036
:105D90007D023700B9023700F502370031033700C2
:105DA0003A0337003C0337003E03370086033700D1
:105DB0008000EB00C0852A00C02C07009B03370041
:105DC0001000200030F4880012F4800023F48000DA
:105DD0000000220001002000800F5100818F590037
:105DE0001E003A0010F4800021F48000DE0B070052
:105DF000E00F5000E08F58001800320066004700A6
:105E0000260D07003E009000100798001E0090002D
:105E10000020A1000030A1000040A1000050A1001E
:105E2000100798001E0090002B0D07003B0D070087
:105E30000000220001002000960C07001E009000C8
:105E40000020A0000030A0000040A0000050A100F1
:105E5000100798001E0090001F0D07005EFF07004E
:105E600072033700110020002E009000D922070095
:105E700000017800D0F38000E1F380006C00400066
:105E8000E0804800470C070068033700110020003D
:105E90002E009000CF22070000417800D0F3800050
:105EA000E1F380006E004000E0804800600C0700D5
:105EB0005E0337002E0090000000E80010407800DC
:105EC00000417800D0F38000E1F380006F004000D3
:105ED000E0804800560C07005403370057FF0700C6
:105EE00052033700110020002E009000B922070055
:105EF00000017800F0F3800001F480006C004000A5
:105F0000E0804800270C07004803370011002000FC
:105F10002E009000AF22070000417800F0F38000CF
:105F200001F480006E004000E0804800400C070053
:105F30003E0337002E0090000000E800104078007B
:105F400000417800F0F3800001F480006F00400011
:105F5000E0804800360C07003403370011002000B1
:105F60002E0090009B22070000417800F0F3800093
:105F700001F4800070004000E08048002C0C070015
:105F80002A0337002E0090000000E800104078003F
:105F900000417800F0F3800001F4800072004000BE
:105FA000E0804800220C0700200337001100200089
:105FB0002E00900087220700CF80DE001DF2070030
:105FC000D232290093EC23000DF30700FBF1070008
:105FD00000017800F0F3800001F4800073004000BD
:105FE000E0804800EF0B070010033700110020008D
:105FF0002E00900077220700CF80DE000DF2070010
:10600000D232290093EC2300FDF20700EBF10700E8
:1060100000017800F0F3800001F48000750040007A
:10602000E0804800DF0B070000033700110020006C
:106030002E00900067220700CF80DE00FDF10700F0
:10604000D232290093EC2300EDF20700DBF10700C8
:1060500000017800F0F3800001F480007700400038
:10606000E0804800CF0B0700F0023700F0F380001B
:1060700001F4800079004000E080480010F48800BE
:1060800021F488000000EB00A0F68800100020003A
:10609000000F7800140037001E00780080007800A0
:1060A0002E009000008040001040780000427800F0
:1060B000A0F680006101B90010F4800021F4800096
:1060C000020040008380480064004000E0804800F7
:1060D00004417800D60B07001E0FE800A0F68000F0
:1060E0000000E800A0F688001E007800800078001C
:1060F0002E00900000804000104078000004E00076
:10610000E5FF3A002E009000104078000041780032
:1061100010F4800021F4800063004000E08048001B
:10612000C30B0700A0F680006101B90010F48000E5
:1061300021F4800002004000838048006401400098
:10614000E081480010F4800021F48000620B070019
:10615000A0F68000640040006101B90010F48000E6
:1061600021F48000020040008380480010F4880081
:1061700021F488000000EB00A0F68800AB02370095
:10618000110020002E00900012220700CF80DE00B8
:10619000A8F10700D232290093EC230098F20700FF
:1061A00086F1070000027800A0F680006101B900C6
:1061B00010F4800021F48000020040008380480039
:1061C00064004000E080480004017800750B07007F
:1061D000A0F680000080E800A0F68800A0F680000D
:1061E00022002000110009000200D80000047800FD
:1061F000F0F3800001F480006C004000E080480073
:10620000080B0700800F540088023A0010F4800049
:1062100021F4800064014000E0814800F0F3800038
:1062200001F4800063004000E08048002A0B070072
:106230002E009000104078000041780010F480009B
:1062400021F4800063004000E0804800780B0700E4
:10625000A0F680006101B90010F4800021F48000F4
:10626000020040008380480064014000E081480053
:1062700010F4800021F48000170B0700A0F68000C6
:10628000640040006101B90010F4800021F4800036
:10629000020040008380480010F4880021F4880048
:1062A0000000EB00A0F6880060023700110020001B
:1062B0002E009000C7210700CF80DE005DF10700AF
:1062C000D232290093EC23004DF207003BF1070086
:1062D00000027800A0F680006101B90010F480008F
:1062E00021F48000020040008380480064004000E8
:1062F000E0804800040178002A0B0700A0F6800027
:106300000080E800A0F68800A0F6800022002000AF
:10631000110009000200D80000047800F0F38000AA
:1063200001F480006C004000E0804800BD0A0700D6
:10633000800F54003D023A0010F4800021F48000E8
:1063400064014000E0814800F0F3800001F4800027
:1063500066004000E0804800DF0A07002E00900041
:10636000104078000041780010F4800021F4800093
:1063700063004000E08048002D0B0700A0F680007D
:106380006101B90010F4800021F480000200400097
:106390008380480064014000E081480010F48000E0
:1063A00021F48000CC0A0700A0F6800064004000C1
:1063B0006101B90010F4800021F480000200400067
:1063C0008380480010F4880021F488000000EB006E
:1063D000A0F6880015023700110020002E00900062
:1063E0007C210700CF80DE0012F10700D2322900A5
:1063F00093EC230002F20700F0F00700000278009F
:10640000A0F680006101B90010F4800021F4800042
:10641000020040008380480064004000E0804800A3
:1064200004017800DF0A0700A0F680000080E80081
:10643000A0F68800A0F680002200200011000900CC
:106440000200D8006104B900F0F3800001F480007C
:1064500079004000E0804800430A07000001BE00C8
:10646000F0F3800001F480000000510081805900A9
:106470007D005000E0805800800F5400818F5C0048
:10648000EA013A0010F4800021F480006401400029
:10649000E0814800F0F3800001F4800069004000D2
:1064A000E08048008C0A07002E0090001040780021
:1064B0000041780010F4800021F480006300400067
:1064C000E0804800DA0A0700A0F680006101B90008
:1064D00010F4800021F48000020040008380480016
:1064E00064014000E081480010F4800021F4800045
:1064F000790A0700A0F68000640040006101B9003D
:1065000010F4800021F480000200400083804800E5
:1065100010F4880021F488000000EB00A0F6880049
:10652000C201370010002000000F7800140037006F
:106530001E007800800078002E009000008040004F
:106540001040780000427800A0F680006101B90098
:1065500010F4800021F48000020040008380480095
:1065600064004000E080480004417800B00A070061
:106570001E0FE800A0F680000000E800A0F68800EA
:106580001E007800800078002E00900000804000FF
:10659000104078000004E000E5FF3A00A0F680001B
:1065A0006101B90010F4800021F480000200400075
:1065B0008380480064004000E08048000041EB0018
:1065C0009B0A0700A0F680000000E800A0F6880003
:1065D00010F4800021F4800064014000E081480054
:1065E000D0F38000E1F3800066004000E0804800C6
:1065F000390A07002E009000104078000041780012
:1066000010F4800021F4800063004000E080480026
:10661000870A0700A0F680006101B90010F480002D
:1066200021F48000020040008380480064014000A3
:10663000E081480010F4800021F48000260A070061
:10664000A0F68000640040006101B90010F48000F1
:1066500021F48000020040008380480010F488008C
:1066600021F488000000EB00A0F688006F013700DD
:1066700010002000000F7800140037001E00780082
:10668000800078002E0090000080400010407800CC
:1066900000427800A0F680006101B90010F480008B
:1066A00021F4800002004000838048006400400024
:1066B000E0804800044178005D0A07001E0FE800F2
:1066C000A0F680000000E800A0F688001E00780018
:1066D000800078002E00900000804000104078007C
:1066E0000004E000E5FF3A0010F4800021F480008F
:1066F00064014000E0814800D0F38000E1F38000B5
:1067000069004000E0804800F30907002E00900077
:10671000104078000041780010F4800021F48000DF
:1067200063004000E0804800410A0700A0F68000B6
:106730006101B90010F4800021F4800002004000E3
:106740008380480064014000E081480010F480002C
:1067500021F48000E0090700A0F6800064004000FA
:106760006101B90010F4800021F4800002004000B3
:106770008380480010F4880021F488000000EB00BA
:10678000A0F688002901370010002000000F7800D3
:10679000140037001E007800800078002E00900062
:1067A000008040001040780000427800A0F6800091
:1067B0006101B90010F4800021F480000200400063
:1067C0008380480064004000E08048000441780075
:1067D000170A07001E0FE800A0F680000000E8007E
:1067E000A0F688001E007800800078002E0090003F
:1067F00000804000104078000004E000E5FF3A000F
:106800002E009000104078000041780010F48000C5
:1068100021F4800063004000E0804800040A070083
:10682000A0F680006101B90010F4800021F480001E
:10683000020040008380480064014000E08148007D
:1068400010F4800021F48000A3090700A0F6800066
:10685000640040006101B90010F4800021F4800060
:10686000020040008380480010F4880021F4880072
:106870000000EB00A0F68800EC00370010002000BC
:10688000000F7800140037001E00780080007800A8
:106890002E009000008040001040780000427800F8
:1068A000A0F680006101B90010F4800021F480009E
:1068B000020040008380480064004000E0804800FF
:1068C00004417800DA0907001E0FE800A0F68000F6
:1068D0000000E800A0F688001E0078008000780024
:1068E0002E00900000804000104078000004E0007E
:1068F000E5FF3A002E00900010407800004178003B
:1069000010F4800021F4800063004000E080480023
:10691000C7090700A0F680006101B90010F48000EB
:1069200021F48000020040008380480064014000A0
:10693000E081480010F4800021F48000660907001F
:10694000A0F68000640040006101B90010F48000EE
:1069500021F48000020040008380480010F4880089
:1069600021F488000000EB00A0F68800AF0037009B
:1069700010002000000F7800140037001E0078007F
:10698000800078002E0090000080400010407800C9
:1069900000427800A0F680006101B90010F4800088
:1069A00021F4800002004000838048006400400021
:1069B000E0804800044178009D0907001E0FE800B0
:1069C000A0F680000000E800A0F688001E00780015
:1069D000800078002E009000008040001040780079
:1069E0000004E000E5FF3A002E009000104078001F
:1069F0000041780010F4800021F480006300400022
:106A0000E08048008A090700A0F680006101B90013
:106A100010F4800021F480000200400083804800D0
:106A200064014000E081480010F4800021F48000FF
:106A300029090700A0F68000640040006101B90048
:106A400010F4800021F480000200400083804800A0
:106A500010F4880021F488000000EB00A0F6880004
:106A600072003700110020002E009000D91F07008F
:106A700000017800D0F38000E1F380007400400052
:106A8000E080480047090700680037004001200007
:106A9000C0F388006500370040012000C0F3880083
:106AA0006200370068004700FC0907004E009000B4
:106AB000100798001E0090000020A1000030A100E7
:106AC0000040A1000050A100100798001E00900097
:106AD000010A0700110A070000002200010020003F
:106AE00080F6880091F688000B00370080F6800061
:106AF00091F680006709070082F6800093F6800017
:106B000000002100010020000200400083804800B6
:106B100080F6880091F6880080F6800091F680006B
:106B200074004000E0804800BE0807000000E0005C
:106B3000EEFF3A001E0090000020A0000030A000F0
:106B40000040A0000050A100100798001E00900017
:106B5000E10907000000220001002000D0F38800B6
:106B6000E1F388006000B800F0F3880001F48800C9
:106B7000000022000100200010F4880021F48800A9
:106B80000000EB0040F4880000002200010020001B
:106B900050F4880061F488006000B80070F4880048
:106BA00081F48800000022000100200090F4880099
:106BB000A1F488000000EB00B0F488000000EB00B6
:106BC000C0F488001900370070F080006200600097
:106BD0000000E0000300320060012000C0F38800E4
:106BE0001200370030F480000000E00003003A009B
:106BF00030012000C0F388000C0037000000EB00DB
:106C000030F4880012F4800023F48000D0F3800078
:106C1000E1F38000B00807009004200050F68800DF
:106C20000200370040012000C0F388002E009000D1
:106C300010407800E14F500004003200C0F38000A3
:106C4000F1020700D0C0B300EF0207004F04BE00FE
:106C50000080FA00000006001000FA00404F980083
:106C6000710798000000EB00000F78000600370065
:106C70009E0078000E80E800808040000040EB001D
:106C8000804878001E0FE800900020009E0F100042
:106C9000F7FF34000E80E800CE48900001487800ED
:106CA0000E80E800FE009000F3F307000E80E8007D
:106CB000371C07000080FA00000006000400FA00FC
:106CC00020479800314798002E409000004F7800F0
:106CD0003E409000104798000E0078002C1C0700E2
:106CE0000080FA00000006001A00FA00889FBE002B
:106CF00070F4800081F4800063004000E080480070
:106D000019080700200F9800310F98002E089000F6
:106D1000BE08900064005000E08058001208070090
:106D2000000F9800110F980070F4800081F480002B
:106D300066004000E08048000B08070060079800EC
:106D40007107980070F4800081F4800069004000B1
:106D5000E0804800040807004007980051079800A9
:106D600050F4800061F4800069004000E080480039
:106D7000FD07070020079800310798002E009000BB
:106D8000BE009000008FBE0001C2B300E0C4B3009B
:106D9000CAFF070070F4800081F48000700040009A
:106DA000E08048003C0807000080FB00B4060700B4
:106DB0008000780010C4B300A7FF070001C3B30030
:106DC00030C4B300BDFF0700F1852A00A0C4B300A2
:106DD000A1FF070001C3B30000C5B300B7FF070060
:106DE00070F4800081F4800073004000E08048006F
:106DF0000C080700A20607008000780020C4B3003A
:106E000095FF070070F4800081F480007500400059
:106E1000E08048000308070099060700800078001A
:106E200080C5B3008CFF070070F4800081F48000FF
:106E300077004000E0804800FA070700900607004E
:106E40008000780090C5B30083FF070070F48000D5
:106E500081F480006C004000E0804800F1070700EA
:106E600050EE880050EE80000000E00003003A0081
:106E700030012000C0F388007B0037000000EB00E9
:106E8000400F980006003700803E200001002000DF
:106E9000E2FA07004E0890000000E800400F98005A
:106EA000CE089000F0702200808F5000F6FF340072
:106EB000350037002E089000BE089000D907070063
:106EC0006F0607008000780030C7B30062FF07003C
:106ED0006E009000FE009000D207070068060700D1
:106EE0008000780060C6B3005BFF07001E00BE0094
:106EF000E9070700004178004E009000DE00900096
:106F00008D0007005E0607008000780040C6B300D1
:106F100051FF07002E089000BE089000620040005C
:106F2000E0804800200F9800310F98006E0090001C
:106F3000FE00900062004000E0804800600798007A
:106F40007107980010002000010020001E0F400073
:106F50005E9748000000EB00400F980006003700E5
:106F6000803E200001002000ACFA07004E0890008F
:106F70000000E800400F9800CE0890003006200086
:106F8000808F5000F6FF34002E099000BE0990005B
:106F90000E0890009E089000800F5100818F5900CC
:106FA000C4FF390001C2B30020C7B30043FF07008C
:106FB00070F4800081F480006B0707000004BE00BD
:106FC00050F4800061F4800067070700800F5400D0
:106FD000818F5C000600310070F4800081F4800035
:106FE0006107070070F4880081F488001E003700F4
:106FF000B0F480000000E800B0F48800B0F4800035
:107000000004780050F4800061F4800074004000B7
:10701000E080480083070700800F5400080031001B
:1070200050F4800061F4800076004000E080480069
:107030004D07070070F4880081F488000A003700CB
:107040000000EB00B0F488000000EB0040F4880082
:1070500050F4800061F480007207070001002000F6
:1070600050F4880061F488004F04BE000080FA00EC
:10707000000006000E00FA00004F980070F4800037
:1070800081F4800079004000E080480020079800EB
:107090003107980050F4800061F480003207070047
:1070A000008FBE00160037002E009000BE0090003A
:1070B00063004000E0804800770707008080FB0005
:1070C0000E4890000000FB00808F500007003A003F
:1070D0002E009000BE00900064004000E080480058
:1070E00050079800610798000F0037002E009000AD
:1070F000BE0090001C070700200798003107980089
:107100002E009000BE009000BE0F5000AE8F5800C1
:10711000E5FF390030012000C0F388006000B800AE
:1071200050079800610798005E009000EE00900004
:107130000080FA00000006001200FA0050079800D4
:1071400061079800624F980070F4800081F480001D
:107150007D004000E080480020079800310798003B
:1071600070F4800081F4800079004000E0804800E5
:10717000FD060700008FBE000000EB0040079800EE
:107180000F0037004E0090006101B9002E00900002
:10719000BE00900002004000838048003E070700C8
:1071A0008080FB006E4890000000FB00808F500044
:1071B0000C0032004E0090000000E80040079800EC
:1071C0004E0090006101B9002E009000BE009000BA
:1071D0000200400083804800BE0F5000AE8F580070
:1071E000E8FF39004E0090006101B9002E009000C8
:1071F000BE0090000200400083804800BE0F500097
:10720000AE8F58000A0031004E0090000000400090
:107210006101B9005E009000EE00900002004000A5
:1072200083804800FF060700000F98000200370027
:107230000000EB00000F98000E0890000080FA009C
:10724000000006000C00FA00C0F480000000E0001E
:1072500007003A0050F4800061F48000760040009E
:10726000E080480070F4880081F488000500370051
:1072700070F4800081F48000BB06070070F4880081
:1072800081F48800C0F480000000E800C0F48800A9
:1072900050F4800061F4800066004000E080480007
:1072A000B1060700200798003107980050F48000CD
:1072B00061F4800069004000E0804800AA060700F1
:1072C000008FBE000000EB0040079800060037006A
:1072D000803E200001002000D0F907004E00900001
:1072E0000000E80040079800CE009000F018200051
:1072F000808F5000F6FF34000000EB00400798003C
:10730000100037004E0090006101B9002E0090007F
:10731000BE0090000200400083804800DE060700A7
:10732000204F98002E489000F80007002E4890004B
:107330000004E000060032004E0090000000E8006B
:10734000400798004E009000F30F5000EDFF34000E
:1073500090C0B300ED0007000000EB00400798006C
:1073600006003700803E200001002000ABF9070036
:107370004E0090000000E80040079800CE0090000A
:10738000F0182000808F5000F6FF34000000EB0062
:10739000400798000F0037004E009000CF80DE00BD
:1073A0003E014000AE8148000200BE00BA06070060
:1073B000204F98002E489000D40007002E489000DF
:1073C0000004E000060032004E0090000000E800DB
:1073D000400798004E009000F30F5000EEFF34007D
:1073E00090C0B300C90007000000EB004007980000
:1073F00006003700803E20000100200087F90700CA
:107400004E0090000000E80040079800CE00900079
:10741000703E2000808F5000F6FF340050F4800052
:1074200061F480006F004000E08048009A06070089
:10743000B600070090C0B300B40007000000EB00E6
:107440004007980006003700803E20000100200021
:1074500072F907004E0090000000E8004007980015
:10746000CE009000F0182000808F5000F6FF34000E
:1074700050F4800061F480006E004000E08048001D
:1074800085060700A100070090C0B3009F00070019
:107490000000EB004007980006003700803E200007
:1074A000010020005DF907004E0090000000E80098
:1074B00040079800CE009000F0182000808F500008
:1074C000F6FF340070F4800081F480007300400007
:1074D000E0804800530607000901070090C0B30090
:1074E0008A0007000080FA00000006000600FA008B
:1074F000100798001E0090000000E800104078007F
:107500000000FB002007980030042000AE0090002F
:10751000808F50000900320040052000AE0090002E
:10752000808F5000010032000800370045FF07003F
:1075300010032000000F780006003700EAFD070066
:1075400010032000000F7800020037002003200005
:10755000000F78001E0078000080FA00000006008E
:107560000000FA00F6C2A800F6E2A800F702A800A0
:10757000F722A800E702A800E722A800D662A80028
:10758000F4C2A800F4E2A800F502A800F522A900C0
:10759000E502A800E522A800D462A800F0C2A90074
:1075A000F0E2A900F102A900F122A900E102A8007D
:1075B000E122A800D062A800113A8000F00B200060
:1075C0000081600061042000700520002374200009
:1075D000814978008049780082497800616A2000FA
:1075E0009140780000CCB30000C0600021C2B3001D
:1075F00001407000A6E6B700416A20009140780083
:1076000000CCB30000C0600081C2B3000140700034
:10761000A4E6B700516D20009140780000CCB30083
:1076200000C06000D5E6B700A16D20009140780051
:1076300000CCB30000C06000DAE6B700316D200076
:107640009140780000CCB30000C06000D3E6B700E2
:10765000113A8000000420000081700061042000C5
:10766000700520002374200081497800804978004B
:1076700082497800000120004011880000012000AC
:10768000C011880000012000C012880000C0240042
:107690000011880000118000801188000011800016
:1076A000801288008560A90087C0A9008E40A900CB
:1076B0008580A90087E0A9008E60A9009560A800D8
:1076C00097C0A8009E40A8009580A80097E0A80059
:1076D0009E60A800F0352200101188001011800073
:1076E00090118800101180009012880021E2A800FB
:1076F00031E2A80051E2A8002342A8003342A800CA
:107700005342A8000080FA00000006000200FA00C0
:10771000004F780080F08000700060000000E00002
:10772000030032009E40780010002000F6F80700A9
:1077300004CCBF000004E0001A003A00113A8000B7
:10774000F00B200000816000610420007005200023
:1077500023742000814978008049780082497800AC
:10776000316D20009140780000CCB30000C0600073
:107770003040B300D3E6B700113A80000004200087
:107780000081700061042000700520002374200037
:1077900081497800804978008249780010C0B300A0
:1077A00004ECB70012802000124178000280FB0038
:1077B0008080E80000802000008040001E487800A3
:1077C0000240E80001E8B70023C2BF006240600049
:1077D0000004E0000A003A00028020001241780014
:1077E0000280FB008080E8000080200000804000D4
:1077F0001040780024E2B7000240E80000E8B7003B
:107800000080FA00000006000200FA00004F780035
:1078100009D0BF000004E0001A003A00113A8000CD
:10782000F00B200000816000610420007005200042
:1078300023742000814978008049780082497800CB
:10784000A16D20009140780000CCB30000C0600022
:107850005040B300DAE6B700113A8000000420007F
:107860000081700061042000700520002374200056
:1078700081497800804978008249780010C0B300BF
:1078800009F0B70062C02000124178008280FB003E
:107890007040200080804000008020000080400078
:1078A0001E4878000240E80006ECB70033C2BF0073
:1078B000624060000004E0000B003A0052C020006B
:1078C000124178008280FB007040200080804000E0
:1078D00000802000008040001040780034E2B700B3
:1078E0000240E80005ECB7000080FA000000060046
:1078F0000200FA00004F78000080FA000000060045
:107900000800FA003007980000C3B3004047980011
:1079100000712200100798000000EB00000F7800B3
:10792000220037004E4090000040E8004047980099
:10793000BE0090001E0090000080500030079800AC
:10794000BE0090001E009000808F5000F5FF3D00AB
:107950001E00E0000B003A00CE40900000C3B300D0
:1079600080CF500007003A001E009000E10F500049
:1079700007003A0000C3B30064FF07001E0FE800D1
:10798000030037004E40900060FF07001E0FE80024
:107990001E009000A2002000110009000200D80083
:1079A0001007980000C3B300404798001E009000E5
:1079B0000000E000E2FF3C000080FA00000006004A
:1079C0000800FA003007980000C3B3004047980051
:1079D00000712200100798000000EB00000F7800F3
:1079E000220037004E4090000040E80040479800D9
:1079F000BE0090001E0090000080500030079800EC
:107A0000BE0090001E009000808F5000F5FF3D00EA
:107A10001E00E0000B003A00CE40900000C3B3000F
:107A200080CF500007003A001E009000E10F500088
:107A300007003A0000C3B30073FF07001E0FE80001
:107A4000030037004E4090006FFF07001E0FE80054
:107A50001E009000A2002000110009000200D800C2
:107A60001007980000C3B300404798001E00900024
:107A70000000E000E2FF3C000080FA000000060089
:107A80000200FA00004F78001E407800070307004C
:107A90001EFF07001E4078000C0307001BFF0700B5
:107AA0000080FA00000006000200FA00004F780093
:107AB0001E407800FD02070053FF07001E407800BB
:107AC0000203070050FF07000080FA0000000600D4
:107AD0000600FA00200798000000EB00000F780075
:107AE000010037001E0FE8001E00780080007800BB
:107AF0002E00900000804000104078000004E0005C
:107B0000F8FF3A000000EB0010079800090037006A
:107B10001E009000800078002E0090000080400041
:107B200010407800F9FE07001E0090000000E800F9
:107B3000100798001E0090009E0F5000F4FF3500C3
:107B40000080FA00000006000800FA001007980004
:107B500021079800320798000000EB00000F780022
:107B6000110037003E009000E10F500007003A007E
:107B70001E007800800078001E0090000080400009
:107B800010407800E1FE0700060037001E00780074
:107B9000800078001E0090000080400010407800B7
:107BA00019FF07001E0FE8002E0090009E0F100026
:107BB000ECFF35000080FA00000006000600FA0025
:107BC000200798000000EB00000F7800010037004C
:107BD0001E0FE8001E007800800078002E00900044
:107BE00000804000104078000004E000F8FF3A00F8
:107BF0000000EB0010079800090037001E009000FD
:107C0000800078002E009000008040001040780036
:107C1000FDFE07001E0090000000E800100798001D
:107C20001E0090009E0F5000F4FF35000080FA0007
:107C3000000006000600FA00200798000000EB0094
:107C4000000F7800010037001E0FE8001E007800CA
:107C5000800078002E0090000080400010407800E6
:107C60000004E000F8FF3A000000EB001007980065
:107C7000090037001E009000800078002E00900060
:107C8000008040001040780019FF07001E0090009F
:107C90000000E800100798001E0090009E0F5000A2
:107CA000F4FF35000080FA00000006000000FA0032
:107CB000010037000140FE0021A020009140780023
:107CC00003CABF0080CF5000FAFF320022A020007C
:107CD000124178000280FB0041202000808040009B
:107CE0000080200000804000104078008080FB0071
:107CF0000240E80002EAB700010078000080FA00C4
:107D0000000006000000FA00010037000140FE00FC
:107D100071E020009140780008CEBF0080CF500075
:107D2000FAFF320072E02000124178008280FB00EE
:107D30009060200080804000008020000080400093
:107D4000104078008080FB000240E80007EEB7009A
:107D5000010078000080FA00000006000000FA0030
:107D6000010037000140FE00C12021009140780051
:107D70000DD2BF0080CF5000FAFF3200C220210098
:107D8000124178008280FB00E0A02000808040004B
:107D90000080200000804000104078008080FB00C0
:107DA0000240E8000CF2B700010078000080FA0001
:107DB000000006000000FA00881F7800BBFF0700E3
:107DC00000447800B9FF07008840780047020700A8
:107DD0000080FB004F0478000080FA0000000600DD
:107DE0000000FA00881F7800C6FF070000447800F2
:107DF000C4FF0700884078003C0207000080FB00B9
:107E00004F0478000080FA00000006000800FA0025
:107E1000404798000000EB00000F7800A3FF070028
:107E200020479800AE409000F0C2B30080CF5000D1
:107E300007003400AE40900090C3B30080CF5000E4
:107E40000A0034000200370098FF0700204798001E
:107E5000AE4090004E40900080CF5000FAFF3A00B4
:107E60001E00780030079800090037001E007800D7
:107E70006A00B900800078002E4090000000FB00EE
:107E80008080400000FD2F00008F4000E3FF37009E
:107E90003E0090000080FA00000006000800FA0092
:107EA000404798000000EB00000F780095FF0700A6
:107EB00020479800AE409000F0C2B30080CF500041
:107EC00007003400AE40900090C3B30080CF500054
:107ED0000A003400020037008AFF0700204798009C
:107EE000AE4090004E40900080CF5000FAFF3A0024
:107EF0001E00780030079800090037001E00780047
:107F00006A00B900800078002E4090000000FB005D
:107F10008080400000FD2F00008F4000E3FF37000D
:107F20003E0090000080FA00000006000200FA0007
:107F3000881F78005DFF0700004478005BFF0700A2
:107F4000084F7800104798001E0078004F04780012
:107F50000080FA00000006000200FA00881F780086
:107F600068FF07000044780066FF0700084F7800AC
:107F7000104798001E0078004F0478000080FA0037
:107F8000000006000400FA00889FBE008A1F7800E7
:107F900046FF07008044780044FF07000045780052
:107FA00042FF07000044780040FF0700094F7800B7
:107FB0001A47980028479800304798001E00BE00D6
:107FC0004F0578004F04BE000080FA000000060054
:107FD0000400FA00889FBE008A1F780049FF07004E
:107FE0008044780047FF07000045780045FF070000
:107FF0000044780043FF0700094F78001A479800B3
:1080000028479800304798001E00BE004F057800B2
:108010004F04BE000080FA00000006000200FA00D3
:1080200021A020009140780003CABF000001EB00AE
:10803000020F780080CF50000200320010002000B4
:10804000000F78001E0078000080FA000000060093
:108050000200FA0071E020009140780008CEBF00D5
:108060000001EB00020F780080CF500002003200C8
:1080700010002000000F78001E0078000080FA0039
:10808000000006000200FA00C120210091407800A3
:108090000DD2BF000001EB00020F780080CF50002E
:1080A0000200320010002000000F78001E0078004F
:1080B0000080FA00000006000E00FA00889FBE0053
:1080C0008A9FBE00500798005E00900090407800A4
:1080D000014F98006000B800200798003107980011
:1080E0000000EB00000F780020002000100798002F
:1080F000040037001E0FE8001E0090000000E8009A
:10810000100798001E009000800078005E0090002C
:1081100000804000104078000004E000F5FF3A00C5
:108120002000200010079800240037002E00900047
:10813000BE009000BFE907000005BE001E009000D1
:10814000800078005E0090000080400010407800C1
:108150008000FB0000FD2F0000804000CF80DE008B
:10816000B4E907000004BE001E0090001E001000CD
:108170000000E800CF80DE00AEE907000001BE008D
:108180000000200001122400D1EA07000001BE0017
:108190000800BE009AEA07000001BE000A00BE0007
:1081A0005DE707003EE907002007980031079800C7
:1081B0001E0090000000E800100798001E009000CC
:1081C000800078005E009000008040001040780041
:1081D0000004E000D5FF3A000E4890000000FB00CC
:1081E0006007980010032000EE009000808F500080
:1081F0000500320020032000EE009000808F500028
:108200001D003200370037002342A90021E2A900F7
:108210002E009000BE00900083E907000002BE001F
:108220000203BE006000B80002482800E3122400E8
:108230000AE807006022B8000600200007FF2300BC
:10824000EFEB070037E907004011880000C0240069
:10825000001188008560A9008580A9009560A800AC
:108260009580A800F03522001011880021E2A800B6
:108270002342A8001B0037003342A90031E2A900C5
:108280002E009000BE00900067E907000002BE00CB
:108290000203BE006000B80002482800E312240078
:1082A000EEE707006022B8000600200007FF230069
:1082B000D3EB07001BE90700C011880000C02400B1
:1082C0008011880087C0A90087E0A90097C0A80096
:1082D00097E0A800F03522009011880031E2A80054
:1082E0003342A8004F05BE004F04BE000080FA00D4
:1082F00000000600809FBE00829FBE003400F80090
:1083000010002000A00188000000FA008560A9008C
:108310000B00370033A02000934178008380FB00DE
:1083200030118000004178004120B0000080200022
:1083300000804000024878000340E80003EAB700EC
:1083400022C2BF00614060000004E000F1FF3A007B
:108350000080FA003400F9004F01BE004F00BE005B
:1083600000400600809FBE00829FBE003400F800DF
:1083700010002000A00188000000FA0087C0A900BA
:108380000C00370083E02000934178008380FB00DD
:10839000B011800000417800906020008080400093
:1083A0000080200000804000024878000340E80080
:1083B00008EEB70032C2BF00614060000004E00078
:1083C000F0FF3A000080FA003400F9004F01BE00CF
:1083D0004F00BE0000400600809FBE00829FBE008E
:1083E0003400F80010002000A00188000000FA000E
:1083F0008E40A9000C003700D32021009341780063
:108400008380FB00B012800000417800E0A02000D3
:1084100080804000008020000080400002487800FA
:108420000340E8000DF2B70052C2BF006140600097
:108430000004E000F0FF3A000080FA003400F90088
:108440004F01BE004F00BE0000400600809FBE00EE
:10845000821F78003400F80010002000A00188007E
:108460000000FA008580A9000A0037000280200081
:10847000124178000280FB008080E800008020002C
:10848000008040001040780024E2B7000240E8007D
:1084900000E8B70023C2BF00624060000004E000B3
:1084A00005003A00018020009140780001C8BF001B
:1084B00080CF5000EDFF3A000080FA003400F90050
:1084C0004F0178004F00BE0000400600809FBE00B4
:1084D000821F78003400F80010002000A0018800FE
:1084E0000000FA0087E0A9000B00370052C020000E
:1084F000124178008280FB007040200080804000A4
:1085000000802000008040001040780034E2B70076
:108510000240E80005ECB70033C2BF0062406000D3
:108520000004E00005003A0051C0200091407800AE
:1085300006CCBF0080CF5000ECFF3A000080FA006C
:108540003400F9004F0178004F00BE0000400600E3
:10855000809FBE00821F78003400F80010002000C9
:10856000A00188000000FA008E60A9000B0037000F
:10857000A2002100124178008280FB00C080200010
:108580008080400000802000008040001040780083
:1085900044E2B7000240E8000AF0B70053C2BF004F
:1085A000624060000004E00005003A00A1002100E4
:1085B000914078000BD0BF0080CF5000ECFF3A0014
:1085C0000080FA003400F9004F0178004F00BE002F
:1085D000004006000400FA00004F780090C0B3008D
:1085E0009E4F100005003E001E4078000043B00082
:1085F0000080FB00100798000A003700F0C0B300AD
:108600009E4F100005003E001E4078007043B000F1
:108610000080FB00100798000200370000032000D4
:10862000100798001E0090000080FA00000006006D
:108630000400FA00004F7800F0C2B3009E4F100013
:108640000900360090C3B3009E4F100006003E00A4
:108650009E40780000CDB30000C040000080FB00C9
:10866000100798000E00370000C4B3009E4F1000A2
:108670000900360060C4B3009E4F100006003E00A3
:108680009E40780090CCB30000C040000080FB000A
:108690001007980002003700F00F20001007980024
:1086A0001E0090000080FA00000006000200FA00A0
:1086B000004F78001E80FB004400DE00C5FF07006D
:1086C0000080FB000080FA00000006000200FA00B3
:1086D000004F78009E4078006FC06000BDFF07002B
:1086E0000080FB000080FA00000006000200FA0093
:1086F000881F7800004F7800114798001E409000B6
:10870000CBFF0700004478001E407800C8FF070038
:108710000080FB004400DD00004074000080FB008E
:108720004F0478000080FA00000006000400FA0000
:10873000000F78001E00E00003003D001E00EA006C
:1087400010079800020037001E00780010079800FC
:108750001E0090000080FA00000006000200FA00EF
:10876000004F78009E80FB00000820000080600021
:108770004780DE00004178009E80FB00000420005E
:10878000008060004580DE00004171009E80FB009B
:1087900000022000008060004380DE008040710005
:1087A0001E80FB00700060000080D10080C070005F
:1087B0001E80FB00680060000000400080C0700068
:1087C0001E80FB00640060004300DD0080C070007C
:1087D0001E80FB00620060004500DD0080C070006C
:1087E0001E80FB00610060004700DD0000C07000DB
:1087F0000080FB000080FA00000006000200FA0082
:10880000004F78001E80FB00A2002000110009002C
:108810000280D8008000FD00804078001E80FB00B0
:10882000A2002000811F7800110009000280D800FA
:1088300001017800CF0078000080FB004400DD00DB
:1088400000C070000080FB000080FA0000000600FD
:108850000200FA00004F78001E4078006F4160006F
:108860001E80FB004400DE000080FB006A00B900AF
:10887000004041000080FB000080FA00000006007C
:108880000800FA003007980000C3B3004047980082
:1088900000712200100798000000EB00000F780024
:1088A000060037009E00780060ED210080804000C7
:1088B0000040EB00804878001E0FE8001E007800A2
:1088C000E40F5000F7FF36000000EB00000F7800C7
:1088D000270037004E4090000040E80040479800D5
:1088E000BE0090001E0090000080500030079800ED
:1088F000BE0090001E009000808F5000F5FF3D00EC
:108900001E00E0000D003A00CE40900000C3B3000E
:1089100080CF500009003A001E009000E10F500087
:108920000E003A001E00780061ED210001004000B9
:10893000CE40900001487800080037009E00780083
:1089400060ED210000804000CE409000014878009A
:108950001E0FE80000C3B300404798001E009000BF
:10896000A2002000110009000200D80010079800A2
:108970001E0090000000E000DDFF3C0060ED2100E3
:108980000080FA00000006000200FA00000F7800E4
:108990001E00780004000700B9FF0700000F7800F0
:1089A0000080FA00000006000C00FA005007980052
:1089B0006000B800008FBE000000EB003007980098
:1089C000030037003E0090000000E80030079800E8
:1089D0003E009000800078005E0090000080400023
:1089E000104078000004E000F6FF3A000000EB00C1
:1089F00040079800180037004E0090008000780073
:108A00005E009000008040001040780008FF0700E2
:108A10000080FB0020079800AE009000F00F2000BF
:108A2000808F5000090032001E00BE004409DD00A6
:108A3000CC01DE00830171004401DD002E009000B6
:108A4000CF80DE00001F4100019749004E009000DA
:108A50000000E80040079800CE0090003E00900023
:108A6000808F5000E4FF35001E00BE000080FA0039
:108A7000000006000600FA00100798002107980081
:108A80002E0090008080E8000040EB0080487800D5
:108A90002E0090008000E8001E0090006F406000F3
:108AA000804878001E0090004480DE0080407800FE
:108AB0002E009000014878000000EB00000F7800C5
:108AC0000F0037001E007800800078002E00900014
:108AD0000080400010407800E94F5000040034004E
:108AE0002E0090007005B0002007980003003700AA
:108AF0002E0090000003B000200798001E0FE80031
:108B0000100020009E0F1000EEFF34002E00900099
:108B10000000E800104078003BFB07002E009000AA
:108B20001040780038FB07002E00900023FC07005F
:108B30002E0090000080FA00000006000200FA00FB
:108B4000F402A800F422A800F002A900F022A90073
:108B5000113A8000F00B20000081600061042000C9
:108B60007005200023742000814978008049780036
:108B700082497800816A20009140780000CCB300DF
:108B800000C06000A1C2B30001407000A8E6B700B9
:108B9000C16C20009140780000CCB30000C06000A0
:108BA0007040B300CCE6B700316C200091407800F3
:108BB00000CCB30000C060000034A000C3E6B700E2
:108BC000113A800000042000008170006104200040
:108BD00070052000237420008149780080497800C6
:108BE000824978008540A9009540A80030122E00E7
:108BF00010128800D0FF21002012880070FA2D008A
:108C000000128800C0C9B300004F78001E00780031
:108C1000B10107000080FA00000006000200FA001F
:108C2000004F780040C2BF00624060000004E000D6
:108C3000FCFF3A001E80FB00401288000100370054
:108C40000140FE0040C2BF000042B2000004E0004C
:108C5000FBFF3A00401280000080FB000080FA0019
:108C6000000006003400F800881F7800180020007B
:108C7000A80188004F0478000000FA008540A90090
:108C80000080FA003400F900004006000200FA00FB
:108C90000E007800810107001E007800610060006E
:108CA0000000E000FAFF3A000080FA000000060031
:108CB0000400FA00008FBE001E00BE004008DE0067
:108CC00001002000D5FF07001E00BE004809DD009E
:108CD0004800DE0000007100C808DE00CFFF07007A
:108CE0001E007800CDFF07000080FA00000006009B
:108CF0000A00FA00881F78001007980021079800E2
:108D00003207980043079800E0FF0700F402A9002B
:108D100030C0B300C1FF07001E009000AE009000FD
:108D2000E3FF07000000EB00000F780007003700AA
:108D30009E0078003E009000008440000040EB0060
:108D4000B6FF0700004C78001E0FE8004E009000B0
:108D50009E0F1000F6FF3900F402A8004F047800BF
:108D60000080FA00000006000C00FA00400798009E
:108D700051079800E40047000040EB00804878006D
:108D8000E40047000040EB0090409800E4004700FA
:108D90000040EB00A0409800640147003300200031
:108DA0004E009000DE009000D1FF070064004700F5
:108DB000104078000080FB0001002000008FBE0002
:108DC0001E00BE004809DD00C801DE0083017100FD
:108DD0004801DD0064004700104090000080FB0067
:108DE00001002000001F4100019749001E00BE0045
:108DF0004809DD00C801DE00830171004801DD0083
:108E000064004700204090000080FB00010020002B
:108E1000001F4100019749001E00BE000080FA00BB
:108E2000000006000800FA002007980031079800AB
:108E30008E80E8000040EB00804878008E80E800DB
:108E40000040EB00904098000000EB00000F78001D
:108E50000E81E800230020002E009000BE0090004C
:108E6000A3FF07000E80E800104078000080FB00A0
:108E7000000F78001E007800C800DD000E80E800BA
:108E8000104090000080FB00008F40001E00780022
:108E90000080FA00000006000600FA0010079800A3
:108EA000210798000040EB00004F78000040EB00E5
:108EB00010479800130020000E0178001E0090005B
:108EC000AE0090008AFF07001E4078000080FB0083
:108ED0000080FA00000006000C00FA00100798005D
:108EE0002107980032079800430798006A0047005E
:108EF000EA0007005E009000000F780030FC2F00B1
:108F00001E0F60001E007800F30007000301070039
:108F10003E009000CE0090004008DE0001002000DE
:108F2000004178001E009000AE0090008200070013
:108F3000FA0007003E009000CE0090004809DD00D6
:108F40004800DE0000007100C808DE000041780023
:108F50001E009000AE00900061004000E0804800DC
:108F600075000700ED0007003E009000004178000A
:108F70001E009000AE00900062004000E0804800BB
:108F80006D00070030FC2F001E0F60001E007800EF
:108F90007C0F70001E007800CF0007000080FA00F0
:108FA000000006000A00FA00100798002107980048
:108FB0003207980068004700B80007004E00900094
:108FC000000F780030FC2F001E0F60001E0078009C
:108FD000C1000700D10007003E0090004800DE00FD
:108FE000004178001E009000AE0090005200070083
:108FF000CA0007003E009000004178001E0090006B
:10900000AE00900061004000E08048004A00070088
:1090100030FC2F001E0F60001E0078007C0F7000D7
:109020001E007800AC0007000080FA000000060077
:109030000A00FA001007980021079800624798007C
:1090400068004700950007004E009000000F780070
:1090500030FC2F001E0F60001E0078009E000700ED
:10906000AE0007006E4190001E009000AE00900020
:109070003100070030FC2F001E0F60001E0078003A
:109080007C0F70001E007800930007000080FA003B
:10909000000006000400FA00008FBE00FBFE07007F
:1090A000F402A90000C2B300DCFE07001E00BE00EF
:1090B000FFFE0700F402A8000080FA00000006008E
:1090C0000400FA00008FBE00F0FE0700F402A900C1
:1090D00020C5B300D1FE07001E00BE00F4FE07004D
:1090E000F402A8000080FA00000006000400FA0064
:1090F000008FBE00E5FE0700F402A90080CDB3009A
:10910000C6FE07001E00BE00E9FE0700F402A8002C
:109110000080FA00000006000000FA00DBFE0700F5
:10912000F402A90000C6B300BCFE0700F402A800C8
:109130000080FA00000006000600FA00008FBE0062
:1091400042479800D1FE0700F402A90020C0B300F6
:10915000B2FE07001E00BE00D5FE07004E40900084
:10916000AEFE0700F402A8000080FA00000006002E
:109170000A00FA00100798002107980032079800AB
:10918000430798000000EB00000F7800BFFE0700C7
:10919000F402A900D0CAB300A0FE07001E00900090
:1091A000AE009000C2FE07009E0078003E009000D6
:1091B00000804000104078001E0FE80097FE070076
:1091C0009E0078003E009000008040000000E80013
:1091D000104078000004E000070032009E00780094
:1091E0003E00900000804000104078001E0FE80014
:1091F0008AFE07000200370000C0EB0087FE070070
:10920000F402A800A1FE07001B003700F402A90029
:10921000D0CAB30081FE07009E0078003E00900097
:1092200000804000104078001E0FE8007BFE070021
:109230009E0078003E009000008040000000E800A2
:10924000104078000004E000070032009E00780023
:109250003E00900000804000104078001E0FE800A3
:109260006EFE07000200370000C0EB006BFE070037
:10927000F402A80085FE07004E0090009E0F10002B
:10928000E2FF3900F402A90040C0B30063FE07000A
:10929000F402A8000080FA00000006000200FA00B4
:1092A000881F780000047800F402A90050C0B300C1
:1092B0005AFE07000040EB0058FE0700004F780000
:1092C000F402A8001E0C7800080078004F04780013
:1092D0000080FA00000006000200FA00000F78008B
:1092E0006AFE0700F402A90000C5B3004BFE0700A8
:1092F000F402A800F422A800F402A90010C0B300F0
:1093000046FE07001E40780044FE0700F402A80055
:10931000F422A9000080FA00000006000000FA0014
:109320005AFE0700F402A90060C0B3003BFE07002C
:10933000F402A8000080FA00000006000000FA0015
:1093400052FE0700F402A90040C0B30033FE07003C
:10935000F402A8000080FA00000006000400FA00F1
:109360004AFE0700F402A90000C9B3002BFE070063
:109370000040EB0029FE07000040EB0027FE07003D
:109380000040EB0025FE07000040EB0023FE070035
:109390000080FB0001002000008FBE001E00BE0008
:1093A000C808DD000080FD00804078000040EB0030
:1093B000008FBE000040EB0018FE07000080FB009D
:1093C000010020001E1F70001E9770001E00BE00CE
:1093D000C808DD000080FD00804078000040EB0000
:1093E000008FBE000040EB000CFE07000080FB0079
:1093F000010020001E1F70001E9770001E00BE009E
:10940000C808DD000080FD00804078000040EB00CF
:10941000008FBE000040EB0000FE07000080FB0054
:10942000010020001E1F70001E977000F402A800AB
:109430001E00BE000080FA00000006000C00FA00CA
:10944000D0FA07004007980051079800CDFA0700AE
:1094500020079800310798000CFE0700F402A900CD
:1094600030C0B300EDFD07004E009000DE0090001C
:109470000FFE07006000B800008FBE000700370035
:109480000040EB00E5FD0700A0F8070010002000F9
:10949000010020001E0F40005E9748002E00900043
:1094A000BE009000BE0F1000AE8F1800F4FF390010
:1094B000F402A800A0C0B30094F807000080FA00EE
:1094C000000006000C00FA00200798003107980001
:1094D00042079800530798000000EB00100798001F
:1094E00000C8B300204798002E019000BE019000F4
:1094F0004E009000DE009000020040008380480093
:1095000061005000E08058004008DE0001002000AB
:10951000004F7800E0C3B3009E4F100007003600F4
:109520001E0090000020A1000030A1000040A1001A
:109530000050A1001007980038003700D0C3B300D6
:109540009E4F1000070036001E0090000020A00073
:109550000030A1000040A1000050A10010079800B9
:109560002E003700B0C3B3009E4F10000700360036
:109570001E0090000020A1000030A0000040A100CB
:109580000050A100100798002400370070C3B300FA
:109590009E4F1000070036001E0090000020A00023
:1095A0000030A0000040A1000050A100100798006A
:1095B0001A003700F0C2B3009E4F100007003600BB
:1095C0001E0090000020A1000030A1000040A0007B
:1095D0000050A1001007980010003700F0C1B30040
:1095E0009E4F1000070036001E0090000020A000D3
:1095F0000030A1000040A0000050A100100798001A
:10960000060037001E0090000020A1000030A000DE
:109610000040A0000050A100100798001E0090001C
:109620002DFF07003DFF07000080FA000000060044
:109630000E00FA0053FA07004007980051079800FF
:1096400050FA070020079800310798006000B80022
:10965000008FBE000000EB0060079800C0C9B30097
:10966000404F98002E019000BE0190004E009000E7
:10967000DE00900093FF0700F402A900D0CAB300F7
:1096800066FD07004E009000DE00900088FD070098
:1096900086F9070061FD0700F402A8007BFD0700C2
:1096A00010002000010020001E0F40005E974800BF
:1096B0000B003700F402A900D0CAB30057FD070021
:1096C0007AF9070055FD0700F402A8006FFD0700B6
:1096D00010002000010020001E0F40005E9748008F
:1096E0002E009000BE009000BE0F1000AE8F18003C
:1096F000F0FF3900F402A90040C0B30047FD0700A5
:10970000F402A8006E009000F3FE0700A0C0B300B2
:10971000FEF707000080FA00000006000E00FA00C5
:1097200018FA0700200798003107980015FA07007B
:10973000008FBE000000EB0040079800C0C9B300D6
:10974000004F98001E01BE002E009000BE00900049
:109750005CFF07001E00BE005007980061079800DC
:1097600000002800010020005E019000EE01900042
:10977000800F5100818F590013003200000020003B
:10978000210020005E019000EE019000800F51004A
:10979000818F5900100032000000210001002000DC
:1097A0005E019000EE019000800F5100818F590002
:1097B000010032000A0037002E009000BE00900029
:1097C00034FE0700090037002E009000BE00900014
:1097D0003BFE0700050037004FFE0700030037007F
:1097E0004E009000BCFE0700040037004E009000C1
:1097F000B9FE0700A0C0B300C4F707000080FA005C
:10980000000006000600FA00008FBE002207980044
:109810000080FA00000006000000FA000080FA0054
:10982000000006000200FA006000B80070F0880036
:1098300081F08800C002A900C022A900C042A9008E
:10984000C062A900C082A900C0A2A900C0C2A9002C
:10985000C0E2A900C942A900C8A2A9000000EB000B
:10986000CA000700D0F82500900888000000EB002F
:10987000500888008500A9009500A800D0F82500B0
:10988000000988000000EB00C00888008780A9005C
:109890009780A80000322000700888000000EB00CC
:1098A000800C88000000EB00900C8800003720003E
:1098B000B00C8800211920009140780000CEB30040
:1098C00000C06000D040B30092E1B7001119200041
:1098D0009140780030CEB30000C060000024A000AA
:1098E00091E1B700011920009140780080CFB300CA
:1098F00000C060003040B30090E1B7008440A90090
:109900009440A8000000EB00D00C88000000EB00A1
:10991000E00C880000372000000D8800C1192000ED
:109920009140780000CEB30000C06000D040B3008A
:109930009CE1B700B11920009140780030CEB3000F
:1099400000C060000024A0009BE1B700A119200026
:109950009140780080CFB30000C060003040B30079
:109960009AE1B70084C0A90094C0A800C442A8002E
:10997000C462A900C4C2A800C4E2A900C402A8002D
:10998000C422A900C482A800C4A2A9000000EB0060
:10999000000F7800300037001E0078006A00B90020
:1099A0008000780020CE2100008040001010A00030
:1099B0001E0078006A00B9008080E80020CE2100F7
:1099C0008080400060012000800878001E00780040
:1099D0006A00B900E400400020CE210080804000F1
:1099E0000000EB00800878001E0078006A00B900D3
:1099F000E600400020CE2100808040000000EB0007
:109A0000800878001E0078006A00B900E800400075
:109A100020CE2100808040000000EB00800878000C
:109A20001E00780080004000E0CD210080804000D2
:109A30000000EB00800878001E0078000000400065
:109A4000E600400040E02100808040000000EB0084
:109A5000800878001E0FE800100020009E0F100004
:109A6000CDFF3400B31007001000200030000700C5
:109A70000E1EA900500107000E1EA8000000EB00FA
:109A80002B00070023002000E23D22006000B80008
:109A900097FC0700E03D2200104078000080FB00AA
:109AA0004800DD00C0ED8800C1ED8000F03D2200DF
:109AB000104078000080FB0000807000C0ED88003E
:109AC00023002000E23D22002000200001002000B1
:109AD00087FC0700E03D2200104078000080FB007A
:109AE0004800DD00D0ED8800D1ED8000F03D22007F
:109AF000104078000080FB0000807000D0ED8800EE
:109B0000C0ED80000000E00002003A00405D20004F
:109B1000C0ED8800D0ED80000000E00002003A00B7
:109B200000462000D0ED88000080FA00000006000A
:109B30000200FA00000F78001E00E0000A00320068
:109B40000000EB005008880013E1A800CD42A900F6
:109B50000001EB00F10F2000F00F2000201F070094
:109B6000DC82A9000700370013E1A900CD42A8005C
:109B70000001EB00F10F20000000EB00181F0700B0
:109B8000DC82A8000080FA00000006000200FA0053
:109B9000000F78001E00E0000E003200CCC2BF00B3
:109BA0000042B2000004E0000C003A000001EB00AB
:109BB0008000EB00F00F2000091F0700CCA2A800D6
:109BC00000202100A107200094EF0700DC42A8003C
:109BD00002003700CCA2A900DC42A9000080FA00F4
:109BE000000006000200FA00000F78000001EB0000
:109BF000F10F2000F00F2000F91E07001E00780072
:109C00006A00B900E800400020CE2100008040003A
:109C1000100178001E0078006A00B900E6004000DC
:109C200020CE21000080400010007800800F5100FD
:109C3000250031001E00780080004000E0CD2100AA
:109C40000080400010007800E30F500007003A0049
:109C50001E00780080004000E0CD210080804000A0
:109C60000000EB00800878000A0037009E007800B2
:109C700001814000E0CD210000004100100078008B
:109C80000001E80081804000E0CD2100008040001C
:109C9000020878001E0178006A10B900E800400050
:109CA00020CE210000804000100078008001E800F4
:109CB0006A10B900E800400020CE2100008040007A
:109CC00003087800240037001E0078008000400060
:109CD000E0CD210000804000100078000000E0008E
:109CE00007003A001E00780080004000E0CD21000F
:109CF0008080400030002000800878000A00370093
:109D00009E00780001814000E0CD2100000041006C
:109D1000100078000001E90081804000E0CD2100C2
:109D200000804000020878001E0178006A10B90027
:109D3000E800400020CE21000080400010007800A4
:109D40008001E9006A10B900E800400020CE21003F
:109D50000080400003087800100020009E0F1000D3
:109D600049003A001E00780080004000E0CD21004C
:109D7000008040001000780021DC2100000040003D
:109D80000100400010007800614060006140600008
:109D90004201DD00412C200091407800B0CFB3009B
:109DA00000C0600002407000C4E2B7001E007800EE
:109DB00080004000E0CD21000080400010007800CD
:109DC00021DC21000000400001004000100078006C
:109DD0000000D10061406000614060004301DD008F
:109DE000412C20009140780070CFB30000C060008B
:109DF00002407000C4E2B7001E00780080004000FE
:109E0000E0CD2100008040001000780021DC21001E
:109E10000000400001004000100078004200DE0019
:109E200061406000614060004601DD00412C20007F
:109E300091407800F0CBB30000C060000240700099
:109E4000C4E2B7001E00780080004000E0CD210091
:109E5000008040001000780021DC2100000040005C
:109E600001004000100078004300DE006140600007
:109E7000C700DD00C4C2BF000074A1000140700033
:109E8000C4E2B7004A0037001E007800800040009E
:109E9000E0CD2100008040001000780021DC21008E
:109EA00000004000010040001000780061406000A8
:109EB00061416000412C200091407800E0CFB30068
:109EC00000C0600002407000C4E2B7001E007800CD
:109ED00080004000E0CD21000080400010007800AC
:109EE00021DC21000000400001004000100078004B
:109EF0000000D1006140600061406000004140000E
:109F0000412C200091407800D0CFB30000C0600009
:109F100002407000C4E2B7001E00780080004000DC
:109F2000E0CD2100008040001000780021DC2100FD
:109F30000000400001004000100078004200DE00F8
:109F400061406000614060004401DD00412C200060
:109F500091407800F0CEB30000C060000240700075
:109F6000C4E2B7001E00780080004000E0CD210070
:109F7000008040001000780021DC2100000040003B
:109F800001004000100078004300DE0061406000E6
:109F9000614060004501DD00412C200091407800C7
:109FA000F0CDB30000C0600002407000C4E2B70012
:109FB0000080FA00000006000600FA000000EB0036
:109FC000F2FE070060E78000610060000000E00032
:109FD0001700320010E78000610060000000E00020
:109FE0001300320070F08000610060000000E000AB
:109FF0000F0032000000EB00000F7800080037006F
:10A000001E0078006A00B900E800400020CE210060
:10A01000808040000000EB00800878001E0FE80000
:10A02000100020009E0F1000F5FF3400E7003700FD
:10A030000E7EA8000000EB00000F78000E00370035
:10A040001E0078006A00B9008080E80020CE210060
:10A050008080400060012000800878001E007800A9
:10A060006A00B9008000780020CE21000080400006
:10A070001010A0001E0FE800100020009E0F10001E
:10A08000EFFF34004E1A070010E7800061406000C7
:10A090000080FB001007980060E7800061406000CE
:10A0A0000080FB002007980070F0800061006000D5
:10A0B0000000E0001B003A001E0090000000E000DD
:10A0C000180032000000EB0060F088000000EB0098
:10A0D00050F0880050E78000800CB00040E7880016
:10A0E000371A07000A00370021C1BF0001C8B300BA
:10A0F000014060000004E00004003A00C0E7800076
:10A100000000E00001003A0021E1A800740C070003
:10A1100041E7800050E78000808F5000F2FF3A0056
:10A12000080037004006200040E7880051E7800023
:10A1300040062000808F500002003E0040062000B4
:10A1400050E7880070F08000610060000000E000CF
:10A1500007003A002E0090000000E00004003200EA
:10A16000A0E78000C012B00090E788001800370018
:10A1700070F0800001002400010060000000E00099
:10A1800005003200A0E78000C1F92F000100400067
:10A1900090E788000E00370060E7800061006000F3
:10A1A0000000E00004003200A0E780004006B0009C
:10A1B00090E7880006003700A1E7800040062000F5
:10A1C000808F5000020036004006200090E7880093
:10A1D0000000EB0060F088000000EB0050F0880009
:10A1E00071F0800000082000008060000000E000A6
:10A1F00017003A0080F08000610060000000E0007D
:10A2000013003A0010002000720007000A00370017
:10A2100021C1BF0001C8B300014060000004E0009C
:10A2200004003A00C0E780000000E00001003A00AE
:10A2300021E1A8002A0C070091E78000A0E7800038
:10A24000808F5000F2FF3A000000EB006100070031
:10A250000000EB00000F78000000EB0060F08800C9
:10A260000000EB0050F08800530037001E0078001B
:10A270006A00B900E600400020CE210000804000C6
:10A28000100078000000E000160032001E00780088
:10A290006A00B900E600400020CE21008080400026
:10A2A0000000EB00800878001E0078006A00B9000A
:10A2B000E800400020CE210080804000007D20008A
:10A2C000800878001E0078006A00B9008080E800ED
:10A2D00020CE2100808040006001200080087800AE
:10A2E000B71907001E0078006A00B90080007800E6
:10A2F00020CE210000804000100078006140600006
:10A300000004E000080032001E0078006A00B90076
:10A31000E800400020CE2100808040000000EB00DB
:10A32000800878001E0FE8001E0078006A00B9005F
:10A33000E800400020CE210000804000100078009E
:10A340000000E0000F003A001E0078006A00B9002B
:10A35000E800400020CE210080804000007D2000E9
:10A36000800878001E0078006A00B9008080E8004C
:10A3700020CE21008080400060012000800878000D
:10A380008F190700100020009E0F10000A003C00EB
:10A3900021C1BF0001C8B300014060000004E0001B
:10A3A00004003A00C0E780000000E00001003A002D
:10A3B00021E1A800CA0B0700100020009E0F10002A
:10A3C000AAFF340021E1A9000E7EA9000080FA0056
:10A3D000000006001800FA00000F98000E08900018
:10A3E0000000E00065003200BC1DA80090012000C4
:10A3F000781A07007219070071E7800020E78000D3
:10A40000808F500002003100BC3DA80001003700E1
:10A41000BC3DA9000000EB00F0ED8800E0ED8000FD
:10A42000620060000000E0004F00320041E7800061
:10A4300050E7800000805000300F98003E089000E8
:10A440000000E00003003D003E0990000201EA0028
:10A45000320F98003E0890000000E0003F003400FA
:10A4600091E78000A0E7800000805000200F980056
:10A470002E0990000200E00003003D002E0890002D
:10A480000000EA00200F98002E0990006110B9002A
:10A49000E8E00700600798007107980041E7800036
:10A4A00050E7800000805000100F98001E089000B8
:10A4B0000000E00003003D001E0990000201EA00D8
:10A4C000120F98001E0990006110B900D9E0070032
:10A4D00040079800510798003033230031FF2300D4
:10A4E00020079800310798006E009000FE00900051
:10A4F0004E019000DE019000B2DF07002E019000B7
:10A50000BE01900083DE0700008FBE006011B8001E
:10A510001E00BE0060E007000000E00001003D00FA
:10A5200003003700A000200000EE88001000370074
:10A530000200200003122C001E00BE00B0E1070044
:10A5400037DF0700020020000312240072DE07003C
:10A5500053E0070000EE880005003700A00020004F
:10A5600000EE8800020037003001200000EE880075
:10A57000100020006EFD070001003700BC1DA9007F
:10A580000080FA00000006000E00FA00881F780024
:10A59000600798006E009000000F780080F0800047
:10A5A0004600DE00614060000040E800614060005D
:10A5B0000080FB00610060004601DD0081F080004A
:10A5C000F0FB2F00008060000200700080F0880027
:10A5D0000000EB00200798000000EB001007980037
:10A5E0003C0037000000EB0020079800080037000F
:10A5F000AE00900066004700808040000040EB0005
:10A60000804878002E0090000000E80020079800A5
:10A610002E009000E40F5000F5FF34000000EB0026
:10A62000200798000A0037002E0190002E009000AD
:10A630001E00400090407800660047000000410086
:10A64000014878002E0090000000E80020079800E4
:10A650002E009000E40F50000B003C002E009000F4
:10A660001E00400090407800C0C2B30080CF500070
:10A67000050032002E0090001E00400010407800BF
:10A680000004E000E8FF3A002E0090001E004000A9
:10A69000000FE80066004700104078000004E0006A
:10A6A000090032001E049000660047002EE50700F6
:10A6B000000178006A40B900E600400020CE210089
:10A6C00000804000020878001E0090000000E800B2
:10A6D000100798001E009000E10F5000C1FF3400E9
:10A6E000100020003BFF07004F0478000080FA00B4
:10A6F000000006000800FA000000EB0010079800B8
:10A700000000EB00000F78000FFEA8000000EB0037
:10A71000100798000F0037001E0190001E009000E7
:10A720006A00B9008080E80020CE2100008040004F
:10A730001000780080007800020041000E00400008
:10A7400064004000010878001E0090000000E8004E
:10A75000100798001E009000E10F5000EEFF34003B
:10A760000000EB0010079800230037001E0078005F
:10A770006A00B900E600400020CE210000804000C1
:10A78000100178001E0078006A00B900E80040005F
:10A7900020CE21000080400010007800800F510082
:10A7A0000D00320021C1BF0001C8B30001406000AC
:10A7B0000004E00004003A00C0E780000000E00070
:10A7C00001003A0021E1A800C50A07000000EB00E3
:10A7D00010079800030037001E0090000000E800FA
:10A7E000100798001E00E000020032001E0FE90072
:10A7F000010037001E0FE8001E009000E10F50001E
:10A80000DAFF34000000EB00100798000F0037005B
:10A810009E0090001E009000000040000E004000CE
:10A820006400400010007800000178006A08B90058
:10A830008080E80020CE21000080400002087800DF
:10A840001E0090000000E800100798001E00900015
:10A85000E10F5000EEFF34000FFEA9000080FA0067
:10A86000000006004400FA00889FBE0020479800C0
:10A870000000EB00000F78002E4090000000FB006D
:10A880006101B9000227980013279800A00020005A
:10A89000010020000E2190009E219000800F5100A9
:10A8A000818F590005043E000E2090009E209000EC
:10A8B000006001000A0037005600370076003700BC
:10A8C0009E003700B0003700760137001F023700C6
:10A8D000420237001F0337005F033700820337004F
:10A8E00001C3B3000000EB0087EC07006000B80074
:10A8F00090F08800A1F088000FDEA8000000EB00B7
:10A90000000F7800070037001E0078006A00B900C9
:10A910008000780020CE2100008040001010A000B0
:10A920001E0FE800110020009E8F1000F6FF34007B
:10A93000B8E40700E2152000110009000200D80069
:10A940008000FD004006B00030E8880010EF800075
:10A95000CF80DE00B7DF07000001BE00000020004E
:10A96000C14824006BDD070002002000832C240076
:10A9700068DD070002002000832C2400A0E007000F
:10A9800002002000832C24008EDE07008BDF0700EE
:10A9900040E7880030E88000CF80DE00A5DF0700B8
:10A9A0000001BE0000002800A14B240059DD070073
:10A9B00002002000832C240091E007000200200008
:10A9C000832C24007FDE07007CDF070090E78800EF
:10A9D00080022000FF180700F917070040E78000F9
:10A9E00091E78000801F7800811F780040402A0096
:10A9F000801F780060412100ABE40700E687570024
:10AA0000604121006DF407001000200048FC0700A1
:10AA1000AA033700139EA80010EF8000CF80DE004D
:10AA200084DF07000001BE0000002000C1482400B0
:10AA300038DD0700020020008334240036DD0700E3
:10AA400002002000832C24006DE00700020020009B
:10AA5000832C24005BDE070058DF070040E78800F6
:10AA600040E78000801F780060412A00801F780046
:10AA7000604121008CE40700E48757006041210019
:10AA80004EF4070040062000D2180700E23CA9005F
:10AA9000CB17070089033700139EA90013BEA80037
:10AAA000123EA80000462000D0ED880058E7800044
:10AAB0006140B9005FDF0700601F9800711F9800B8
:10AAC0000800E00007003D00020020000378240099
:10AAD0006E189000FE1890000FDD0700601F9800B0
:10AAE000711F980002002000031A24006E189000C5
:10AAF000FE18900007DD070030DF070040E7880000
:10AB000040E7800051E78000801F7800811F7800B7
:10AB100050422A00801F78006041210062E4070053
:10AB2000E68757006041210024F40700400620001A
:10AB3000A8180700A217070060033700123EA900FB
:10AB4000121EA800E06C200090E78800E23CA800FC
:10AB5000EC3CA90090E78000801F780000442A00A8
:10AB6000801F7800604121004FE40700E487570010
:10AB70006041210011F407004006200095180700ED
:10AB80008F1707004D033700121EA900A0E78000B1
:10AB9000801F7800D0442A00801F78006041210087
:10ABA00041E40700E48757006041210003F40700F7
:10ABB00090F08000640060000000E00026003A0091
:10ABC000A8E780006140B9001ADF0700401F980025
:10ABD000511F98000800E00007003D00020020001F
:10ABE000037824004E189000DE189000CADC07009D
:10ABF000401F9800511F980002002000832C240061
:10AC00004E189000DE189000FDDF070002002000C3
:10AC1000832C2400EBDD0700E8DE0700B0EE88009F
:10AC200090F080004200DE00614060000040E800DB
:10AC3000614060000080FB00610060004201DD00B7
:10AC400091F08000B0FF2F000080600002007000D3
:10AC500090F088005300370090F08000680060009A
:10AC60000000E00026003A00A8E780006140B9003B
:10AC7000F0DE0700201F9800311F98000800E00058
:10AC800007003D0002002000037824002E189000E9
:10AC9000BE189000A0DC0700201F9800311F98000C
:10ACA00002002000832C24002E189000BE18900073
:10ACB000D3DF070002002000832C2400C1DD070041
:10ACC000BEDE0700C0EE880090F080004300DE008A
:10ACD000614060000040E800614060000080FB00CF
:10ACE000610060004301DD0091F0800070FF2F00E3
:10ACF000008060000200700090F08800290037009A
:10AD000090F08000700060000000E00025003A0034
:10AD1000A8E780006140B900C6DE0700001F980068
:10AD2000111F98000800E00007003D00020020000D
:10AD3000037824000E1890009E18900076DC07001F
:10AD4000001F9800111F980002002000832C24008F
:10AD50000E1890009E189000A9DF07000200200046
:10AD6000832C240097DD070094DE0700D0EE8800D6
:10AD700090F080004400DE00614060000040E80088
:10AD8000614060000080FB00610060004401DD0064
:10AD900091F08000F0FE2F00008060000200700043
:10ADA00090F0880090F08000700060000000E000EB
:10ADB0002A003200210020000000EB00C202070040
:10ADC0000000E00012003A0090F0800001402000F6
:10ADD000010060000000E0000600320012DEA80062
:10ADE0000000EB0069FB0700B0452A0073F3070081
:10ADF000B2023700135EA800125EA900127EA900FD
:10AE0000129EA90070472A006CF307001300370058
:10AE1000B1EE8000C0A22F000080400080EF8800CB
:10AE20007CE30700221C2000110009000200D8006A
:10AE30008000FD007400400030E888006000B80029
:10AE400090F08800A1F0880013DEA800139EA800EF
:10AE500050C0B30083FE070098023700A1E78000CE
:10AE600040FC2F000080400090E788004006200052
:10AE7000D8170700D2160700123EA80090E78000FE
:10AE8000801F780050482A00801F78006041210010
:10AE900085E30700E48757006041210047F307007E
:10AEA00086023700125EA90090F0800001002100A8
:10AEB000010060000000E0001C003200A1E78000FB
:10AEC00030E88000008450006140B90059DE07007E
:10AED00060179800711798000800E00007003D0017
:10AEE00002002000037824006E109000FE109000F5
:10AEF00009DC070060179800711798000200200015
:10AF0000832C24006E109000FE1090003CDF0700A0
:10AF100002002000832C24002ADD070027DE070022
:10AF200090E78800139EA9007A00370090F0800017
:10AF3000700060000000E0003A003A0090F08000ED
:10AF400001402000010060000000E0001A00320013
:10AF5000A0E780006A0440006140B90035DE0700C8
:10AF600040179800511798000800E00007003D00C6
:10AF700002002000037824004E109000DE109000A4
:10AF8000E5DB0700401798005117980002002000E9
:10AF9000832C24004E109000DE10900018DF070074
:10AFA00002002000832C240006DD070003DE0700DA
:10AFB00090E7880057003700A1E78000A0D82F0055
:10AFC000008440006140B9001ADE07002017980095
:10AFD000311798000800E00007003D000200200043
:10AFE000037824002E109000BE109000CADB0700EA
:10AFF000201798003117980002002000832C2400AD
:10B000002E109000BE109000FDDE07000200200010
:10B01000832C2400EBDC0700E8DD070090E78800C4
:10B020003C00370090F08000700060000000E000FD
:10B030001F00320090F0800001022000010060003B
:10B040000000E0001A003A00A0E780006A04400017
:10B050006140B900F7DD070000179800111798004C
:10B060000800E00007003D000200200003782400F3
:10B070000E1090009E109000A7DB070000179800AC
:10B080001117980002002000832C24000E1090005D
:10B090009E109000DADE070002002000832C2400BE
:10B0A000C8DC0700C5DD070090E7880019003700FD
:10B0B000A0E78000740450006140B900DDDD0700A6
:10B0C000600F9800710F98000800E00007003D0035
:10B0D00002002000037824006E089000FE08900013
:10B0E0008DDB0700600F9800710F980002002000B0
:10B0F000832C24006E089000FE089000C0DE07003C
:10B1000002002000832C2400AEDC0700ABDD07002A
:10B1100090E7880090E78000801F780020492A008F
:10B12000801F780060412100DFE20700E4875700BC
:10B1300060412100A1F2070040062000251707000A
:10B140001F160700123EA800DC013700123EA900BE
:10B1500048E780006140B900B6DD0700400F980065
:10B16000510F98000800E00007003D000200200099
:10B17000037824004E089000DE08900066DB07008C
:10B18000400F9800510F9800020020000322240075
:10B190004E089000DE0890005FDB070087DD0700A7
:10B1A00040E7880040E78000801F7800004A2A00BE
:10B1B000801F780060412100BBE20700E487570050
:10B1C000604121007DF207004006200001170700C2
:10B1D000FB150700121EA800B8013700121EA900B7
:10B1E00050E78000801F7800C04A2A00801F780046
:10B1F00060412100ACE20700E48757006041210074
:10B200006EF2070090F08000700060000000E00027
:10B210000D003A0090F080004300DE0061406000C5
:10B220000080FB0052E780006600B90080007800D3
:10B2300060DD21000080400002087800129EA80016
:10B24000139EA900A000370090F0800070006000FD
:10B250000000E0001100320090F0800001022000A8
:10B26000010060000000E0000C003A0090F0800057
:10B270004300DE00614060000080FB0052E7800078
:10B280006600B9008080E80060DD21000080400099
:10B290000208780012BEA8008B00370090F08000F2
:10B2A0004300DE00614060000080FB0052E7800048
:10B2B0006600B900E400400060DD2100008040002D
:10B2C0000208780090F080004300DE0061406000DA
:10B2D0000080FB00110020007B0107000000E0005F
:10B2E0000F003A0090F08000014020000100600053
:10B2F0000000E0000600320012DEA8000000EB00B3
:10B3000022FA0700B0452A002CF207006C00370033
:10B31000135EA80070472A0028F207006800370073
:10B3200090F08000680060000000E00063003200E0
:10B33000E1EE8000B0EE800000805000A0EF8800B9
:10B34000A0EF800002282000110009000200D800B0
:10B350008000780030E880000088B9008000780024
:10B36000B0EE80008080400010EF800080804000C0
:10B3700000BA2F000080400090EF8800E0EE8000CF
:10B38000B1EE8000801F7800811F7800B04B2A004A
:10B39000801F78006041210043E20700E6875700E4
:10B3A0006041210005F20700109EA80080EF800098
:10B3B0007400400080EF880080EF80000000E00013
:10B3C00004003D00D0C2B300D0F00700D0C2B300EB
:10B3D0000DF1070080EF8000000F78001E00E000F4
:10B3E00001003D001E0FEA001E00780044F1070036
:10B3F0001E00780072F1070090C0B300C3F0070090
:10B40000C0C2B30000F1070090EF80000000E00030
:10B4100004003D00D0C2B300BCF00700D0C2B300AE
:10B42000F9F0070090EF8000000F78001E00E000A8
:10B4300001003D001E0FEA001E00780030F10700F9
:10B440001E0078005EF1070090C0B300AFF0070067
:10B45000C0C2B300ECF00700A0EF80000000E000E5
:10B4600004003D00D0C2B300A8F00700D0C2B30072
:10B47000E5F00700A0EF8000000F78001E00E0005C
:10B4800001003D001E0FEA001E0078001CF10700BD
:10B490001E0078004AF10700F04C2A008CF10700EA
:10B4A000F04C2A00C5F10700109EA90012DEA8008A
:10B4B0000000EB00B5F9070001003700127EA8007C
:10B4C000129EA90012BEA90058E780006140B90091
:10B4D000D8DC0700200F9800310F98000800E0002A
:10B4E00007003D0002002000037824002E08900091
:10B4F000BE08900088DA0700200F9800310F9800EE
:10B5000002002000031A24002E089000BE089000BC
:10B5100080DA0700A9DC070040E788004006200029
:10B520002C1607002615070040E78000801F7800D2
:10B53000204D2A00801F780060412100DAE10700D9
:10B54000E4875700604121009CF10700125EA800CB
:10B55000DA00370001C3B3000000EB006AE907001E
:10B560006000B80090F08800A1F088000FDEA8000D
:10B5700013FEA800121EA80090EF8000CF80DE000E
:10B58000ACDC070002002000F346240062DA07006A
:10B5900002002000832C240099DD07000200200017
:10B5A000832C240087DB070084DC070040E7880049
:10B5B00060EF8000CF80DE009EDC07000001BE004F
:10B5C00000002800A14B240052DA070002002000EE
:10B5D000833424004FDA07000004BE0080EF8000AF
:10B5E000CF80DE0093DC07000001BE000800BE0033
:10B5F00049DA070002002000832C240080DD0700C8
:10B6000002002000832C24006EDB07006BDC0700A7
:10B6100090E7880040E7800091E78000801F780075
:10B62000811F7800E04D2A00801F780060412100D2
:10B630009DE10700E6875700604121005FF10700A8
:10B6400060012000E3150700DD1407001000200052
:10B6500037F9070099003700121EA900123EA80012
:10B6600098E780006140B90072DC0700000F980085
:10B67000110F98000800E00007003D0002002000C4
:10B68000037824000E0890009E08900022DA07003C
:10B69000000F9800110F980002002000833C240046
:10B6A0000E0890009E0890001BDA070043DC07009C
:10B6B00090E7880090E78000801F7800E04E2A0025
:10B6C000801F78006041210077E10700E487570080
:10B6D0006041210039F1070040062000BD15070038
:10B6E000B714070075003700A0E78000801F7800BE
:10B6F000B04F2A00801F7800604121006AE10700F6
:10B70000E4875700604121002CF1070001C3B3001A
:10B710000000EB00FCE80700109EA800A8E78000EE
:10B720006140B90043DC070060079800710798008A
:10B730000800E00007003D0002002000037824001C
:10B740006E009000FE009000F3D90700600798009B
:10B750007107980002002000832C24006E009000E6
:10B76000FE00900026DD070002002000832C24004C
:10B7700014DB0700CADB0700C0ED8800C1ED8000C4
:10B7800060EF800080804000C0A22F000080400059
:10B79000A0EF8800405D2000C0ED8800A0EF800091
:10B7A00074004000A0EF8800A0EF80000000E000DF
:10B7B00004003D00D0C2B300D4EF0700D0C2B300F4
:10B7C00011F00700A0EF8000000F78001E00E000DD
:10B7D00001003D001E0FEA001E00780048F007003F
:10B7E0001E00780076F00700F04C2A00B8F0070041
:10B7F000F04C2A00F1F00700109EA900A8E7800095
:10B800006140B9000BDC0700400798005107980021
:10B810000800E00007003D0002002000037824003B
:10B820004E009000DE009000BBD907004007980052
:10B830005107980002002000832C24004E00900045
:10B84000DE009000B3D90700DCDB070090E788003A
:10B8500058E780006140B900F6DB07002007980038
:10B86000310798000800E00007003D0002002000BA
:10B87000037824002E009000BE009000A6D9070097
:10B88000200798003107980002002000832C240034
:10B890002E009000BE0090009ED90700C7DB070075
:10B8A00040E78800123EA900125EA80012DEA80040
:10B8B0006001200047150700411407004F04BE0037
:10B8C0000080FA00000006000E00FA004007980011
:10B8D000510798000000EB00000F7800A0502A00EC
:10B8E000B6F007004E0090006600B90080007800B6
:10B8F00060DD210000804000100178004E009000C3
:10B900006600B9008080E80060DD21000080400012
:10B91000900078005E00900000804000800F510091
:10B9200014003E004E0090006600B90080007800D0
:10B9300060DD210000804000100178004E00900082
:10B940006600B9008080E80060DD210000804000D2
:10B95000900078005E00900000805000800F510041
:10B96000040039001E0FE8008E80E800100020005F
:10B97000800878004E0090006600B90080007800D2
:10B9800060DD210000804000100178004E00900032
:10B990006600B900E400400060DD21000080400046
:10B9A000900078005E00900000804000800F510001
:10B9B00014003E004E0090006600B9008000780040
:10B9C00060DD210000804000100178004E009000F2
:10B9D0006600B900E400400060DD21000080400006
:10B9E000900078005E00900000805000800F5100B1
:10B9F000040039001E0FE8008E80E80010002000CF
:10BA0000A00098004E0090006600B9008080E80019
:10BA100060DD210000804000100178004E009000A1
:10BA20006600B900E400400060DD210000804000B5
:10BA3000900078005E00900000804000800F510070
:10BA400014003E004E0090006600B9008080E800BF
:10BA500060DD210000804000100178004E00900061
:10BA60006600B900E400400060DD21000080400075
:10BA7000900078005E00900000805000800F510020
:10BA8000040039001E0FE8008E80E800100020003E
:10BA9000B0009800100020009E0F1000200034001D
:10BAA000CE0190004E0090006600B9008000780042
:10BAB00060DD210000804000100178004E00900001
:10BAC0006600B9008080E80060DD21000080400051
:10BAD00010007800000141004E0090006600B9009F
:10BAE000E400400060DD210000804000100078008C
:10BAF0000000410032002000110009000280D8003F
:10BB0000000178006618B9008000780060DD21002F
:10BB10000080400002087800135EA9004D00370045
:10BB20001E00E000480032000E80E800100078009F
:10BB30000000E00015003200CE0190004E009000A1
:10BB40006600B9008000780060DD210000804000C0
:10BB5000100178004E0090006600B9008080E80077
:10BB600060DD2100008040001000780000004100EE
:10BB70000001D1006618B9008000780060DD210066
:10BB800000804000020878002D0037000E80E80099
:10BB9000100090000000E00015003200CE0190007F
:10BBA0004E0090006600B9008000780060DD210042
:10BBB00000804000100178004E0090006600B9003F
:10BBC000E400400060DD21000080400010007800AB
:10BBD000000041000001D1006618B9008000780023
:10BBE00060DD21000080400002087800140037006A
:10BBF000CE0190004E0090006600B9008080E80001
:10BC000060DD210000804000100178004E009000AF
:10BC10006600B900E400400060DD210000804000C3
:10BC200010007800000041000001D1006618B90042
:10BC30008000780060DD210000804000020878006C
:10BC4000135EA900030037000000EB0060079800B6
:10BC50000400370070512A00D8EF070010002000C0
:10BC6000600798006E0090000080FA000000060057
:10BC70000200FA00B6DDBF000080FB00000F780074
:10BC80001E007800E40F5000410032001E007800D2
:10BC9000E40F50000A003C001E007800E20F500044
:10BCA0002D0032001E007800E20F500023003C00FF
:10BCB0001E007800E10F50001C0032004E003700DB
:10BCC0001E007800E80F5000450032001E0078008A
:10BCD000E80F500004003C001E007800E60F500002
:10BCE00021003200440037001E007800E90F5000A8
:10BCF000040032001E007800EC0F50002B003200D0
:10BD00003D00370040E780000000E80040E7880081
:10BD1000A0E78000EA0F50003700360090E780006F
:10BD20000000E90090E788003300370040E780001A
:10BD30000000E80040E788002F00370040E780005F
:10BD40000000E80040E7880090E780000000E8007D
:10BD500090E788002800370090E780000000E800A6
:10BD600090E788002400370050E78000EA0F500079
:10BD70000300360040E780000000E90040E788004B
:10BD800090E780000000E80090E788001A00370084
:10BD900050E78000EA0F50001700360040E78000AF
:10BDA0000000E90040E788001300370050E78000FA
:10BDB000EA0F50000300360040E780000000E90071
:10BDC00040E78800A0E78000EA0F50000A00360034
:10BDD00090E780000000E90090E788000600370047
:10BDE000A0E78000EA0F50000300360090E78000D3
:10BDF0000000E90090E788000080FA0000000600DB
:10BE00001E00FA00881F78002047980070F080001C
:10BE100001402000010060000000E00072013A00D3
:10BE20002E4090000000FB00600F9800E00620000C
:10BE3000EE089000808F50001E003200E0062000C7
:10BE4000EE089000808F50000D003C00200620007E
:10BE5000EE089000808F50005B0132004006200009
:10BE6000EE089000808F50009700320030052000CF
:10BE7000EE089000808F50004A0132005A013700CE
:10BE800030072000EE089000808F50004C003200F8
:10BE900080072000EE089000808F500016003200CE
:10BEA00020072000EE089000808F50002100320013
:10BEB0004D0137000EFEA90070F080000110200037
:10BEC000010060000000E000020032000F9EA800A8
:10BED000010037000F9EA9000F1EA9000F3EA90008
:10BEE0000F5EA9000F7EA9006000B80090F08800E6
:10BEF000A1F088003C01370040E78000630040006B
:10BF000040E78800E0012000B2130700AC120700F0
:10BF1000C0512A0029EF070090E78000A8EE070033
:10BF2000C0C2B30038EE070040E78000A4EE07006F
:10BF30002D01370070F08000010820000100600032
:10BF40000000E0001A003A00E0C6B300ACFF0700B2
:10BF50000000EB00B0EE88000000EB00C0EE8800AF
:10BF60000000EB00E0EE88000000EB00F0EE88003F
:10BF70000EFEA80010002000EDF6070010002000C3
:10BF8000E50F07001000200012F90700B0522A0048
:10BF90000AEF070090E7800089EE0700C0C2B300F7
:10BFA00019EE070040E7800085EE07000200370029
:10BFB00080C7B30092FF07000F5EA8000A01370098
:10BFC00070F080004B00DE00614060008080FB006C
:10BFD00070F080004900DE00614060000080FB00DE
:10BFE000811F7800801F7800B0532A00801F7800DE
:10BFF000604121002CDF0700E687570060412100E7
:10C00000EEEE070071F0800000202000008060004C
:10C010000000E00019003A0070F08000018020006C
:10C02000010060000000E0000B003A00A0E7800083
:10C03000C0EE880050E7800063005000B0EE88003A
:10C0400041E7800050FB2F000080400040E788005F
:10C050000F7EA800050037000F7EA90020F08000A9
:10C0600067005000AC0F07000F3EA80060012000E1
:10C0700058130700521207000200370080C7B300B0
:10C080005FFF07000F5EA80050E7800041E78000D7
:10C09000A2E7800093E78000801F7800811F78006E
:10C0A000821F7800831F780070562A00801F780056
:10C0B00060412100FCDE0700EA8757006041210053
:10C0C000BEEE0700C800370070F0800001002200BB
:10C0D000010060000000E0005E003A00A0E7800080
:10C0E000F0EE880050E7800063005000E0EE88002A
:10C0F000C1EE8000F0EE8000808F500051003200D1
:10C10000E8EE80006140B900CAD90700400F9800EE
:10C11000510F98000800E00007003D0002002000D9
:10C12000037824004E089000DE0890007AD70700BC
:10C13000400F9800510F9800B8EE80006140B900A0
:10C14000BCD90700200F9800310F98000800E000CC
:10C1500007003D0002002000037824002E08900014
:10C16000BE0890006CD70700200F9800310F980090
:10C170002E099000BE0990004E089000DE08900045
:10C1800064D70700000F9800110F9800F8EE8000A8
:10C190006140B900A7D907006007980071079800AF
:10C1A0000800E00007003D000200200003782400A2
:10C1B0006E009000FE00900057D7070060079800BF
:10C1C00071079800C8EE80006140B90099D9070056
:10C1D00040079800510798000800E00007003D0064
:10C1E00002002000037824004E009000DE00900042
:10C1F00049D7070040079800510798004E0190006A
:10C20000DE0190006E009000FE00900041D7070014
:10C210000001BE000E0890009E08900069D807003B
:10C22000B0E98800C1E98800B0E98000C1E9800078
:10C2300001F0A10095D70700D0E98800E1E9880066
:10C240004D0037006000B800B0E98800C1E98800FF
:10C2500049003700A05B2A0058EE0700B0EE8000CE
:10C26000D7ED0700A05C2A0054EE0700D1ED800056
:10C2700010EF80008080500090EF80000080400030
:10C28000CFED070061DF21009140780020C4B300AA
:10C2900080CF50000A003200D1ED800010EF800006
:10C2A0008080500090EF8000008040008000780087
:10C2B000B0EE800000805000000F780009003700C9
:10C2C000D1ED800010EF80008080500090EF800062
:10C2D0000080400080007800B0EE800000805000B8
:10C2E000000F78008040EB000000EB0006E607003E
:10C2F000109EA800F04C2A0030EE07001E00E0005F
:10C3000004003400D0C2B30000ED0700D0C2B30077
:10C310003DED07001E00780030079800BE00900039
:10C320000100E00003003D003E0090000000EA0034
:10C33000300798003E00900071ED0700F04C2A0095
:10C34000E3ED07009E007800210798002E00900082
:10C350000000E00003003D00AE0090008100EA0014
:10C36000210798002E00900095ED0700F04C2A0060
:10C3700012EE0700109EA9000F1EA8000EFEA900D5
:10C380000F3EA90040E7800051FB2F000100400054
:10C3900040E788000F7EA800E00120008D12070012
:10C3A0001100370050E7800063005000B0EE8800B5
:10C3B000A0E78000C0EE88000FBEA80040C6B30012
:10C3C0008FFE07000800370070F080000100210098
:10C3D000010060000000E000010032000F1EA80014
:10C3E0000000EB0030F088004F0478000080FA0075
:10C3F000000006000600FA00881F78000000EB002D
:10C40000000F780030F08000801F7800D05D2A0097
:10C41000801F78006041210023DE0700E487570079
:10C4200060412100E5ED070080F0800061006000C0
:10C430000000E0005A003A0001C3B3000000EB0026
:10C44000B1E507006000B80090F08800A1F0880016
:10C4500010DEA900101EA800121EA800123EA8009F
:10C46000129EA90012BEA90030F0800030F08800B2
:10C470000000EB0050F0880030F08000A60E0700AE
:10C480000000EB001A110700000F7800D1ED8000CA
:10C4900010EF80008080500090EF8000008040000E
:10C4A0009E00400050FB2F0000804000CF80DE0047
:10C4B000E0D8070002002000832C2400D0D9070018
:10C4C00002002000832C2400BED70700BBD8070041
:10C4D00040E7880090F08000640060000000E00009
:10C4E0001900320090F08000680060000000E00059
:10C4F00015003A0098E780006140B900CDD80700E8
:10C5000010079800210798000800E00007003D0090
:10C5100002002000037824001E009000AE0090006E
:10C520007DD6070010079800210798000200200020
:10C53000031F24001E009000AE00900076D6070076
:10C540009ED8070090E788006001200021120700B4
:10C550001B1107001000200075F5070040E7800060
:10C5600091E78000801F7800811F7800C05E2A005C
:10C57000801F780060412100CBDD0700E68757006F
:10C58000604121008DED070000642000E008880074
:10C590000000EB00C008880021E1A800000237007D
:10C5A00090F0800001022000010060000000E00027
:10C5B0001401320050E78000A1E78000801F78005E
:10C5C000811F7800A05F2A00801F78006041210051
:10C5D000B5DD0700E68757006041210077ED0700D1
:10C5E00041E7800050E78000808F50001F003A0034
:10C5F0000000EB0040F088000D003700703E200086
:10C60000EFEC0700D0C0B3007FEC0700A0C0B30080
:10C610007DEC0700703E2000B9EC070090C0B3002D
:10C620003AEC070040F080000000E80040F088008D
:10C6300040F080008000780050EE8000808F500035
:10C64000EEFF3900101EA800131EA800129EA900BC
:10C650000000EB0020F088000000EB0030F08800C4
:10C6600050C6B30029EC0700CD01370090F08000E0
:10C67000640060000000E0000700320090F08000DD
:10C68000680060000000E00003003A0050F0800005
:10C6900010E88800980037000000EB0094100700B5
:10C6A000000F780090F08000680060000000E0005B
:10C6B0001F00320090F08000014020000100600067
:10C6C0000000E00007003A0012EF800051F0800007
:10C6D00010E88000008050000000510080E98800D0
:10C6E0004C00370090F080000180200001006000C5
:10C6F0000000E00007003A0012EF800051F08000D7
:10C7000010E88000008050000000510090E988008F
:10C710004000370012EF800051F0800010E88000E8
:10C720000080500000005100A0E988003900370067
:10C7300090F0800001402000010060000000E00057
:10C740000D003A0010EF80000001780053E78000F0
:10C75000D1ED800010EF80008080500090EF8000CD
:10C76000008040001E004000008051000000510089
:10C7700080E988001E00370090F0800001802000D2
:10C78000010060000000E0000D003A0010EF8000A2
:10C790000001780053E78000D1ED800010EF8000A9
:10C7A0008080500090EF8000008040001E0040001C
:10C7B000008051000000510090E988000C00370013
:10C7C00010EF80000001780053E78000D1ED800079
:10C7D00010EF80008080500090EF800000804000CB
:10C7E0001E0040000080510000005100A0E98800B8
:10C7F0001E007800801F780090602A00801F78005B
:10C800006041210028DD0700E487570060412100D6
:10C81000EAEC070090F08000018020000100600039
:10C820000000E00022003200A0E9800091E98000D1
:10C8300082E98000801F7800811F7800821F7800C5
:10C84000A0612A00801F78006041210016DD0700EA
:10C85000E887570060412100D8EC070030F08000E5
:10C8600032002000110009000200D8008001780089
:10C8700081E9800090E9800080804000A0E980008C
:10C880000080400032002000110009000200D800A2
:10C89000000178006618B900E4004000E0D32100F0
:10C8A0000080400002087800135EA90012003700E3
:10C8B00090F0800001402000010060000000E000D6
:10C8C00007003A0090F08000012020000100600085
:10C8D0000000E00002003200135EA80006003700EE
:10C8E00090F0800001202000010060000000E000C6
:10C8F00001003200137EA8000000EB00FC0F0700CF
:10C90000000F780091F0800000402000008060005F
:10C910000000E0001D003A0090F08000018020003F
:10C92000010060000000E0001800320090F080007C
:10C9300001202000010060000000E0001300320030
:10C94000D1ED800010EF80008080500090EF8000DB
:10C95000008040009E00400050FB2F0000804000FF
:10C96000CF80DE00B3D7070002002000832C240014
:10C97000A3D8070002002000832C240091D60700D2
:10C980008ED7070040E788000D00370090F0800048
:10C9900001202000010060000000E00004003200DF
:10C9A00050E780007400500040E788000400370022
:10C9B00050E7800081FD2F000100400040E7880023
:10C9C000E001200003110700FD0F070040E7800091
:10C9D00091E7800052F08000801F7800811F78006E
:10C9E000821F7800D0622A00801F780060412100F9
:10C9F000ADDC0700E8875700604121006FEC0700BD
:10CA0000E700370090F08000700060000000E00058
:10CA1000B600320030F08000320020001100090022
:10CA20000200D8008000780050EE80000000E9008D
:10CA3000808F50004200390090F0800001402000BB
:10CA4000010060000000E0003D003A0090F080002E
:10CA500001802000010060000000E000380032008A
:10CA6000101EA800129EA9000000EB0020F0880014
:10CA70000000EB0030F08800E0E78000D0E788009D
:10CA800001C3B3000000EB001FE40700109EA800E4
:10CA90000000EB0040F088001700370040F08000F5
:10CAA0006600B900E4004000E0D3210000804000AF
:10CAB00010007800C2EB0700D0C0B30052EB0700B3
:10CAC000A0C0B30050EB070040F080006600B90042
:10CAD000E4004000E0D32100008040001000780016
:10CAE00087EB070090C0B30008EB070040F0800020
:10CAF0000000E80040F0880040F0800080007800EE
:10CB000050EE8000808F5000E4FF390050C6B30023
:10CB1000FEEA070050C6B3003BEB0700109EA900D9
:10CB2000101EA800131EA800129EA9000000EB0012
:10CB300020F088000000EB0030F0880098003700FB
:10CB400090F08000640060000000E0000600320009
:10CB500090F08000680060000000E00002003A00F1
:10CB6000127EA8001B00370090F08000610060007A
:10CB70000000E00010003A0090F08000012020004A
:10CB8000010060000000E0000B00320090F0800027
:10CB900001402000010060000000E0000D003A00AC
:10CBA00030F080006300400030F08800137EA90060
:10CBB000133EA9000700370090F08000610060007C
:10CBC0000000E00002003200121EA9000100370040
:10CBD000133EA800123EA90030F08000CE0C0700E2
:10CBE00091F0800000402000008060000000E00024
:10CBF00009003A0090F08000012020000100600050
:10CC00000000E0000400320090E780006500400072
:10CC100090E788000800370090F080000180200035
:10CC2000010060000000E0000300320090E7800097
:10CC30006500500090E788000000EB002C0F070013
:10CC4000000F780050E7800040E7880091F08000F6
:10CC500000202000008060000000E00012003A0088
:10CC6000D1ED800010EF80008080500090EF8000B8
:10CC7000008040009E00400050FB2F0000804000DC
:10CC8000CF80DE00EBD6070002002000832C2400BA
:10CC9000DBD7070002002000832C2400C9D5070041
:10CCA000C6D6070040E78800EC3CA800E23CA9009B
:10CCB0006001200047100700410F070040E7800097
:10CCC00091E78000801F7800811F7800C0642A00EF
:10CCD000801F780060412100F3DB0700E6875700E2
:10CCE00060412100B5EB07002D0037000000EB008C
:10CCF00050F088000000EB00FD0E0700000F7800E8
:10CD0000D1ED800090EF8000008040009E00400048
:10CD1000B0F52F0000804000CF80DE00C5D60700B0
:10CD200002002000832C2400B5D707000200200059
:10CD3000832C2400A3D50700A0D6070040E7880075
:10CD4000EC3CA800E23CA90091F08000002020000B
:10CD5000008060000000E00003003200800C200032
:10CD60001C10070002003700E00120001910070026
:10CD7000130F070040E7800091E78000801F7800D4
:10CD8000811F7800F0652A00801F78006041210033
:10CD9000C5DB0700E68757006041210087EB0700ED
:10CDA0004F0478000080FA00000006000200FA003C
:10CDB000004F780030C7B3009E4F10000A003A00C1
:10CDC0001000200071F3070010FEA80000E8230007
:10CDD000D00888000000EB00A00888001FE1A80030
:10CDE000CA1607000600370060C6B3009E4F100049
:10CDF00003003A000000EB0064F3070010FEA900F6
:10CE00000080FA00000006000000FA0080F08000B8
:10CE10006C0060000000E0001C003A0010002000E0
:10CE200043F307000001EB00F10F2000F00F20009A
:10CE30006B120700803E200040E78800E00E0700EC
:10CE400080F080004200DE00634060000040E800A7
:10CE5000634060000080FB00630060004201DD0071
:10CE600081F0800030FF2F00008060000200700021
:10CE700080F0880000642000E00888000000EB00DB
:10CE8000C008880021E1A8002400370080F080005D
:10CE90006C006000E40F500017003A000001EB0046
:10CEA0008000EB00F00F20004D1207001000200062
:10CEB00036F30700803E200090E78800C00E070090
:10CEC00080F080004200DE00634060000040E80027
:10CED000634060000080FB00630060004201DD00F1
:10CEE00081F0800030FF2F000080600002007000A1
:10CEF00080F08800090037000001EB00F10F2000EE
:10CF0000F00F2000361207002BF40700105EA90076
:10CF1000107EA9000000EB0005F307000080FA0076
:10CF2000000006003400F800881F78001800200078
:10CF3000A80188004F0478000000FA008440A9008E
:10CF4000C442A900C462A900C4C2A900C4E2A900E5
:10CF50000080FA003400F900004006003400F800B8
:10CF6000881F780018002000A80188004F0478006E
:10CF70000000FA0084C0A900C402A900C422A900CC
:10CF8000C482A900C4A2A9000080FA003400F900FC
:10CF9000004006003400F800881F780018002000C8
:10CFA000A80188004F0478000000FA008720A9003B
:10CFB000C522A900C542A900C5C2A900C5E2A900B1
:10CFC0000080FA003400F90000400600809FBE0097
:10CFD000821F78003400F80010002000A0018800B3
:10CFE0000000FA008500A9000000EB00500888004E
:10CFF00013E1A80000E7800021DC210000004000D0
:10D000000100400010007800614060006140600055
:10D010004201DD00412C200091407800B0CFB300E8
:10D0200000C0600002407000C4E2B70000E780006A
:10D0300021DC2100000040000100400010007800C9
:10D040000000D10061406000614060004301DD00EC
:10D05000412C20009140780070CFB30000C06000E8
:10D0600002407000C4E2B70000E7800021DC21002C
:10D070000000400001004000100078004200DE0087
:10D0800061406000614060004601DD00412C2000ED
:10D0900091407800F0CBB30000C060000240700007
:10D0A000C4E2B70000E7800021DC2100000040005E
:10D0B00001004000100078004300DE006140600085
:10D0C000C700DD00C4C2BF000074A10001407000B1
:10D0D000C4E2B700F0E6800021DC2100000040003F
:10D0E0000100400010007800614060006141600074
:10D0F000412C200091407800E0CFB30000C06000D8
:10D1000002407000C4E2B700F0E6800021DC21009C
:10D110000000400001004000100078000000D10035
:10D12000614060006140600000414000412C2000EF
:10D1300091407800D0CFB30000C060000240700082
:10D14000C4E2B700F0E6800021DC210000004000CE
:10D1500001004000100078004200DE0061406000E5
:10D16000614060004401DD00412C200091407800C6
:10D17000F0CEB30000C0600002407000C4E2B7000F
:10D18000F0E6800021DC21000000400001004000AA
:10D19000100078004300DE006140600061406000E4
:10D1A0004501DD00412C200091407800F0CDB30016
:10D1B00000C0600002407000C4E2B70091E7800048
:10D1C000A0E78000808F500006003A0060E78000F2
:10D1D000620060000000E000020032000019200040
:10D1E000B00C880041E7800050E78000808F50003D
:10D1F00006003A0010E78000620060000000E000D6
:10D200000200320000192000000D88000080FA00A2
:10D210003400F9004F0178004F00BE0000400600C6
:10D22000809FBE00829FBE003400F80010002000E6
:10D23000A00188000200FA008780A90021E1A9006E
:10D2400010002000C0E788000000EB00000F78000D
:10D250001B0037001E0078006A00B900E80040009B
:10D2600020CE210000804000100178001E007800D0
:10D270006A00B900E600400020CE21000080400096
:10D2800010007800800F51000C0032001E01780061
:10D290006A10B900E400400020CE21000080400068
:10D2A000100078008001E8006A10B900E400400036
:10D2B00020CE210000804000030878001E0FE80007
:10D2C000100020009E0F1000E2FF34000080FA00E2
:10D2D0003400F9004F01BE004F00BE0000400600C0
:10D2E0000A00FA000000EB00000F7800C0E78000A1
:10D2F0000000E0002001320070F080006200600059
:10D300000000E00020003A0070F08000680060003B
:10D310000000E0001C003A0070F080000140200096
:10D32000010060000000E00017003A0070F080008B
:10D3300001002400010060000000E00012003A003B
:10D3400070F0800001002800010060000000E00093
:10D350000D003A0080F08000610060000000E000F5
:10D3600009003A0080F080006C0060000000E000DE
:10D3700005003A0080F080000104200001006000F8
:10D380000000E000FC00320070F0800064006000EB
:10D390000000E000F8003A000000EB0010079800E1
:10D3A0005A0037001E0090006A00B900E6004000F5
:10D3B00020CE210000804000100078004007980037
:10D3C0004E0090000000E00003003D00CE00900001
:10D3D0008100EA004107980080BB2000CE00900049
:10D3E000808F50000D003400F0662A00F3E907003A
:10D3F00090E7800072E90700C0C2B30002E90700AD
:10D4000040E780006EE90700D0682A00600207004C
:10D4100080C3B300BDE80700440237001E0090003F
:10D420006A00B900E400400020CE210000804000E6
:10D43000100178001E0090006A00B9008080E800AA
:10D4400020CE21000080400010007800800F5100A5
:10D450002B0039001E0090006A00B900E600400071
:10D4600020CE210000804000100178001E009000B6
:10D470006A00B900E800400020CE21000080400092
:10D4800010007800800F51001D0032001E00900037
:10D49000D4F107001E0090006A00B900E4004000CB
:10D4A00020CE2100808040000000EB008008780042
:10D4B0009E009000018040006601400040E0210095
:10D4C00000004100100078000001E80001804000E9
:10D4D000E600400040E021000080400002087800A3
:10D4E000E0ED80000000D100614060008080FB0022
:10D4F0001E009000808F500001003A00BC5DA80023
:10D500001E0090000000E800100798001E00900028
:10D51000E10F5000A3FF3400E0ED800061006000E7
:10D520000000E0008E003200E0ED8000640060004A
:10D530000000E0008A003200F0ED8000E40F5000AF
:10D5400004003C00F0ED80000000E800F0ED8800F1
:10D5500082003700E0ED80000000D10061406000F3
:10D560000080FB006A00B900E600400020CE2100E8
:10D570000080400010017800E0ED80000000D10044
:10D58000614060000080FB006A00B900E8004000D4
:10D5900020CE2100008040001000780000005100E3
:10D5A000300798003E0090000000E00003003D00BE
:10D5B000BE0090008100EA00310798003E01900013
:10D5C000E0ED80000000D100614060000080FB00C1
:10D5D0006A00B9008080E80020CE21000080400071
:10D5E00010007800790010006500B900800F51002C
:10D5F00041003600E0ED80000000D1006140600095
:10D600000080FB006A00B9008080E80020CE210085
:10D61000008040009000780000EE8000808F500075
:10D620004C003600E0ED80000000D1006140600059
:10D630000080FB006A00B900E600400020CE210017
:10D640000080400010017800E0ED80000000D10073
:10D65000614060000080FB006A00B900E800400003
:10D6600020CE210000804000100078000000510012
:10D67000200798002E0090000000E00003003D000D
:10D68000AE0090008100EA00210798002E01900072
:10D69000E0ED80000000D100614060000080FB00F0
:10D6A0006A00B9008080E80020CE210000804000A0
:10D6B000100078007A0010006500B900800F51005A
:10D6C00024003600E0ED80000000D10061406000E1
:10D6D0000080FB006A00B9008080E80020CE2100B5
:10D6E00000804000100078000000E900B90D07003C
:10D6F000B30C070017003700E0ED80000000D100F8
:10D70000614060000080FB006A00B9008080E80092
:10D7100020CE21000080400010007800F80F50005B
:10D720000C003E00E0ED80000000D1006140600090
:10D730000080FB006A00B9008080E80020CE210054
:10D7400000804000100078000000E800A10D0700F4
:10D750009B0C07000000EB00F0ED8800BC5DA90009
:10D7600000642000E00888000000EB00C00888008A
:10D770000000EB00C0E788000000EB0010079800F5
:10D78000120037001E0090006A00B900E800400057
:10D7900020CE210000804000100178001E00900083
:10D7A0006A00B900E600400020CE21000080400061
:10D7B00010007800800F510001003A001E0FE800B1
:10D7C0001E0090000000E800100798001E00900066
:10D7D000E10F5000EBFF340021C1BF0001C8B300CE
:10D7E000014060000004E0001C003A0070F080007E
:10D7F000620060000000E00017003A0070F0800056
:10D8000001402000010060000000E00012003A002A
:10D8100070F0800001002400010060000000E000C2
:10D820000D003A0080F08000610060000000E00020
:10D8300009003A0080F080006C0060000000E00009
:10D8400005003A0080F08000010420000100600023
:10D850000000E0000100320021E1A80010002000DB
:10D860009E0F10003101340070F0800068006000ED
:10D870000000E0002D013A0080F0800061006000AF
:10D880000000E0003200320090F080000102200031
:10D89000010060000000E0000400320012BEA90098
:10D8A000129EA800D3FA07002001370090F08000F4
:10D8B000700060000000E00003003200129EA9002A
:10D8C000CCFA07001901370090F080006100600079
:10D8D0000000E0000700320090F080006800600067
:10D8E0000000E00003003A00129EA800C1FA070001
:10D8F0000E01370090F08000011020000100600050
:10D900000000E00005003A0090F0800001082000CF
:10D91000010060000000E0000A0032006000B80072
:10D9200090F08800A1F088000000EB0097F007005D
:10D93000A1F107000000EB007DF00700101EA90018
:10D940000300370012BEA800AAFA0700F70037004C
:10D9500070F0800001002400010060000000E00081
:10D960005900320090F080000104200001006000A6
:10D970000000E00054003A0090F080000100220016
:10D98000010060000000E0000700320090F080001D
:10D99000620060000000E0000300320030C0B3000D
:10D9A000B0F307005B00370090F080000100240016
:10D9B000010060000000E0000700320090F08000ED
:10D9C000620060000000E0000300320060C0B300AD
:10D9D000A4F307004F00370090F0800001002400FE
:10D9E000010060000000E0000700320090F08000BD
:10D9F000640060000000E0000300320050C0B3008B
:10DA000098F307004300370090F0800001002800E1
:10DA1000010060000000E0000700320090F080008C
:10DA2000640060000000E00003003200A0C0B3000A
:10DA30008CF307003700370090F0800001002800C9
:10DA4000010060000000E0000700320090F080005C
:10DA5000610060000000E0000300320090C0B300ED
:10DA600080F307002B00370090F0800001002100B8
:10DA7000010060000000E00004003A0090F0800027
:10DA8000610060000000E0000C0032006000B8009F
:10DA900090F08800A1F0880080C3B3001BE7070066
:10DAA0000000EB0039F0070043F107000000EB0035
:10DAB0001FF007000FDEA9001600370010C0B300EA
:10DAC00068F307001300370070F0800001002400A5
:10DAD000010060000000E0000E00320090F08000C5
:10DAE00001042000010060000000E0000900320095
:10DAF0006000B80090F08800A1F088000000EB0002
:10DB000022F007002CF107000000EB0008F00700EE
:10DB10000FDEA90080F080000104200001006000F9
:10DB20000000E0000500320010DEA9000000EB005C
:10DB300028F207000000EB00FDEF070070F0800006
:10DB400001402000010060000000E0000A003200F7
:10DB500070F0800001802000010060000000E00003
:10DB6000040032000F5EA90030C7B300A4F807001C
:10DB7000010037000F5EA90070F080000110200046
:10DB8000010060000000E0000B00320070F0800037
:10DB900001802000010060000000E000060032006B
:10DBA0000F7EA90030F08000DB0807000EDEA80021
:10DBB0000000EB00000F780080F080006C00600037
:10DBC0000000E0000200320000692A007000070037
:10DBD00070F08000640060000000E00053003A0034
:10DBE00070F08000680060000000E0004F003A0024
:10DBF00070F0800001802000010060000000E00063
:10DC00004A003A0080F08000610060000000E000FF
:10DC100046003A0070F08000620060000000E00002
:10DC20004200320050E7800080007800A0E78000CA
:10DC3000AE080700D0C0B300F3E60700A0C0B300F1
:10DC4000F1E60700D0C0B300EFE60700A0C0B300C4
:10DC5000EDE6070031F0800020F08000808F50005A
:10DC60000A003D00CCC2BF000042B2000004E00048
:10DC700002003A0010002000C4EF070030F08000DE
:10DC8000A508070030F088002800370031F0800038
:10DC900020F08000808F500012003A0070F0800069
:10DCA00001022000010060000000E00008003A00CE
:10DCB00040E780007E00500040E7880060012000BF
:10DCC000440C07003E0B07000EBEA80017003700EB
:10DCD00030F080000000E80030F088000EBEA9009F
:10DCE000120037000EDEA9000000EB00A7EF0700CE
:10DCF0000000EB0030F0880001C3B3000000EB002F
:10DD000081DF0700109EA80060C3B3007FE6070014
:10DD1000109EA90030692A00A8E70700A6F00700B6
:10DD20000000EB0082EF07000E3EA9000080FA0021
:10DD3000000006000000FA00501680004800DE00D7
:10DD4000610060000004E00003003200E21CA90052
:10DD5000DC02A80002003700E21CA800DC02A900D7
:10DD6000501680004900DE00610060000004E00001
:10DD700003003200EC1CA900DC22A80002003700DE
:10DD8000EC1CA800DC22A9000080FA0000000600BC
:10DD90001800FA00100798001E009000104078004C
:10DDA0000000FB006101B900F0FB2F00F1FF2F0024
:10DDB0000201400083814800220F9800330F980031
:10DDC00090032000010020002E099000BE09900061
:10DDD000800F5100818F5900BB023E002E08900039
:10DDE000BE089000006001008B0037009D003700E6
:10DDF0006E0037003A0237000A013700B2023700DE
:10DE0000B102370032003700AF023700740037002C
:10DE1000AD023700AC023700AB023700F00137002B
:10DE20007E02370077003700A7023700A6023700CE
:10DE3000440037002B003700A3023700A20237004E
:10DE40004D003700ED003700F10037009E0237002B
:10DE50009D0237009C0237009B0237009A02370070
:10DE600099023700980237000802370096023700FF
:10DE700084013700AA003700EF003700990037000F
:10DE800091023700900237008F0237008E02370070
:10DE90008D023700020237008B0237008A023700FA
:10DEA00089023700880237008702370012013700E5
:10DEB0007A0037000F0237008302370082023700F2
:10DEC00081023700800237007F023700E901370006
:10DED00080C4B3000DE60700006A2A0037E7070098
:10DEE0007C0237001E0090000000E800104078001F
:10DEF0008000FB0000FD2F0000804000D0E788007C
:10DF000080F08000620060000000E0000400320049
:10DF1000D0E78000E0E7880020002000D0E78800FC
:10DF2000D1E78000E00F2000808F500069023600AA
:10DF30000000EB00D0E7880031032000110F9800AB
:10DF400066023700110020001E009000A1020700A9
:10DF500050EE880051EE8000E00F2000808F5000CE
:10DF60005C0236000000EB0050EE88003203200017
:10DF7000120F980059023700110020001E00900077
:10DF80009402070090EE880091EE8000E00F2000E0
:10DF9000808F50004F0236000000EB0090EE8800AA
:10DFA00033032000130F98004C02370011002000AB
:10DFB0001E0090008702070070EE880071EE80005E
:10DFC000E00F2000808F5000420236000000EB007E
:10DFD00070EE880030032000100F98003F023700D9
:10DFE0001E0090000000E80010407800F6FDB70029
:10DFF0001E0090000000E80010407800F7FDB70018
:10E0000034023700110020001E009000710207004A
:10E01000A0EE88002F023700110020001E009000A3
:10E020006C02070080007800400B200001005000C7
:10E0300022002000110009000200D80080EE8800B4
:10E0400081EE8000E00F2000808F5000210236001A
:10E050000000EB0080EE880031032000110F9800D3
:10E060001E023700110020001E0090005902070018
:10E0700010EF880010EF800010E8880010EF80009B
:10E08000E10F400013023A000000EB0010EF88009F
:10E0900032032000120F98001002370040F0800079
:10E0A0008000780050EE8000808F500003003A001E
:10E0B00053032000130F98000802370011002000BE
:10E0C0001E00900043020700F0EF8800F0EF800090
:10E0D000E10F4000FF013A0030032000100F9800CC
:10E0E000FE013700110020001E00900039020700D9
:10E0F00000F0880000F080006600500000F088000A
:10E1000000F0800020E8880000F08000E10F40006F
:10E11000F0013A0031032000110F9800EF013700A1
:10E12000110020001E0090002A02070010F0880055
:10E1300080F08000620060000000E0001500320006
:10E1400040F08000F2EF80006600B90080007800A7
:10E15000E0D32100008040000208780040F08000F9
:10E1600002F080006600B9008080E800E0D3210062
:10E17000008040000208780040F0800012F080002B
:10E180006600B900E4004000E0D3210000804000B8
:10E190000208780010F08000E10F400003003A0010
:10E1A00032032000120F9800CC01370064004700B2
:10E1B00021F0800032F0800043F0800054F08000B5
:10E1C00065F080007402070064004700800078005A
:10E1D00040E021001101BE000288BE006400400042
:10E1E000E48040001101BE000288BE0064004000CF
:10E1F000E480400011087800B601370011002000CB
:10E200001E0090002702070080EF8800B101370050
:10E21000110020001E0090002202070090EF8800ED
:10E22000AC013700110020001E0090001D02070005
:10E23000A0EF8800A7013700306A2A005FE60700D8
:10E240001E0090000000E80090407800F0C6B30087
:10E2500080CF5000060032001E0090000080E800D1
:10E2600090407800F0C6B30080CF500003003A0021
:10E27000A06A2A0051E60700960137001E009000B0
:10E280000000E8009040780040C6B30080CF500006
:10E29000060032001E0090000080E80090407800E8
:10E2A00040C6B30080CF500005003A00206B2A0022
:10E2B00042E60700125EA800127EA9008501370021
:10E2C00080F08000620060000000E00004003A007E
:10E2D000103EA800F06B2A0038E607007D013700E9
:10E2E000406C2A0035E607000000EB0030F08800A3
:10E2F00040F8070077013700D0C0B30042E50700BF
:10E30000A0C0B30040E50700D0C0B3003EE5070061
:10E31000A0C0B3003CE5070001C3B3000000EB0060
:10E32000F9DD07001E0090000000E8009040780032
:10E33000D0C6B30080CF500009003A001E00900004
:10E340000080E8009040780000C3B30080CF500008
:10E3500002003A000E9EA900010037000E9EA800A0
:10E3600040F080008000780050EE8000808F5000E8
:10E3700041003A0070F080000000D1006140600070
:10E3800000C0EA00614060000080FB0061006000A6
:10E390000001400071F08000D0FF2F00008060007D
:10E3A0000200700070F0880081F0800000042000FE
:10E3B000008060000000E0000100320010DEA900D3
:10E3C00010002000DAED070030F080000000E000CF
:10E3D00040013A0070F08000620060000000E00040
:10E3E0003C01320070F08000010420000100600058
:10E3F0000000E00037013A0070F0800001082000C2
:10E40000010060000000E0000800320070F08000B1
:10E4100001202000010060000000E0000300320045
:10E4200040C6B30076F607002A01370070F080007E
:10E4300001082000010060000000E000030032003D
:10E4400030C5B3006EF607002201370070F080007F
:10E4500001802000010060000000E00002003A009E
:10E4600030F08000AC06070010002000D9EF070054
:10E470000EDEA8001701370073032000130F980069
:10E48000160137000000EB00C0ED07000000EB00B4
:10E4900090E788000000EB0040E788000000EB00F8
:10E4A00060F088000000EB0050F0880071F0800000
:10E4B00000082000008060000000E0000200320040
:10E4C000E0C6B3004EF6070070F080006200600006
:10E4D0000000E00023003A0070F0800001082000F6
:10E4E000010060000000E0001E003A0080F08000A3
:10E4F000610060000000E0001A003A0090F0800027
:10E50000610060000000E00016003A0080F080002A
:10E51000620060000000E00012003A0090F080000D
:10E5200001022000010060000000E0000D003A0040
:10E5300090F08000700060000000E00009003A00E8
:10E5400090F08000640060000000E00005003A00E8
:10E5500080F0800001042000010060000000E00065
:10E560000F0032006000B80070F0880081F0880071
:10E570000E1EA8000000EB00000F7800040037001A
:10E58000803E20000100200024DD07001E0FE8006F
:10E59000F07C20009E0F1000F9FF340086EE07008B
:10E5A0006000B80070F0880081F088006000B8005A
:10E5B00090F08800A1F088000E1EA8000000EB007B
:10E5C00020F088000000EB0030F088000000EB0035
:10E5D00040F088000000EB0055ED0700BD0037005B
:10E5E0000000EB0050EE88000000EB0060EE8800B9
:10E5F0000000EB0020F088000000EB0030F0880005
:10E600000000EB0040F088000000EB00A0EE880066
:10E61000103EA900101EA900125EA900127EA900DA
:10E620006000B80090F08800A1F088001000200081
:10E630003FED0700E0C6B300F1F507005EEE07000E
:10E640000000EB003AED07001E0090000000E8001B
:10E6500090407800D0C6B30080CF50009D003A00B3
:10E660001000200032ED0700306D2A00C6EF0700D1
:10E6700098003700100020002DED07004EEE070037
:10E680000000EB002AED0700920037001E0090000A
:10E690000000E80010407800D9F507008D00370031
:10E6A0001E0090000000E80090407800A0C6B30073
:10E6B00080CF500007003A00210020001E0090008B
:10E6C000C400070060EF880080C0B30065F0070059
:10E6D000800037000040EB0062F007007D0037004B
:10E6E0001E0090000000E80010407800AFF907001D
:10E6F000780037001E0090000000E800104078000D
:10E700000000FB00000F9800000720008E0890001A
:10E71000808F500020003200000720000E0990007A
:10E72000800F510005003C00D00420008E099000AD
:10E73000808F51000C003200660037002007200057
:10E740008E089000808F50000D00320030072000AE
:10E750000E099000800F5100010032005D0037006B
:10E76000A9F907005B003700C06D2A00D8E4070054
:10E770001E0090000080E80083EF0700550037007E
:10E78000306E2A00D2E4070010002000E8EC0700F9
:10E790000E9EA8004F00370001C3B3000000EB003D
:10E7A000D9DC0700109EA8000000EB0030F08800C4
:10E7B0000E00370030F080004B00070031F0800081
:10E7C00020F080000000E900808F500004003D0030
:10E7D00090C0B300CDE3070090C0B3000AE4070087
:10E7E00030F080000000E80030F0880031F0800058
:10E7F00020F08000808F5000EEFF3500F04C2A00A2
:10E80000B3E40700F04C2A00ECE40700109EA900D6
:10E810000000EB0030F088002E0037001E00900052
:10E820000000E800104078000000FB00700798002E
:10E8300030062000FE019000808F51001A00320047
:10E8400030072000FE009000808F5000050032004D
:10E85000700420007E019000800F51000A003200F9
:10E860001600370010BEA80001C3B3000000EB0083
:10E87000A5DC0700A06E2A000FE60700300020008C
:10E8800060F688000D00370001C3B3000000EB0004
:10E890009DDC0700106F2A0007E6070050002000EB
:10E8A00060F688000500370010BEA900106F2A002E
:10E8B00001E607000000EB0060F68800130320006B
:10E8C000130F98000500370020032000100F980058
:10E8D0000200370011032000110F98001E0890005D
:10E8E0000080FA00000006000800FA0030079800D7
:10E8F0000000EB00000F7800240037003E0090007D
:10E90000000040001E004000000040008000780031
:10E910000000210000804000CF80DE0023002000A6
:10E92000E23D2200F2E807009E007800E03D220070
:10E93000104078000080FB004800DD0000017800F6
:10E94000018040000E0040000080E80002087800CE
:10E950001E0178001E007800000040000E004000FC
:10E960000080E80090007800F03D22001040780020
:10E970000080FB0080807000020041000E0040001B
:10E980000080E800010878001E0FE8001000200059
:10E990009E0F1000D9FF34001E009000AE009000C2
:10E9A000801F7800811F7800906F2A00801F7800F8
:10E9B00060412100BCD40700E68757006041210078
:10E9C00043E40700604121007CE407000080FA0076
:10E9D000000006000E00FA0050079800610798003A
:10E9E0000000EB00100798000000EB00000F78001B
:10E9F000230037006E0090001E0040008000780069
:10EA00005E009000008040009040780090C3B3000A
:10EA100080CF500009003C006E0090001E004000B6
:10EA2000800078005E0090000080400090407800F8
:10EA3000F0C2B30080CF500006003C009E0078007A
:10EA400064004700808040000040EB008048780070
:10EA50000A0037001E0178006E0090001E00400082
:10EA6000800078005E0090000080400090407800B8
:10EA70006400470000004100014878001E0FE800D4
:10EA8000400020009E0F1000DAFF340064004700B1
:10EA900035D40700100798001E0090000080FA008F
:10EAA000000006000E00FA00500798006107980069
:10EAB0000000EB00100798000000EB00000F78004A
:10EAC0002C0037006E0090001E004000800078008F
:10EAD0005E009000008040009040780090C3B3003A
:10EAE00080CF500009003C006E0090001E004000E6
:10EAF000800078005E009000008040009040780028
:10EB0000F0C2B30080CF50000F003C006E009000B8
:10EB10001E004000800078005E00900000804000F1
:10EB200090407800D0C2B30080CF50000600320081
:10EB30009E00780064004700808040000040EB00A9
:10EB4000804878000A0037001E0178006E009000AF
:10EB50001E004000800078005E00900000804000B1
:10EB600090407800640047000000410001487800B0
:10EB70001E0FE800400020009E0F1000D1FF34005F
:10EB800064004700F8D30700100798001E009000AB
:10EB90000080FA00000006008200FA00889FBE0094
:10EBA0000087980070004700010878001200980064
:10EBB00023009800340098004500980088EE8000FB
:10EBC0006140B9001BCF0700603F9800713F98007B
:10EBD0000800E00007003D00020020000378240048
:10EBE0006E389000FE389000CBCC0700603F980054
:10EBF000713F980052A32F00E3C823006E389000A5
:10EC0000FE389000FECF07007FD107001007980064
:10EC1000210798007E0090000020A1007007980056
:10EC20000000EB00000F780010EF80000000E00013
:10EC300002003A006018200010EF880010EF8000FA
:10EC40008000780010F080000080500010F08800F4
:10EC5000D0C0B300ECE20700A0C0B300EAE20700B6
:10EC600070004700100078000000E00049003A0002
:10EC700061DF21009140780010C4B30080CF5000C4
:10EC80000700320061DF21009140780020C4B3000A
:10EC900080CF50000200320010C4B300F6FDB70070
:10ECA000F6DDBF000080FB00503F980010042000FC
:10ECB000DE389000808F50000500320020042000D4
:10ECC0005E399000800F51001200320021003700A1
:10ECD000F1EF8000E0192000808F500003003E001B
:10ECE0000000EB00A0EE88001A003700F1EF800072
:10ECF000802E2000808F500003003E0060272000FF
:10ED0000A0EE880013003700C03E2000A0EE88006F
:10ED100010003700F1EF8000E0192000808F5000D4
:10ED200003003E000000EB00A0EE88000900370061
:10ED3000F1EF8000802E2000808F500003003E0005
:10ED4000C01E2000A0EE880002003700C03E200058
:10ED5000A0EE8800F06F2A0098E30700F6DDBF0000
:10ED6000A9E20700D0C0B300A7E20700A0C0B3002B
:10ED7000A5E20700E0702A0090E30700A0EE800003
:10ED80000FE30700D0C0B3009FE20700A0C0B300AC
:10ED90009DE20700A0EE80000000E0003C00320091
:10EDA000F0EF800030EF880070004700100078001E
:10EDB0000000E00030003A00F1EF800000F0800039
:10EDC0000000D100008440006140B90099CE0700E6
:10EDD000303F9800413F98000800E00007003D00E8
:10EDE00002002000037824003E389000CE389000C6
:10EDF00049CC0700303F9800413F980018F0800050
:10EE00006140B9008BCE0700103F9800213F980069
:10EE10000800E00007003D00020020000378240005
:10EE20001E389000AE3890003BCC0700103F980091
:10EE3000213F98001E019000AE0190001E38900006
:10EE4000AE3890005FCD07000001BE003E38900054
:10EE5000CE38900030CC070011CE070040EF88007C
:10EE600040EF800080007800F0EF800000805000CC
:10EE7000F0EF880006003700C1EF800020EF80002F
:10EE80008080400030EF800000805000F0EF88006C
:10EE9000D0E78000E20F50002903320070004700E5
:10EEA000100078000000E00087003A00F1EF8000D9
:10EEB00000F080000000D100008450006140B900E3
:10EEC0005CCE070070379800013F98000800E00012
:10EED00007003D0002002000037824007E309000EF
:10EEE0008E3890000CCC070070379800013F9800D6
:10EEF00018F080006140B9004ECE070050379800EE
:10EF0000613798000800E00007003D000200200083
:10EF1000037824005E309000EE309000FECB0700B6
:10EF200050379800613798001E019000AE019000A4
:10EF30005E309000EE30900022CD07000001BE0050
:10EF40007E3090008E389000F2CB07006011B80040
:10EF5000CFCD07000000E0000100340003003700BF
:10EF600040012000400798002A003700F1EF8000A0
:10EF700000F080000000D100008450006140B90022
:10EF80002CCE070030379800413798000800E00089
:10EF900007003D0002002000037824003E3090006E
:10EFA000CE309000DCCB0700303798004137980016
:10EFB00018F080006140B9001ECE0700103798009D
:10EFC000213798000800E00007003D000200200003
:10EFD000037824001E309000AE309000CECB0700A6
:10EFE00010379800213798001E019000AE01900064
:10EFF0001E309000AE309000F2CC07000001BE0041
:10F000003E309000CE309000C2CB0700EBCD070021
:10F01000400798000000EB003007980070004700A0
:10F02000100178003E009000CE0090005A030700C7
:10F0300070004700100078008000E8007000470072
:10F0400001087800F1EF800000F080000000D1009E
:10F05000008050004007980010F0800030079800B2
:10F0600070004700100178003E009000CE00900034
:10F070004903070070004700100078008000E80096
:10F080007000470001087800F1EF800000F0800078
:10F090000000D10000804000400798007000470049
:10F0A000100178003E009000CE0090003A03070067
:10F0B00070004700100078008000E80070004700F2
:10F0C00001087800C4023700D0E780000000E000AB
:10F0D0007A023A00C1EF8000D0EF80000000D1003A
:10F0E000008440006140B900D2CD0700702F980025
:10F0F000013798000800E00007003D0002002000F2
:10F10000037824007E2890008E30900082CB070088
:10F11000702F980001379800E8EF80006140B90037
:10F12000C4CD0700502F9800612F98000800E00020
:10F1300007003D0002002000037824005E289000B4
:10F14000EE28900074CB0700502F9800612F980094
:10F150001E019000AE0190005E289000EE28900005
:10F1600098CC07000001BE007E2890008E309000F1
:10F1700069CB070091CD070050079800F1EF8000A0
:10F1800000F080000000D100008450006140B90010
:10F19000A8CD0700302F9800412F98000800E0000C
:10F1A00007003D0002002000037824003E28900064
:10F1B000CE28900058CB0700302F9800412F9800A0
:10F1C00018F080006140B9009ACD0700102F980018
:10F1D000212F98000800E00007003D0002002000F9
:10F1E000037824001E289000AE2890004ACB070028
:10F1F000102F9800212F98001E019000AE01900062
:10F200001E289000AE2890006ECC07000001BE00C2
:10F210003E289000CE2890003ECB070067CD070027
:10F2200060079800DE0090006E009000808F500014
:10F23000E5013600E1EF800010F08000808F500083
:10F24000000136005E0490006140B90079CD0700EE
:10F2500070279800012F98000800E00007003D008B
:10F2600002002000037824007E2090008E28900069
:10F2700029CB070070279800012F980018F0800014
:10F280006140B9006BCD07005027980061279800B6
:10F290000800E00007003D00020020000378240081
:10F2A0005E209000EE2090001BCB070050279800B6
:10F2B000612798001E019000AE0190005E20900032
:10F2C000EE2090003FCC07000001BE007E209000A1
:10F2D0008E2890000FCB070038CD0700500798000C
:10F2E000C1EF8000D0EF80000000D100008040001E
:10F2F00040079800E0EF800030079800700047005A
:10F30000100178003E009000CE009000A20207009D
:10F3100070004700100078008000E800700047008F
:10F3200001087800C1EF8000D0EF80000000D1001C
:10F33000008440006140B9003ECD070030279800AE
:10F34000412798000800E00007003D00020020006F
:10F35000037824003E209000CE209000EECA0700E3
:10F360003027980041279800E1EF800010F08000DE
:10F37000008450006140B9002ECD0700102798008E
:10F38000212798000800E00007003D00020020004F
:10F39000037824001E209000AE209000DECA0700F3
:10F3A00010279800212798001E019000AE019000C0
:10F3B0001E209000AE20900002CC07000001BE008D
:10F3C0003E209000CE209000D3CA0700B4CC0700A6
:10F3D000000F78001E017800F1EF800000F080003F
:10F3E0000000D10000805000800F51004200360024
:10F3F0001E007800CF80DE000ECD07000004BE00A6
:10F400001E019000AE01900000002000011A2400AF
:10F41000ECCB07000001BE000800BE00BECA07001A
:10F42000E6CC07004007980010F080007400500000
:10F430003007980070004700100178003E009000EF
:10F44000CE009000540207007000470010007800C2
:10F450008000E80070004700010878001E00780076
:10F46000CF80DE00F3CC07000004BE001E01900038
:10F47000AE01900000002000011A2C00D1CB070043
:10F480000001BE000800BE00A3CA0700CBCC0700E5
:10F490004007980070004700100178003E0090007F
:10F4A000CE0090003C02070070004700100078007A
:10F4B0008000E80070004700010878001E00780016
:10F4C0004007980010F08000300798007000470057
:10F4D000100178003E009000CE0090002E02070040
:10F4E00070004700100078008000E80070004700BE
:10F4F00001087800B80137005E019000F1EF80004C
:10F5000000F080000000D100808050005E0090007C
:10F51000008050000000D10000004100400798002A
:10F5200018F080006140B900C2CC0700701F98003D
:10F53000012798000800E00007003D0002002000BD
:10F54000037824007E1890008E20900072CA070075
:10F55000701F980001279800F1EF800000F08000F4
:10F560000000D100808050005E00900000805000BC
:10F570000004D1006140B900AECC0700501F9800D4
:10F58000611F98000800E00007003D000200200015
:10F59000037824005E189000EE1890005ECA070001
:10F5A000501F9800611F98001E019000AE0190004E
:10F5B0005E189000EE18900091CD07000001BE008B
:10F5C0007E1890008E20900052CA07007BCC070066
:10F5D0003007980070004700100178003E0090004E
:10F5E000CE009000EC01070070004700100078008A
:10F5F0008000E8007000470001087800F1EF80000B
:10F6000000F080000000D10000805000400798000A
:10F6100010F080003007980070004700100178005B
:10F620003E009000CE009000DB0107007000470014
:10F63000100078008000E8007000470001087800A2
:10F64000650137006E0490006140B90079CC070075
:10F65000301F9800411F98000800E00007003D009F
:10F6600002002000037824003E189000CE1890007D
:10F6700029CA0700301F9800411F9800E8EF80005A
:10F680006140B9006BCC0700101F9800211F980043
:10F690000800E00007003D0002002000037824007D
:10F6A0001E189000AE1890001BCA0700101F98008B
:10F6B000211F98001E019000AE0190001E189000BE
:10F6C000AE1890003FCB07000001BE003E1890002E
:10F6D000CE18900010CA070038CC070060079800C9
:10F6E000F1EF800000F080000000D10000845000A5
:10F6F0006140B9004FCC070070179800011F9800B7
:10F700000800E00007003D0002002000037824000C
:10F710007E1090008E189000FFC9070070179800A7
:10F72000011F980011F08000E0EF8000008450007D
:10F730006140B9003FCC070050179800611798004E
:10F740000800E00007003D000200200003782400CC
:10F750005E109000EE109000EFC90700501798005F
:10F76000611798001E019000AE0190005E1090009D
:10F77000EE10900013CB07000001BE007E10900039
:10F780008E189000E3C90700C5CB0700000F780072
:10F790001E017800C1EF8000D0EF80000000D10092
:10F7A00000804000800F5100200031001E007800D2
:10F7B00040079800E0EF8000300798007000470095
:10F7C000100178003E009000CE009000720107000A
:10F7D00070004700100078008000E80070004700CB
:10F7E00001087800F1EF800000F080000000D100F7
:10F7F000008050004007980010F08000300798000B
:10F8000070004700100178003E009000CE0090008C
:10F810006101070070004700100078008000E800D8
:10F820007000470001087800EB003700C1EF80004E
:10F83000D0EF80000000D100008040004007980019
:10F84000E0EF80003007980070004700100178005A
:10F850003E009000CE0090004F010700700047006E
:10F86000100078008000E800700047000108780070
:10F87000C1EF8000D0EF80000000D1008081400007
:10F880006E019000C1EF8000D0EF80000000D10039
:10F8900000804000000051000000D10000804100C5
:10F8A00040079800E8EF80006140B900E1CB070015
:10F8B00030179800411798000800E00007003D004D
:10F8C00002002000037824003E109000CE1090002B
:10F8D00091C9070030179800411798006E019000F9
:10F8E000C1EF8000D0EF80000000D1000080400018
:10F8F000000051000004D1006140B900CDCB0700E9
:10F9000010179800211798000800E00007003D003C
:10F9100002002000037824001E109000AE1090001A
:10F920007DC9070010179800211798001E0190004C
:10F93000AE0190001E109000AE109000B0CC0700F9
:10F940000001BE003E109000CE10900071C907006B
:10F950009ACB07003007980070004700100178002C
:10F960003E009000CE0090000B01070070004700A1
:10F97000100078008000E80070004700010878005F
:10F98000F1EF800000F080000000D1000080500006
:10F990004007980010F08000300798007000470082
:10F9A000100178003E009000CE009000FA000700A1
:10F9B00070004700100078008000E80070004700E9
:10F9C0000108780084003700C1EF8000D0EF80008C
:10F9D0000000D1000080400040079800E0EF800068
:10F9E0003007980070004700100178003E0090003A
:10F9F000CE009000E800070070004700100078007B
:10FA00008000E80070004700010878005E00900068
:10FA1000400798000000EB00300798007000470096
:10FA2000100178003E009000CE009000DA00070040
:10FA300070004700100078008000E8007000470068
:10FA4000010878006E0090004007980070004700A1
:10FA5000100178003E009000CE009000CE0007001C
:10FA600070004700100078008000E8007000470038
:10FA700001087800F1EF800000F080000000D10064
:10FA8000008050004007980010F080003007980078
:10FA900070004700100178003E009000CE009000FA
:10FAA000BD00070070004700100078008000E800EB
:10FAB000700047000108780047003700F1EF800030
:10FAC00000F080000000D100008050004007980046
:10FAD00010F0800030079800700047001001780097
:10FAE0003E009000CE009000AB0007007000470081
:10FAF000100078008000E8007000470001087800DE
:10FB0000F1EF800000F080000000D1000080400094
:10FB10004007980070004700100178003E009000F8
:10FB2000CE0090009C000700700047001000780095
:10FB30008000E800700047000108780026003700C8
:10FB4000F0EF8000400798000000EB0030079800BD
:10FB500070004700100178003E009000CE00900039
:10FB60008D00070070004700100078008000E8005A
:10FB7000700047000108780010F0800030079800FE
:10FB800070004700100178003E009000CE00900009
:10FB90008100070070004700100078008000E80036
:10FBA00070004700010878000000EB003007980063
:10FBB00070004700100178003E009000CE009000D9
:10FBC0007500070070004700100078008000E80012
:10FBD0007000470001087800700047002000900086
:10FBE0008000E80070004700210098007000470086
:10FBF000200090008000780050EE8000808F500040
:10FC00004D003A00D0E78000E20F50004A00320079
:10FC1000D0E780000000E00011003A00F1EF800022
:10FC200000F080000000D1000080400040079800F4
:10FC300010F0800030079800700047001001780035
:10FC40003E009000CE009000530007007000470077
:10FC5000100078008000E80070004700010878007C
:10FC6000F1EF800000F080000000D100008440002F
:10FC70006140B900EFCA0700700F980001179800A3
:10FC80000800E00007003D00020020000378240087
:10FC90007E0890008E1090009FC80700700F98009B
:10FCA0000117980018F080006140B900E1CA070010
:10FCB000500F9800610F98000800E00007003D0019
:10FCC00002002000037824005E089000EE089000F7
:10FCD00091C80700500F9800610F98001E01900016
:10FCE000AE0190005E089000EE089000B5C90700D4
:10FCF0000001BE007E0890008E10900086C80700AC
:10FD0000AECA0700400798000000EB0030079800DB
:10FD100070004700100178003E009000CE00900077
:10FD20001D00070070004700100078008000E80008
:10FD3000700047000108780010F08000E0EF8800B4
:10FD4000F0EF8000C0EF880000F08000D0EF880066
:10FD500030EF800020EF88007000470080007800BE
:10FD60000E8090001101BE000288BE0064004000B9
:10FD7000E48040001101BE000288BE006400400023
:10FD8000E4804000110878000E8090004F04BE000F
:10FD90000080FA00000006000C00FA00200798001E
:10FDA00031079800420798006A0047003BE50700CA
:10FDB0005E009000100798001E0090000020A10037
:10FDC0000030A1000040A1000050A10010079800E1
:10FDD0001E00900040E507004E0090000000E0008B
:10FDE00004003A004DE5070000002100010020005A
:10FDF000A8E407000000EB00000F780022003700A5
:10FE000046E507001E007800000040000E0040009C
:10FE10006400400010007800004178004E0090001F
:10FE2000000040001E0040000000400080007800FC
:10FE30001000210000804000CF80DE00BEE40700FB
:10FE400036E507001E007800000040000E0040006C
:10FE500064004000100078004800DE000041780097
:10FE60004E009000000040001E00400000004000D6
:10FE7000800078000000210000804000CF80DE007C
:10FE8000ADE407001E0FE800100020009E0F1000D8
:10FE9000DBFF34001E0090000020A0000030A00016
:10FEA0000040A0000050A100100798001E00900024
:10FEB00009E507004E009000C1DE0700E0712A004E
:10FEC0003EDF07002E009000800078003E0090008A
:10FED00006000700D0C0B3004BDE0700A0C0B3008F
:10FEE00049DE07000080FA00000006000400FA0066
:10FEF000000F7800110798001E007800B0DE0700A0
:10FF0000C0C2B30040DE07001E009000ACDE070058
:10FF10000080FA00000006002800FA00889FBE005A
:10FF2000600798000000EB00100798000000EB004D
:10FF3000200798000000EB00000F78002700370032
:10FF40006E009000000040001E00400000004000D5
:10FF500080007800000021000080400001002000A7
:10FF600023002000E23D220061E307009E007800AC
:10FF7000E03D2200104078000080FB004800DD00DA
:10FF8000000178006A08B900E600400020CE210098
:10FF900000804000020878009E0178001E00780072
:10FFA0006A00B900E600400020CE21000080400039
:10FFB00090007800F03D2200104078000080FB00A7
:10FFC000008170006A18B900E600400020CE2100D0
:10FFD00000804000020878001E0FE800100020009A
:10FFE0009E0F1000D6FF360061DF2100914078009F
:10FFF00020C4B30080CF500009003A0010EF800009
:020000040001F9
:1000000022002000110009000200D80080007800C2
:10001000504F200001005000D0ED88000200370052
:1000200000462000D0ED880050EF80000000E00086
:100030001200320070F0800001102000010060000A
:100040000000E0000D003A0070F080000108200080
:10005000010060000000E00008003A0043E7800073
:1000600091E7800050EF8000000178001100090046
:100070008280D8000080510040E78800A0EE800018
:100080000000E0000C003200C0ED8000800078002D
:10009000A0EE80008080500040EF80008080400013
:1000A00090E780008080500080EF8000008040005A
:1000B00090E7880007003700C0ED800080007800DE
:1000C00090E780008080500080EF8000008040003A
:1000D00090E78800A0EF80000000E00007003200F9
:1000E0001000200002020700200798000000EB002B
:1000F000FF01070010079800040037000000EB0024
:10010000200798000000EB001007980091E780009E
:100110002E0090000080400090E788006E00900064
:100120000000E00019003A0070F080000104200097
:10013000010060000000E00014003A0070F0800050
:1001400001082000010060000000E0000F003A00FC
:1001500070F0800001102000010060000000E0004D
:100160000A003A00D1ED800010EF8000808050003E
:1001700090EF8000808040001E00900000804000D2
:100180007E00500040E788004C00370070F080008F
:1001900001082000010060000000E00010003200B3
:1001A00061DF21009140780020C4B30080CF50006F
:1001B0000B003200D1ED800010EF800080805000F5
:1001C00090EF8000808040001E0090008080400002
:1001D00050FB2F000080400040E7880037003700C8
:1001E00070F0800001082000010060000000E000C5
:1001F0000B003200D1ED800010EF800080805000B5
:1002000090EF8000808040001E00900080804000C1
:1002100050FB2F000080400040E788002700370097
:1002200070F0800001102000010060000000E0007C
:100230000B003A0041E78000D0ED80008080400054
:1002400090EF8000808040001E0090008080400081
:1002500010EF80000080500040E788001700370052
:100260006E0090000000E0000B003A0041E78000C3
:10027000D0ED800000814000D0ED8000800078004B
:10028000B0EE800000805000000051007E00500061
:1002900040E788000900370041E78000D0ED80008A
:1002A00000814000D0ED800080007800B0EE80003A
:1002B000008050000000510040E7880070F080008E
:1002C00001102000010060000000E0004700320043
:1002D000B1EE8000E0EE8000808F500043003200DD
:1002E00048E780006140B90052C907002017980014
:1002F000311798000800E00007003D0002002000D0
:10030000037824002E109000BE10900002C7070052
:100310002017980031179800C8EE80006140B9009E
:1003200044C9070000179800111798000800E00062
:1003300007003D0002002000037824000E1090000A
:100340009E109000F4C6070000179800111798003F
:1003500098E780006140B90036C90700600F980037
:10036000710F98000800E00007003D000200200027
:10037000037824006E089000FE089000E6C607008F
:10038000600F9800710F98006E099000FE099000B0
:100390000E1090009E109000DEC60700B2E98000AB
:1003A000C3E9800016CA07000001BE002E109000AD
:1003B000BE109000D7C6070000C9070040E78800BC
:1003C0006E0090000000E00008003A0070F080002D
:1003D00001042000010060000000E00003003A007A
:1003E00040E780007E00500040E7880042E7800040
:1003F0009E00900090EF800000804000B03CB00074
:10040000800F51000C00390071DF2100914078000D
:1004100030C5B30080CF500014013A0042E780009D
:100420009E00900090EF800000804000A03FB00050
:10043000800F51000D0131000000EB00000F78002B
:100440002D0037001E0078006A00B900E40040006B
:1004500020CE2100808040000000EB008008780062
:100460009E017800530F98001E0078006A00B900C2
:10047000E600400020CE21000080400010047800FB
:100480006140B900EBC80700300F9800410F980099
:100490000800E00007003D0002002000037824006F
:1004A0003E089000CE0890009BC60700300F9800D1
:1004B000410F980002002000832C24003E08900089
:1004C000CE089000CEC9070002002000832C240033
:1004D000BCC70700B9C8070000017800DE0990001A
:1004E0006A18B900E600400020CE210000804000DC
:1004F000020878001E0FE800100020009E0F100078
:10050000D0FF36000000EB00000F78003600370007
:100510001E0078006A00B900E600400020CE2100ED
:1005200000804000100178001E0078006A00B900C9
:10053000E800400020CE210000804000100078003C
:10054000800F5100140036009E0178001E007800D4
:100550006A00B900E600400020CE21000080400083
:10056000100178001E0078006A00B900E800400021
:1005700020CE2100008040001000780000005100D3
:1005800080007800038041000E00400068004000B9
:1005900001087800130037009E0178001E007800E3
:1005A0006A00B900E800400020CE21000080400031
:1005B000100178001E0078006A00B900E6004000D3
:1005C00020CE210000804000100078000000510083
:1005D00080007800038041000E0040006800400069
:1005E000010878001E0FE800130020009E8F110004
:1005F000C7FF3600CE0090005E009000808F500054
:10060000040034003E0090000000A0003007980075
:10061000030037003E0090000000A1003007980062
:100620003E0090006140600000C0EA006140600050
:10063000BE0090000080FB006100600000014000EF
:10064000D0FF2F008080600082807000310798000A
:100650006E0090000000E0001200320070F0800098
:1006600001082000010060000000E0000D003A00D9
:100670003E0090000000D100614060000081FB005E
:1006800070EE80006C00B900F60140006A10B900FD
:100690008080E80020CE2100008040000308780020
:1006A0000A0037003E0090000000D1006140600069
:1006B0000080FB006A00B9008080E80020CE2100A5
:1006C0008080400060012000800878003E0090009B
:1006D000614060000080FB00000040000E00400010
:1006E00068004000100078000000E0003E00340088
:1006F0003E009000614060000080FB00200F9800E9
:100700003E0090000000D100614060000080FB00CE
:100710006A00B9008080E80020CE210000804000FF
:10072000100478006140B90042C80700000F98002B
:10073000110F98000800E00007003D0002002000B3
:10074000037824000E0890009E089000F2C5070070
:10075000000F9800110F98003E0090000000D1009B
:10076000614060000080FB00000040000E0040007F
:100770006800400010007800CF80DE002DC8070020
:100780000001BE000E0890009E0890001CC90700E2
:100790000004BE003E009000614060000080FB004D
:1007A000000040000E00400068004000100078008B
:1007B000CF80DE001FC807000001BE000800BE0099
:1007C00000C70700FDC7070000017800AE099000D0
:1007D0006A18B9008080E80020CE21000080400027
:1007E00002087800090037003E0090006140600078
:1007F0000080FB006A00B9008080E80020CE210064
:1008000080804000803E2000800878000064200046
:10081000E008880021E1A8000000EB00C008880083
:100820006700070070F08000700060000000E000CA
:100830000200320020722A0055F507006E00900079
:100840000000E800600798000000EB00E1E6070008
:100850000000EB0060F088000000EB0050F0880022
:100860006E009000700798001D00370042E780007E
:100870009E00900090EF80000080400080005100BA
:1008800050C32F00008040009E00900092EF800037
:1008900043E78000801F7800811F7800821F780066
:1008A000B03C2000801F7800831F780040722A002F
:1008B000801F780060412100FBCC0700EC875700C7
:1008C00060412100BDDC0700D0682A0030F5070038
:1008D00080C3B3008DDB07008001EB007307980035
:1008E0007E0090004F04BE000080FA000000060069
:1008F0000C00FA00889FBE0040079800A0EF80001F
:10090000CF80DE00CBC70700020020000342240096
:10091000ACC60700DDC50700008FBE00C1ED80003A
:1009200080EF8000008040008000780090E7800029
:1009300000805000300798003E009000CF80DE001D
:10094000BCC707000004BE001E00BE003CC6070076
:100950000001BE000800BE00A9C8070050C707007C
:10096000200798004E009000E10F500005003A006B
:10097000BE0090002E00900080805000510798002B
:100980000B0037002E009000CF80DE00A9C70700C3
:100990000004BE001E00BE001BCA07000001BE000E
:1009A0000800BE0096C807003DC707005007980022
:1009B0005E0090004F04BE000080FA0000000600B8
:1009C0003000FA00881F780071E78000A003200043
:1009D000808F500003003E0000372000B00C8800DC
:1009E0003500370071E78000703E2000808F500096
:1009F0000300360000192000B00C88002E003700DC
:100A000071E7800060FC2F0000804000E23A200087
:100A1000110009000280D800000478006140B9008C
:100A200081C7070040179800511798006217980077
:100A3000731798000800E0000C003D006022B80029
:100A400006002000070F24004E109000DE109000DA
:100A50006E119000FE119000B1C40700401798007D
:100A6000511798006217980073179800040020002F
:100A700005C02E00F6FF2F00370724004E1090000F
:100A8000DE1090006E119000FE119000E7C7070085
:100A90006022B80006802800370D2400E3C7070055
:100AA0006022B80006002000970724009CC40700BD
:100AB0001CC70700B00C880091E78000A0E7800009
:100AC000808F500002003A0000192000B00C88000E
:100AD00021E7800060072000808F500003003E0067
:100AE00000372000000D88003500370021E7800026
:100AF000703E2000808F5000030036000019200057
:100B0000000D88002E00370021E78000A0F82F009C
:100B10000080400022372000110009000280D80028
:100B2000000478006140B9003FC707000017980033
:100B30001117980022179800331798000800E0005A
:100B40000C003D006022B80006002000070F2400C2
:100B50000E1090009E1090002E119000BE1190007B
:100B60006FC407000017980011179800221798000B
:100B7000331798000400200005C02E00F6FF2F0058
:100B8000370724000E1090009E1090002E11900048
:100B9000BE119000A5C707006022B800068028009B
:100BA000370D2400A1C707006022B800060020000E
:100BB000970724005AC40700DAC60700000D880012
:100BC00041E7800050E78000808F500002003A002B
:100BD00000192000000D8800B80C80006140B900A9
:100BE00011C70700400F9800510F9800620F98003E
:100BF000730F98000800E0000C003D006022B80070
:100C000006002000070F24004E089000DE08900028
:100C10006E099000FE09900041C40700400F980043
:100C2000510F9800620F9800730F98006022B8006F
:100C300006002000970724004E089000DE08900070
:100C40006E099000FE09900020C607000000E00039
:100C500001003A0022003700080D80006140B90011
:100C6000F1C60700000F9800110F9800220F98009E
:100C7000330F98000800E0000C003D006022B8002F
:100C800006002000070F24000E0890009E08900028
:100C90002E099000BE09900021C40700000F9800A3
:100CA000110F9800220F9800330F98006022B800AF
:100CB00006002000970724000E0890009E08900070
:100CC0002E099000BE0990005FC507000000E000FB
:100CD000010032000200370000372000B00C88000D
:100CE000080D80006140B900CFC60700400798009A
:100CF0005107980062079800730798000800E00009
:100D00000C003D006022B80006002000070F240000
:100D10004E009000DE0090006E019000FE019000F9
:100D2000FFC307004007980051079800620798002A
:100D3000730798006022B80006002000970724007F
:100D40004E009000DE0090006E019000FE019000C9
:100D5000DEC507000000E00001003A001A0037007D
:100D6000B80C80006140B900AFC60700009FBE000C
:100D70000297BE000800E00008003D006022B800B5
:100D800006002000070F24003E00BE002E01BE001A
:100D9000E3C30700009FBE000297BE006022B800B8
:100DA00006002000970724003E00BE002E01BE0072
:100DB00025C507000000E0000100320002003700F6
:100DC00000372000000D88004F0478000080FA00F2
:100DD000000006001000FA00889FBE00400798003F
:100DE0000000EB00000F7800360037001E0078008E
:100DF0006A00B900E600400020CE210000804000DB
:100E0000100178001E0078006A00B900E800400078
:100E100020CE21000080400010007800800F51009B
:100E2000140036009E0178001E0078006A00B900A8
:100E3000E600400020CE2100008040001001780034
:100E40001E0078006A00B900E800400020CE2100B2
:100E50000080400010007800000051008000780001
:100E6000038041000E00400064004000010878004B
:100E7000130037009E0178001E0078006A00B90058
:100E8000E800400020CE21000080400010017800E2
:100E90001E0078006A00B900E600400020CE210064
:100EA00000804000100078000000510080007800B1
:100EB000038041000E0040006400400001087800FB
:100EC0001E0FE800100020009E0F1000C7FF360024
:100ED000AE0090003E009000808F5000040034006F
:100EE0001E0090000000A0001007980003003700CB
:100EF0001E0090000000A100100798001E00900046
:100F00006140600000C0EA00614060009E00900007
:100F10000080FB006100600000014000D0FF2F0056
:100F20008080600082807000110798001E00900091
:100F30000000D100614060000080FB004E01900085
:100F40006A00B9008080E80020CE210000804000C7
:100F5000020878001E009000614060000080FB00E5
:100F6000000040000E0040006400400010007800C7
:100F70000000E0003E0034001E0090006140600070
:100F80000080FB00700798001E0090000000D10058
:100F9000614060000080FB006A00B9008080E800CA
:100FA00020CE210000804000100478006140B9008C
:100FB00020C6070050079800610798000800E0006D
:100FC00007003D0002002000037824005E0090002E
:100FD000EE009000D0C3070050079800610798000A
:100FE0001E0090000000D100614060000080FB0006
:100FF000000040000E004000640040001000780037
:10100000CF80DE000BC607000001BE005E0090002E
:10101000EE009000FAC607000004BE001E0090001B
:10102000614060000080FB00000040000E004000B6
:101030006400400010007800CF80DE00FDC507008E
:101040000001BE000800BE00DEC40700DBC50700CB
:1010500000017800FE0190006A18B9008080E80065
:1010600020CE2100008040000208780009003700EF
:101070001E009000614060000080FB006A00B90023
:101080008080E80020CE210080804000803E20004B
:10109000800878004F04BE000080FA0000000600BF
:1010A0000000FA00E482A800E082A900001E2000EF
:1010B0008A0107000080FA00000006000600FA001E
:1010C000000F7800110798001E007800104078008B
:1010D0008000FB0050072000808F5000010032008C
:1010E000070037001E009000950007001E009000CA
:1010F000ED0007000000EB00200798000200370019
:1011000020032000200798002E0090000080FA00A5
:10111000000006001000FA00881F78007007980091
:101120000000EB00000F7800060037001E0078007A
:101130000E81E800800040000000EB008030790064
:101140001E0FE800500020009E0F1000F7FF340033
:101150000000EB00000F7800070037001E00780049
:10116000800078007E009000808040000040EB000E
:10117000804878001E0FE800C00020009E0F10007D
:10118000F6FF340030032000F10007000000E0000B
:1011900001003A00FFFF37002D0107000000EB00BF
:1011A000000F7800070037001E04780028010700B0
:1011B000000178008E80E8000800440002B078004A
:1011C0001E0FE800500020009E0F1000F6FF3400B4
:1011D0001F010700E482A800E082A9000000EB00E4
:1011E000000F7800060037001E0078008E80E800AF
:1011F0000000400060807800F1D907001E0FE80071
:10120000500020009E0F1000F7FF3400B0002000B7
:10121000000F78003E0037001E007800610060007B
:101220000004E0000E0032001E007800800078000C
:101230007E009000808140001E0078002200200087
:10124000110009000200D8008E80E8000000400074
:10125000608078006F406000804978000D003700A2
:101260001E007800800078007E00900080814000A1
:101270001E00780022002000110009000200D800A2
:101280008E80E80000004000608078004480DE002E
:10129000804978001E007800800078007E00900071
:1012A0000080400010407800E94F50000C003C00E6
:1012B0001E007800800078007E00900000814000D1
:1012C0001E007800800078007E00900000804000C2
:1012D000104078000043B000004978000B00370050
:1012E0001E007800800078007E00900000814000A1
:1012F0001E007800800078007E0090000080400092
:10130000104078007045B000004978001E0FE900D9
:101310001E00E000C0FF3C0080C2B3003AD90700C5
:101320007E00900025DA070090C2B30036D907008E
:101330007E0090004F0478000080FA000000060054
:101340001000FA00881F7800700798000000EB007A
:10135000000F7800060037001E0078000E81E800BC
:10136000800040000000EB00803079001E0FE80094
:10137000400020009E0F1000F7FF340030032000D3
:10138000730007000000E00001003A00FFFF370093
:10139000AF0007000000EB00000F780007003700E7
:1013A0001E047800AA000700000178008E80E80083
:1013B0000800440002B078001E0FE8005000200032
:1013C0009E0F1000F6FF3400A1000700E482A80081
:1013D000E082A9007E009000610060000004E0004F
:1013E0000C0032000000EB00000F78000600370010
:1013F0001E0078008E80E8000000400060807800C9
:10140000C2D807001E0FE800500020009E0F1000F9
:10141000F7FF34007E0090000000D1006100600002
:101420000004E0000C0032000000EB00000F780028
:10143000060037001E0078008E80E80000004000A3
:1014400060807800F0D807001E0FE80050002000F0
:101450009E0F1000F7FF34007E0090004200DE0077
:10146000610060000004E0000C0032000000EB00AE
:10147000000F7800060037001E0078008E80E8001C
:10148000000040006080780019D907001E0FE800B6
:10149000500020009E0F1000F7FF34004F0478002A
:1014A0000080FA00000006000200FA00000F780039
:1014B0009E007800618060000004E00008003200B7
:1014C00000C1B30091D8070050C0B3008FD8070007
:1014D00090C0B3008DD8070010C0B3008BD80700B0
:1014E0001E0078000000D100610060000004E000F0
:1014F0000800320000C1B300C3D8070050C0B300D9
:10150000C1D8070090C0B300BFD8070010C0B30017
:10151000BDD807001E0078004200DE0061006000B8
:101520000004E0000800320000C1B300F0D807005A
:1015300050C0B300EED8070090C0B300ECD807004D
:1015400010C0B300EAD807000080FA0000000600CF
:101550000800FA0020079800270007000000E000BC
:1015600003003A000000EB00300798001F0037002E
:101570000000EB0010079800170037002E009000C5
:10158000610060000004E000030032001000200051
:10159000000F780002003700C0032000000F780021
:1015A000E482A900E082A9001E0078004B00070039
:1015B000E482A800100420001E005000470007002D
:1015C0002E0090000080D100200798001E0090009F
:1015D0000000E800100798001E009000E70F500080
:1015E000E6FF340010002000300798003E00900015
:1015F0000080FA00000006000200FA000040EB0044
:10160000004F7800E482A900E082A900001E2000BB
:1016100032000700E482A800E082A800C003200096
:101620002E000700101780004400DE0061006000FB
:101630000000E00001003A001E4FE800B004200066
:10164000260007001E80FB000080FA000000060054
:101650000400FA000000EB00100798000000EB0007
:10166000000F78000000EB00000F78001500370035
:101670001E0090000000400010079800E482A900BE
:10168000E082A9005000200014000700E082A800BA
:101690001000200011000700101780004400DE0039
:1016A000610060000004E000030032001E009000B2
:1016B0000000E80010079800600320000700070002
:1016C0001E0FE800700020009E0F1000E8FF34009D
:1016D0001E0090000080FA00000006000400FA00DE
:1016E000100798000000EB00000F78000D00370095
:1016F00000000000000000000000000000000000EA
:1017000000000000000000000000000000000000D9
:1017100000000000000000000000000000000000C9
:101720001E0FE8001E0090009E0F1000F0FF350015
:101730000080FA00000006000200FA000000EB0042
:10174000000F7800D802A900D822A900D842A90029
:10175000D862A900D882A900E802A900E822A9005D
:10176000E842A9000000EB00000F78000E003700EF
:101770001E00780080004000C0EB21008080400007
:101780000000EB00800878001E0078000000400098
:10179000E6004000C0EB2100808040000000EB002C
:1017A000800878001E0FE800200020009E0F100027
:1017B000EFFF3400020007000080FA00000006007E
:1017C0000000FA00DC02A800DC22A800DC42A8002D
:1017D000DC62A800DC82A8000080FA00000006009D
:1017E0000600FA00000F7800110798002207980001
:1017F0001E007800E0F588001E009000F0F58800DB
:101800002E00900000F688000000EB0010F6880023
:101810000000EB0020F688000000EB0030F68800A6
:10182000E1F58000F00F2000808F500001003A00A9
:10183000EC02A800F1F58000F00F2000808F50002E
:1018400001003A00EC22A80001F68000F00F200011
:10185000808F500001003A00EC42A800E0F58000C3
:101860000000E00001003A00EC02A900F0F5800061
:101870000000E00001003A00EC22A90000F6800020
:101880000000E00001003A00EC42A9000080FA00EC
:10189000000006000400FA00000F78001E00780027
:1018A000100798001E009000E10F50001300320056
:1018B0001E009000E20F50001F0032001E0090003A
:1018C0000000E0000100320029003700ECC2BF0038
:1018D0006140600000C0EA0061406000614160005A
:1018E000C12E200091407800E0CFB30000C060001E
:1018F00002407000ECE2B7001D003700ECC2BF00F0
:101900000080FB000000D1006140600000C0EA00E0
:10191000614060006140600000414000C12E200035
:1019200091407800D0CFB30000C06000024070004A
:10193000ECE2B7000E003700ECC2BF000080FB00F5
:101940004200DE006140600000C0EA0061406000CB
:10195000614060004201DD00C12E2000914078000E
:10196000B0CFB30000C0600002407000ECE2B700EE
:101970000080FA00000006000200FA00F0F6800085
:101980000000E800F0F68800F0F68000E80F500054
:10199000020034000000EB00F0F68800F0F6800052
:1019A000000F78001E007800E40F50003500320070
:1019B0001E007800E40F500011003C001E0078006B
:1019C000E10F5000200032001E007800E10F5000AF
:1019D00004003C001E0078000000E000150032000A
:1019E000410037001E007800E20F50001B0032005B
:1019F0001E007800E30F50001D0032003A0037004F
:101A00001E007800E60F5000280032001E0078000B
:101A1000E60F5000200035001E007800E70F500050
:101A2000270032001E007800E80F50002900320025
:101A30002D0037000001EB008000EB000000EB0000
:101A400067FF07002C0037000001EB008000EB006F
:101A5000F00F200062FF0700270037000001EB00B5
:101A6000510A2000F00F20005DFF07002200370020
:101A70000001EB00F10F2000F00F200058FF0700DD
:101A80001D0037000001EB00F10F20000000EB000B
:101A900053FF070018003700F20F2000F10F20005D
:101AA0000000EB004EFF070013003700F20F20008C
:101AB0008000EB000000EB0049FF07000E0037003C
:101AC000F20F20008000EB00F00F200044FF070021
:101AD00009003700F20F2000F10F2000F00F200066
:101AE0003FFF0700040037000001EB008000EB001F
:101AF0000000EB003AFF07000080FA00000006003B
:101B00000800FA000000EB00200798000000EB003E
:101B1000100798000000EB003007980001C3B300E5
:101B20000000EB00F8CF07004E00070020079800E8
:101B30002E009000E10F40004800320040EE2100EE
:101B4000104078000080FB00000F78001E00780035
:101B50004800DD00000F780050EE210010407800B2
:101B60000080FB001E0F40002E0090009E0F5000D2
:101B700029003A000000EB00100798000A00370027
:101B80009E00900020EE2100614078008080FB00E4
:101B90003E00900001004000300798001E009000B9
:101BA0000000E800100798002E0090008000E90077
:101BB0001E009000808F5000F1FF3C003E0090001E
:101BC00002102000110009000200D8008000FD0072
:101BD000300798002E0090008000E90020EE2100E0
:101BE000614078008080FB003E009000808F5000B4
:101BF00009003A0070C4B30003D7070020EE2100AB
:101C0000120020009E007800CFD7070070C4B300F8
:101C1000FDD607001100370020C4B300FAD6070034
:101C20000000EB0010079800070037001E0190002D
:101C300021EE21000040EB0000F178001E00900032
:101C40000000E800100798009E009000F01F2000A0
:101C5000808F5000F5FF3400AAFF37000080FA00A3
:101C6000000006000E00FA00881F78000000EB005C
:101C7000400798000000EB00300798000000EB00E0
:101C8000200798000000EB00100798003D00370087
:101C9000EFD807000004E0002300320019D8070045
:101CA000004F780010002000300798004E00900090
:101CB000E10F500017003C00CE0090006A00470082
:101CC000008040001E4878004E0090000000E000B8
:101CD0000C0032001E0490006A0047009040900003
:101CE0006A0047001040780080DA070080407800E2
:101CF00020EE2100017478001E0090000000E80032
:101D0000100798004E0090000000E800400798007F
:101D1000020037000000EB0040079800400120005F
:101D200030F38800DD020700BCD807000004E000A3
:101D300014003200DDD70700004F7800F0C4B30074
:101D40009E4F100003003A0010002000200798006A
:101D50000C00370030C6B3009E4F100009003A0057
:101D60002E0090000000E0000600320020862A00CD
:101D700007F0070065D607000080EB0060079800B9
:101D800008003700A0F280000000E000C0FF320031
:101D90003E0090000000E000BDFF32001E009000F9
:101DA000600798006E0090004F0478000080FA00F1
:101DB000000006000400FA00000F780011079800E8
:101DC0001E00780042D70700C0C2B3004FD60700FC
:101DD0001E0090003ED70700D0C0B3004BD60700CE
:101DE0000080FA00000006000200FA000040EB004C
:101DF000004F780002003700C2D707001E4FE800EE
:101E0000E0C0B3009E4F1000FBFF360090C4B3004B
:101E100022D80700D0F48800BAD70700B9D7070046
:101E20000080FA00000006000400FA00881F780015
:101E30000000EB00000F78000000EB00000F7800BE
:101E40000C0037001E00780080004000A0E1210057
:101E5000808040000000EB00800878009E00780041
:101E600060E42100808040000040EB008048780062
:101E70001E0FE800B00020009E0F1000F1FF34009C
:101E80000000EB00000F7800070037001E0078000C
:101E90008000400020E32100808040000000EB0033
:101EA000800878001E0FE800900020009E0F1000B0
:101EB000F6FF3400B0C4B30053D6070091D7070033
:101EC00090D707008FD707008080FB0000FD2F0010
:101ED00000804000B0F08800C0C2B300EFD7070018
:101EE000C0C2B300EDD70700B0F58800C0C2B30090
:101EF000EAD70700C0F58800C0C2B300E7D70700E3
:101F0000D0F58800C0C2B300E4D70700E0F4880031
:101F10000000EB00000F780017003700B0F08000E1
:101F20000000E00009003A001E047800C0C2B300BF
:101F3000DAD707000001780088004400A0E1210002
:101F400000804000020878000A003700B0F58000E9
:101F50001E0050000004E900C0C2B300CFD7070044
:101F60000001780088004400A0E1210000804000CA
:101F7000020878001E0FE800B0F580009E0F1000E8
:101F8000E6FF350003003700C0C2B300C3D7070027
:101F90001E0FE800B00020009E0F1000FAFF340072
:101FA0000000EB00000F7800090037001E047800E5
:101FB000C0C2B300B9D70700000178008800440010
:101FC00020E3210000804000020878001E0FE80096
:101FD000900020009E0F1000F4FF3400C0C2B30038
:101FE000AED7070047D7070046D707000000EB0031
:101FF000000F780043D7070020479800AE409000BC
:1020000070C4B30080CF50000E003A0010032000CF
:10201000C0F08800020037003AD707002047980038
:10202000AE40900070C4B30080CF5000FAFF320081
:10203000AE409000A0C4B30080CF5000F6FF320045
:102040005300370000032000C0F08800B0F080008B
:102050000000E0000F003A009E0078002E41900042
:1020600060E4210000804000024878001E017800F2
:102070002E4090008080FB0000FD2F0080814000FA
:1020800082004100E0E92100008040000308780060
:1020900010003700B0F580008000E9002E4190006C
:1020A00060E421000080400002487800B0F5800024
:1020B0000001E9002E4090008080FB0000FD2F0011
:1020C0008081400082004100E0E921000080400062
:1020D000030878001E0FE8002D00370009D707001D
:1020E000204798002E409000C7D50700AE409000D2
:1020F00080C4B30080CF500028003200B0F08000D0
:102100000000E0000F003A009E0078002E41900091
:1021100060E4210000804000024878001E01780041
:102120002E4090008080FB0000FD2F008081400049
:1021300082004100E0E921000080400003087800AF
:1021400012003700B0F580001E0050008000E9004A
:102150002E41900060E42100008040000248780099
:10216000B0F580001E0050000001E9002E409000F4
:102170008080FB0000FD2F00808140008200410034
:10218000E0E9210000804000030878001E0FE8000D
:10219000B0F580009E0F1000D0FF3500D9D60700A3
:1021A000204798002E40900097D50700900420000B
:1021B00050F688004F0478000080FA000000060006
:1021C0000601FA0090C6B30050D5070040C5B30021
:1021D0004ED50700C0F08000C9D50700D0C0B300BD
:1021E0004AD50700A0C0B30048D5070090C6B30089
:1021F00046D5070010C4B30044D50700A005200051
:10220000BFD50700D0C0B30040D50700A0C0B300C1
:102210003ED5070090C6B3003CD5070060C6B300AA
:102220003AD50700D0F48000B5D50700D0C0B30080
:1022300036D50700A0C0B30034D5070090C6B30060
:1022400032D50700E0C6B30030D50700D0F58000D6
:10225000ABD50700D0C0B3002CD50700A0C0B30099
:102260002AD5070090C6B30028D5070080C7B30061
:1022700026D50700C0F58000A1D50700D0C0B30067
:1022800022D50700A0C0B30020D50700D0F58000FC
:10229000000F78000F00370090C6B3001BD5070071
:1022A00040C6B30019D507001E007800800040002A
:1022B00020E32100008040001000780090D5070046
:1022C000D0C0B30011D50700A0C0B3000FD50700E0
:1022D0001E0FE800C0F580009E0F1000EEFF3500D5
:1022E00090C6B30009D5070020C6B30007D5070084
:1022F000D0F58000000F7800080037001E0078003D
:1023000080004000E0E921000080400010007800DB
:102310000043B000FDD407001E0FE800C0F58000A8
:102320009E0F1000F5FF3500D0C0B300F7D40700B2
:10233000A0C0B300F5D407000000EB00000F780048
:102340000F00370090C6B300F0D4070030C7B300C9
:10235000EED407001E00780080004000A0E12100BC
:10236000008040001000780065D50700D0C0B300A1
:10237000E6D40700A0C0B300E4D407001E0FE800B5
:10238000B0F580009E0F1000EEFF350090C6B30040
:10239000DED4070030C7B300DCD407008E80E8002D
:1023A00090C6B300804878008E80E80030C7B30044
:1023B00090409800B0F58000000040008040780018
:1023C0000E80E800214098000000EB00000F78002C
:1023D0001A0037001E007800000040006401400031
:1023E0001E00780080004000A0E121000080400035
:1023F00010007800804078000E80E8000000410066
:10240000014878001E007800000040006301400091
:102410001E00780080004000A0E121000080400004
:10242000100078004880DE00804078000E80E800D0
:1024300000004100014878001E0FE800B0F5800060
:102440009E0F1000E3FF35000000EB00000F780046
:10245000060037009E0078000E80E80000804000F3
:1024600010407800A9D407001E0FE8000E80E80095
:10247000204090000000FB00630040009E0F5000D1
:10248000F4FF3C00FFFF37000200FA00A0842A009E
:102490003FEE0700C0F080008040780040C5B300E8
:1024A00006D20700A0052000F5D8070080007800BC
:1024B00010C4B300E8D10700B0F58000F0D80700E1
:1024C0008000780030C5B300E3D1070021C3B3001A
:1024D00030C4B300F9D107000000EB00000F780012
:1024E0001E0037001E00780080004000A0E121009F
:1024F0000080400010007800E1D8070080007800DC
:1025000030C7B300D4D10700D0F48000DCD8070076
:102510008000780060C6B300CFD107001E007800AD
:1025200080004000E0E92100008040009000780039
:10253000D0F58000008040008000400020E32100B2
:102540000080400010007800CDD80700800078009F
:1025500040C6B300C0D107001E0FE800B0F58000F0
:102560009E0F1000DFFF3500D0842A0008EE070020
:102570000080FA00000006000000FA0000852A0032
:1025800053D5070046DEBF000004E000040032001F
:1025900060E421004ED50700070007000200370065
:1025A00030852A004AD50700D0C0B30057D40700B1
:1025B0000080FA00000006000200FA000000EB00B4
:1025C000000F78000000EB00000F780006003700D5
:1025D0009E00780060E42100808040000040EB0015
:1025E000804878001E0FE800B00020009E0F100009
:1025F000F7FF34000080FA00000006003600F80003
:10260000809FBE00829FBE00849FBE00869FBE004A
:102610003400F80010002000A00188000000FA003B
:102620008660A900C3ED0700110107000080FA00D1
:102630003400F9004F03BE004F02BE004F01BE0040
:102640004F00BE003600F900004006003600F800DA
:10265000809FBE00829FBE00849FBE00869FBE00FA
:102660003400F80010002000A00188000400FA00E7
:102670008760A9001FE1A9000000EB001007980087
:102680000000EB00000F780021F3800030F38000A1
:10269000808F500004003D0020F380000000E8001F
:1026A00020F388000200370010002000A0F288000C
:1026B00061F3800070F38000808F500004003D00C3
:1026C00060F380000000E80060F38800020037003B
:1026D00010002000C0F2880081F3800090F3800099
:1026E000808F500004003D0080F380000000E8006F
:1026F00080F388000200370010002000E0F288001C
:10270000A1F38000B0F38000808F500004003D00F2
:10271000A0F380000000E800A0F38800020037006A
:1027200010002000F0F288000000EB00000F78009D
:102730003E0037001E00780080004000C0EB210002
:1027400000804000100078000000E00036003400F7
:102750001E00780080004000C0EB21000080400097
:1027600090007800E00F2000808F50002E003C0089
:102770009E0078000180400066014000C0EB21000F
:1027800000004100100078000001E80001804000D6
:10279000E6004000C0EB2100008040000208780005
:1027A0001E00780000004000E6004000C0EB210061
:1027B00000804000100178001E007800800040007A
:1027C000C0EB21000080400010007800800F510015
:1027D00015003A001E0078002EFC07009E017800CC
:1027E0001E00780080004000C0EB21000080400007
:1027F00090007800F00F200001015000838041001C
:10280000C0EB210000804000020878001E00780024
:1028100000004000E6004000C0EB21008080400046
:102820000000EB00800878001E0FE8002000200068
:102830009E0F1000BFFF340010002000100798000A
:102840001E0090000000E0000500320000E82300B8
:10285000D00888000000EB00A00888001FE1A80055
:102860000080FA003400F9004F03BE004F02BE00A2
:102870004F01BE004F00BE003600F90000400600C8
:102880000000FA000000EB0000F388000000EB00FD
:1028900090F288000080FA00000006000000FA00B4
:1028A0000000EB0020F388000000EB00A0F288009D
:1028B0000080FA00000006000000FA000000EB00B3
:1028C00040F388000000EB00B0F288000080FA00BE
:1028D000000006000000FA000000EB0060F3880032
:1028E0000000EB00C0F288000080FA000000060043
:1028F0000000FA000000EB0080F388000000EB000D
:10290000E0F288000080FA00000006000000FA00F3
:102910000000EB00A0F388000000EB00F0F288005C
:102920000080FA00000006000000FA00C902A800BA
:10293000C922A800C842A800C862A800C9E2A8002D
:10294000C8C2A8009660A8006340A8006360A80001
:102950006180A8006300A8005580A9006F00A9004D
:10296000ADC0A800ADA0A800AD80A80050F825001B
:10297000F00888000000EB00A00888008760A9002C
:102980009760A8000000EB00D0F28800400620000D
:1029900010F388000071220030F38800800C2000C2
:1029A00050F388000008200070F38800E02E20001B
:1029B00090F3880080382100B0F3880010F3800085
:1029C00000F3880030F3800020F3880050F380008B
:1029D00040F3880070F3800060F3880090F380007B
:1029E00080F38800B0F38000A0F3880000E82300A3
:1029F000D00888000000EB00A00888001FE1A800B4
:102A00000080FA00000006000000FA005016800066
:102A10004200DE00610060000004E00002003200BD
:102A20009004200050F688000080FA0000000600A4
:102A30000000FA00501680004300DE0061006000D4
:102A40000004E000020032009004200050F68800EC
:102A50000080FA00000006000000FA00DC62A90015
:102A600010002000A0A088000080FA0000000600EE
:102A70000000FA00501680004600DE000000A200B0
:102A8000610060000004E0004F003200DC22A90079
:102A900080F08000610060000000E0001100320062
:102AA00090F0800001022000010060000000E000C2
:102AB0000C003A0090F08000700060000000E00020
:102AC00008003A0090F08000620060000000E00022
:102AD00004003A00E07B2A0038D4070012BEA800A8
:102AE00044E6070070F0800001002400010060004F
:102AF0000000E0003500320090F08000010021006D
:102B0000010060000000E00005003200607C2A0047
:102B10002AD4070020C0B30052DF07002B00370083
:102B200090F0800001002200010060000000E00041
:102B30000900320090F08000610060000000E000B9
:102B400005003200307D2A001CD4070040C0B300CD
:102B500044DF07001D00370090F0800001002400D2
:102B6000010060000000E0000900320090F08000E9
:102B7000610060000000E00005003200007E2A00D5
:102B80000ED4070070C0B30036DF07000F00370017
:102B900090F0800001002800010060000000E000CB
:102BA0000A00320090F08000620060000000E00047
:102BB00006003200D07E2A0000D40700A0C0B30077
:102BC00028DF070001003700DC22A8000080FA009F
:102BD000000006000400FA00000F78001FC1BF00CB
:102BE00001C8B300014060000004E00005003A00A5
:102BF00000E82300D00888000000EB00A00888004F
:102C00001FE1A8001E007800100798001E00900029
:102C1000E30F5000160032001E009000E30F50003A
:102C200004003C001E009000E10F50000B00320039
:102C30002E0037001E009000E50F500025003200E6
:102C40001E009000E50F50000E0035001E009000A1
:102C5000E60F500022003200240037000000EB0095
:102C600000F388001000200090F288001F00370059
:102C70000000EB0040F388000000EB00B0F2880099
:102C80001A003700D0F280000000E0000600320099
:102C9000CCA2A8009000200070F388000000EB0098
:102CA000D0F28800060037000000EB00B7DB070019
:102CB0000008200070F3880010002000D0F2880087
:102CC0000000EB0060F388000000EB00C0F2880019
:102CD000060037006702070005FF07000300370002
:102CE00010FEA9000000EB00A8DB07000080FA003E
:102CF000000006000000FA00ED02A800ECA2A90006
:102D0000E902A900E8A2A900EF02A8000080FA00E9
:102D1000000006000000FA0080F829006CD30700CC
:102D200000242400F10020003CCB0700C0F829005B
:102D300067D3070040062000B501070050F92900BD
:102D400063D307000080FA00000006000E00FA00BE
:102D50000040EB00404798000000EB00100798008F
:102D60000000EB00000F78004E0090000000A10072
:102D7000400798004E0090000010A1004007980006
:102D80000000EB0010079800070037001E019000BC
:102D9000210E22000040EB0000F178001E009000A0
:102DA0000000E800100798009E009000002020001E
:102DB000808F5000F5FF34000000EB00000F78001A
:102DC00080F8290042D3070000242400F1002000ED
:102DD00012CB0700C0F9290078D30700C0FA2900F8
:102DE00076D3070060FD290074D307000000370088
:102DF00097D407000004E00079013200C1D3070036
:102E0000604798004E009000610060000000E00004
:102E1000F10032004E009000620060000000E0000F
:102E2000ED003A006E4090000000FB006007980043
:102E3000E0042000EE009000808F50007A00320005
:102E4000E0042000EE009000808F500009003C005C
:102E5000A0022000EE009000808F5000D1003200D0
:102E600030042000EE009000808F50000A003200F5
:102E70005B01370050052000EE009000808F50006D
:102E80001700320080072000EE009000808F500075
:102E9000CA0032005201370000FF290047D3070063
:102EA00040002A0045D3070090012A0043D30700C1
:102EB00030032A0041D3070090042A003FD30700C3
:102EC000D0052A003DD30700E0062A003BD30700C7
:102ED0004E0090000010A00040079800400137000D
:102EE00060082A00FAD20700800C20004801070081
:102EF0000000E0003A013A0020092A00F4D207005D
:102F0000800C2000420107000000E00034013A007C
:102F100090092A00EED20700803E20003C01070005
:102F20000000E0002E013A0080F82900E8D20700F6
:102F3000800C2000360107000000E00028013A0064
:102F4000200A2A00E2D20700800C2000300107008E
:102F50000000E00022013A00000C2A00DCD2070049
:102F6000800C20002A0107000000E0001C013A004C
:102F7000F00D2A00D6D20700800C200024010700A3
:102F80000000E00016013A00500F2A00D0D20700DE
:102F9000800C20001E0107000000E00010013A0034
:102FA00050102A00CAD20700800C20001801070028
:102FB0000000E0000A013A00C0112A00C4D2070054
:102FC00000FA2000120107000000E00004013A00AE
:102FD00030122A00BED20700800C20000C0107002E
:102FE0000000E000FE003A00803E200008010700DB
:102FF0000000E000FA003A0090092A00B4D207006D
:10300000803E2000020107000000E000F4003A00CA
:1030100080F82900AED20700800C2000FC000700D9
:103020000000E000EE003A0000132A00A8D20700DA
:10303000800C2000F60007000000E000E8003A00E5
:1030400040142A00A2D20700800C2000F0000700E4
:103050000000E000E2003A0060152A009CD2070060
:10306000800C2000EA0007000000E000DC003A00CD
:1030700090162A0096D20700800C2000E40007007A
:103080000000E000D6003A00E0172A0090D20700C6
:10309000800C2000DE0007000000E000D0003A00B5
:1030A00000192A008AD20700800C2000D8000700EF
:1030B0000000E000CA003A00B01A2A0084D20700DB
:1030C000800C2000D20007000000E000C4003A009D
:1030D000401B2A007ED20700800C2000CC00070095
:1030E0000000E000BE003A00101D2A0078D2070060
:1030F000800C2000C60007000000E000B8003A0085
:10310000701E2A0072D20700800C2000C000070049
:103110000000E000B2003A0020092A006CD207004B
:10312000800C2000BA0007000000E000AC003A006C
:1031300090092A0066D20700803E2000B4000700F4
:103140000000E000A6003A0080F8290060D20700E5
:10315000800C2000AE0007000000E000A0003A0054
:10316000901F2A005AD20700800C2000A8000700F8
:103170000000E0009A003A0020092A0054D207001B
:10318000800C2000A20007000000E00094003A003C
:1031900090092A004ED20700800C20009C000700F6
:1031A0008F0037004E0090000000A10040079800FB
:1031B000F0202A0081D207008900370050F9290049
